:020000040000fa
:020000040001f9
:08e0000012f104000000000011
:020000040000fa
:020000040001f9
:10e224008f972100007f2400000188000000000077
:10e234000c00070000572600110020001100070001
:10e24400000020000000e000020032000000020094
:10e25400000000005a420200010000000040da0001
:10e264000000fe004440a900208620000000e000d9
:10e274000300320020002000a00188004440a800d0
:10e284000000060091018800800078000000eb0087
:10e2940015003700e280400032a0b4009101ba00ba
:10e2a400e280400032a0b4009102ba00e280400053
:10e2b40032a0b4000002eb00472bde00f507b200e9
:10e2c400602ce10004003a000059eb008301e900ee
:10e2d400fdff3e00040037006128e1000100320028
:10e2e4000082eb00040007001101ba000200e00004
:10e2f400e8ff3a00000006003159ba008301e90042
:10e304000c0032002159ba008301e90008003200f0
:10e314000400e00003003a00e280400032a0b400b0
:10e32400f5ff370011d9ba008301e900faff3a007a
:10e334008100e800e180400032a0b4000000060043
:10e34400aaf104000000000004f204000000000030
:10e35400881f78000204780073000700080040005a
:10e364004f04780000000600881f7800000478003d
:10e37400820178000101780088007800a01a2f003b
:10e3840070000700800078000000e0000200350003
:10e394000040eb0000f47800010078004f0478009e
:10e3a4000000060080007800010037000000e8004b
:10e3b4001004e000fdff3a000100500000000600d8
:10e3c400881f78000004780030ab80000000e00073
:10e3d4000100320000000100805621000048eb00db
:10e3e40000ab80000000e0000100320000000100ea
:10e3f4006140b80010ab880021ab88004f0478005e
:10e4040000000600881f7800020478004600070018
:10e41400080040004f047800000006000000fa00e5
:10e42400881f7800000478003fb99700ea815700fc
:10e434008000780040202f00420007008000780010
:10e444000000e000020035000040eb0000f478001a
:10e45400010078004f0478000080fa0000000600f4
:10e46400800178008002eb000100370084597800b5
:10e4740005035100828f52000900320065c2780002
:10e484008502e8000404e000f8ff3a008300780005
:10e49400068141008058eb00828f5000fdff3a0056
:10e4a4000000060080017800000178003140780007
:10e4b400005978000004e000fcff3a0003007800f3
:10e4c40000000600040037000204e0000a003200e5
:10e4d4000000e8008100e80010417800914f5100ed
:10e4e400f9ff32000081eb0010407800914f50009a
:10e4f40004003900020037000001eb00010037007e
:10e504001200200002007800000006008001eb00e9
:10e5140002003700817178008301e800828f510086
:10e52400fcff3a00000006008001eb000200370007
:10e5340061f079008301e800828f5100fcff3a000a
:10e54400000006006200fa00889fbe008a9fbe0099
:10e554000004be00020578008300780060f92f00f3
:10e564000f0040000501070088979f0099979f00be
:10e574000000eb00a09f9f009a4578000b80fb00f1
:10e584000000ea00cf04de0050c2b30080cf550083
:10e594000200320009047800010037000904e90090
:10e5a4000800e0000b0034001f9097000801780079
:10e5b4008a0078008f9197000300010090979f00d4
:10e5c4000000e000930032002f9897000000440000
:10e5d400a09f9f000905450050c2b30080cf55009d
:10e5e400040032000b04e000e3ff3a002f98970088
:10e5f400890037000000eb00809f9f00f0979f0088
:10e60400e0979f00d0979f00c0979f00b0979f000e
:10e61400c09f9f0009003700a055210000805000d2
:10e6240000004000e1542100e10078004f98970079
:10e6340001007000c09f9f000a05e8001a4478009a
:10e644008800fb00a0552100d1000700800078005d
:10e654000000e000f0ff3a00a0c2b300804f540075
:10e664000e003a00bf8897000180e900b08f9f0038
:10e6740010007800b09f9f000000e00005003d00fe
:10e684000000ea00b09f9f004f9897000020a00070
:10e69400c09f9f000a05e80010003700b19f9f004b
:10e6a40003fd2f00f4ff2700080037003f98970070
:10e6b400840f5000040032006a00b90000004100d9
:10e6c40003004000b09f9f000a05e8001a01fb0008
:10e6d40003004100e90f5000f4ff3600e0c2b3002c
:10e6e4009a4f1000040032000080eb00909f9f00be
:10e6f4008a0478001c0037008a04e800a0c2b30032
:10e70400994f100007003a00bf8897000180e90084
:10e71400b08f9f0010007800909f9f008a84e800cb
:10e72400110037000000eb00909f9f0003fd2f00b5
:10e73400f4ff2700080037001f989700840f50004b
:10e74400040032006a00b9000000410003004000e8
:10e75400909f9f008904e8001901fb000300410019
:10e76400e90f5000f4ff3600194478008800fb00dc
:10e77400a0562100860007000000e00002003a00d5
:10e7840000447800010037008904e800a87f9f0056
:10e7940080c6b300804f540004003a00994f14001f
:10e7a4000a003a006640500006003700c0c6b300b5
:10e7b400804f540005003a00994f140003003a00ba
:10e7c40065404000a07f9f008904e8000905e80037
:10e7d400c8fb2f000f04440060f92f000f00400015
:10e7e4008085e8008801780019417800800078006d
:10e7f4000b0078006f0007000000e00005003a00fd
:10e80400880078000b007800e70107000000e000b2
:10e8140059ff3d000080eb004f05be004f04be00d1
:10e824000080fa0000000600881f780030ab8000ea
:10e834000000e000010032000000010000ab800095
:10e844000000e000010032000000010080a180000f
:10e854000000e000010032000000010050a180002f
:10e864000000e00001003200000001008056210099
:10e874001004e00026003a0010ab800021ab8000b9
:10e884000004eb00d2602600930120009b080700df
:10e89400f2352f00e3c623000000410081804900c7
:10e8a4000804e800e80f5400f6ff3a0010ab8800b3
:10e8b40021ab880028432100d26026009301200068
:10e8c40010ab800021ab80008c080700f2352f00cc
:10e8d400e3c62300000041008180490010ab88009a
:10e8e40021ab8800009cbe00204b2100800f540007
:10e8f400f1ff3a0070a5800081a5800060a1880026
:10e9040071a1880011c0b30080562100014878002d
:10e91400d26026009301200010ab800021ab800060
:10e9240076080700f2352f00e3c6230000004100fb
:10e934008180490010ab880021ab8800c2422100cd
:10e94400120178007f0161004211dd0023432100a0
:10e95400030141001202be0064a1880075a1880071
:10e964000089be0060a1800071a180004008de0023
:10e9740000f0a1004f047800000006000200fa0035
:10e98400f1bf9f00010878000080fa000000060033
:10e99400040037000204e00001003a000000050012
:10e9a4000000e80010417800814f5100f9ff3a005f
:10e9b40000000600889fbe008a1f780000047800cb
:10e9c40001027800824478000305780070c6b30021
:10e9d400804f510021003c0000c0e900804f5100ed
:10e9e400de003d0072405000804f51004b01320068
:10e9f4000d003c006c405000804f51005e013c0013
:10ea040000c0e900804f5100d4003d0050c2b30063
:10ea1400804f5100550132007c404000804f51002e
:10ea240055013a00cd00370010c6b300804f5100a5
:10ea3400ca00320004003c0069405000804f51007d
:10ea44004d013a007200370030c6b300804f5100c8
:10ea5400180032000040e8000900370000c7b30086
:10ea6400804f51001e01320008003c0000c0e90044
:10ea7400804f5100e400320065003c0065405000c6
:10ea840080cf54003c013a000f00370050c7b30058
:10ea9400804f51005e00320063404000804f5100bf
:10eaa4005b00320065405000804f510032013a0053
:10eab4001a0137009180e900010a7800780090007b
:10eac4009171780032013700a8609000c0c6b3008d
:10ead40080cf50000a003a0094007800648050000f
:10eae400000a78001000be004f89de00cf91de00de
:10eaf4000002be000203780082037800130037008e
:10eb040010c7b30080cf500003003200a0c6b3008a
:10eb140080cf500006003a009400780068805000ce
:10eb2400000a78003002be002003be000700370050
:10eb34001480e900000a78001000780000027800d0
:10eb4400cfa2de000503780086037800049cbe0093
:10eb54000694be00a860900080c6b30080cf500029
:10eb64000e00320020c6b30080cf500005003a00ea
:10eb74000400fb00cf80de000101780082017800f0
:10eb84000a00370040c7b30080cf500003003200b2
:10eb94006640400080cf500006003a000400780030
:10eba400cf80de000101780082017800009cbe0065
:10ebb4000294be003800be002801be00e00f5000e1
:10ebc400e08f5800e00f5900e08f590003003d002a
:10ebd40078009000d1c2b3000a00370008109000fa
:10ebe4000018a3000300320078009000b1c2b30003
:10ebf400040037000008a30053003200780090009e
:10ec040001c2b300017578000000e8004d00370030
:10ec1400a8609000c0c6b30080cf500006003a0040
:10ec24009400780064805000000a78001002be004e
:10ec34006033b8001300370010c7b30080cf500012
:10ec440003003200a0c6b30080cf500006003a0093
:10ec54009400780068805000000a78003002be00fa
:10ec64002003be00070037001480e900000a780082
:10ec74001000780000027800050020000600200043
:10ec840007002000049cbe000694be00a86090000b
:10ec940080c6b30080cf50000e00320020c6b300ff
:10eca40080cf500005003a000480fb0001002000e2
:10ecb40002002000030020000a00370040c7b30010
:10ecc40080cf5000030032006640400080cf5000e7
:10ecd40006003a0004007800010020000200200031
:10ece40003002000009cbe000294be0008109000a7
:10ecf4000038a300140032003800be002801be0012
:10ed0400e00f5000e08f5800e00f5900e08f5900e9
:10ed14000d00320080c7b30080cf540003003200de
:10ed240080c5b30080cf540007003a0078009000fb
:10ed340001c3b300017578008000e80009f578008c
:10ed44000080e800700498007800900000004500fe
:10ed540060049800894078006d003700a860900036
:10ed6400c0c4b30080cf500006003a00940078007d
:10ed740068805000000a78005001be004000be00c8
:10ed8400050037009400780064805000000a780081
:10ed94001000be00d2080700009cbe000294be0012
:10eda400380090000000e00003003d00780090006f
:10edb400d1c2b3000a003700081090000018a30065
:10edc4000300320078009000b1c2b30004003700a1
:10edd4000008a300050032007800900001c2b300cf
:10ede400017578000000e800700498007800900035
:10edf400000045006004980089407800080078000d
:10ee04003301070064003700a8609000c0c6b30057
:10ee140080cf5000250032000a003c0064405000be
:10ee240080cf50002800320000c0e80080cf50009e
:10ee3400140032006840500080cf500022003a0095
:10ee44000a00370040c7b30080cf50001e003200d4
:10ee54006640400080cf50001b00320069405000e3
:10ee640080cf500018003a00060037001480e900f3
:10ee7400000a780010007800485c90000848780088
:10ee8400450037001480e900000a78001002780079
:10ee940068089000cf80de000101780082017800cc
:10eea400009abe000292be003b0037001480e900c5
:10eeb400000a78001001780068089000cf80de0016
:10eec4000089be00340037001480e900000a78008d
:10eed40010007800680c9000080878002e003700b5
:10eee4001180e9008008780010007800cf80de00ef
:10eef4000101780082017800009cbe000294be00eb
:10ef040078009000000045006004980081c7b300b9
:10ef140008007800170307001f0037001480e90079
:10ef2400000a7800100078006004980058099000e6
:10ef34000200e00002003d001afd0700090037004e
:10ef44008000eb0094040700800078000000e000db
:10ef54000300320068009000008050000100370078
:10ef640058089000100c98000b00370078009000af
:10ef74000275780006003700780090008000450094
:10ef84000904e00001003a0059c2b300894878003e
:10ef94000000e800700498000000eb004f057800c2
:10efa4004f04be00000006000400fa00889fbe0063
:10efb4008a9fbe008c1f7800000478000106780048
:10efc40070089000f800900001005000880890003c
:10efd400010050009808900001005000a80890001b
:10efe40001005000b808900001005000c8089000cb
:10eff400810550000002220090bf9f0000032300ff
:10f00400a0bf9f00081090000028a30018003a0039
:10f014000b00e000160034008b047800090578002a
:10f02400e28f5400020036002a002000020037005c
:10f034000900e0000b00340058009000c801900063
:10f044000a017800ee805700030001005004980084
:10f054000000e000960032006808900000004500bf
:10f06400600c98008a8454004240a900ebff3c00e5
:10f07400780190000200e0000b003400580090007a
:10f08400c80190008c00780003000100500498002f
:10f094000000e0008600320068089000f80090004c
:10f0a40001004000600c9800880c90000900e0000a
:10f0b4001500340009057800e28f54000200360080
:10f0c4002a002000020037000900e0000b00340091
:10f0d40058009000c80190000a017800ec805700a5
:10f0e40003000100500498000000e00070003200aa
:10f0f4006808900000004500600c98008a84540061
:10f104004240a900ebff3c00180990000200e00017
:10f114000b003400e800900058009000c8019000f3
:10f1240003000100500498000000e0006000320079
:10f13400680890009808900001004000600c980056
:10f14400a80c90000900e0001500340009057800bf
:10f15400e28f5400020036002a002000020037002b
:10f164000900e0000b00340058009000c801900032
:10f174000a017800ec805700030001005004980055
:10f184000000e0004a0032006808900000004500da
:10f19400600c98008a8454004240a900ebff3c00b4
:10f1a400380990000200e0000d003400e8009000ef
:10f1b400180890008080400058009000c80190001a
:10f1c40003000100500498000000e0003800320001
:10f1d40068089000b808900001004000600c980096
:10f1e400c80c90000900e0001500340009057800ff
:10f1f400e28f5400020036002a002000020037008b
:10f204000900e0000b00340058009000c801900091
:10f214000a017800ec8057000300010050049800b4
:10f224000000e00022003200680890000000450061
:10f23400600c98008a8454004240a900ebff3c0013
:10f24400081090000028a3001b0032000b00e0000f
:10f25400190034008b04780009057800e28f54000b
:10f26400020036002a002000020037000900e000f6
:10f274000b00340058009000c80190000a01780087
:10f28400ee80570003000100500498000000e000e5
:10f29400070032006808900000004500600c9800e8
:10f2a4008a8454004240a90003003400eaff370076
:10f2b4000080eb00010037000000eb004f067800ef
:10f2c4004f05be004f04be000080fa000000060097
:10f2d4008f04b000889fbe008a9fbe008c9fbe0032
:10f2e4008e1f7800f0b79f0081f79f005001be0089
:10f2f4004000be00f0979f00819f9f00929f9f0057
:10f30400a39f9f0010c6b3000ff19700804f5100d8
:10f314001600320010c4b300804f510013003200b5
:10f32400ffb19700530890000000e00003003d0087
:10f3340060002000d00998000c0037000000e000b5
:10f344000a003a0070c6b3000ff29700804f5200d3
:10f354000300320070c4b300804f520003003a002f
:10f3640010002000ffb29700d00a9800ffb0970069
:10f37400c0fa2f000f0040009103070080017800bd
:10f38400e20f500015003a0030002000ffb0970053
:10f394009008980010c6b3000ff19700804f5100f9
:10f3a4000a00320064404000804f510007003200e0
:10f3b4000040e800804f510004003200a14f2100ba
:10f3c4000040e800804f510001003a00e14f210065
:10f3d400ffb1970063009000160037000000e000c2
:10f3e40018003400300020007fb29700100a980003
:10f3f40010c6b3008ff2970080cf52000a0032008b
:10f404006440400080cf5200070032000040e80012
:10f4140080cf520004003200215021000040e80057
:10f4240080cf520001003a00615021007fb1970063
:10f434006200900031587800315878001148780003
:10f44400c601370014c6b3008ff2970084cf520070
:10f454000300320010c4b30080cf520013003a00fe
:10f464007fb09700600190008200780000c3b30071
:10f4740080587800ffb29700e102980080c7b3007b
:10f484008ff2970084cf52000100320080c5b30090
:10f49400804878000280e800ffb09700e000980000
:10f4a400710090000080e800f00098000300e00084
:10f4b40005003a00e3979f0064fb2f000f01420010
:10f4c40003077800a0013700a5502100e5b79f008d
:10f4d40010c6b3008ff0970080cf500005003200b3
:10f4e40010c4b30080cf5000a7003a00b2512100ed
:10f4f400e2b79f00ffb19700530890001e0220005e
:10f504000000e000010035000007e8000e02e800fa
:10f51400d4b79f006022b8006033b8007f90970092
:10f524008f9897001f999700af9997000b070700d2
:10f53400ffb097003102be002103be000000e000ce
:10f5440004003d000400be000601be0003f0a2005a
:10f55400020037000400be000601be00f0979f00c1
:10f56400819f9f00929f9f00a39f9f006f91970090
:10f5740064015100e2979f00c3fa2f008f8141007c
:10f584006a8041000048eb006b824100c4b79f00d1
:10f5940031003700c201200003002000e5fa2f00eb
:10f5a4000f804200320307007f9497008f9c9700de
:10f5b4001f9d9700af9d97000800be000a01be0082
:10f5c400eb0607000006be005fb19700670151001b
:10f5d400d2b79f004240a9000a0034001007070078
:10f5e4000002be000203be000800be000a01be0005
:10f5f4000e070700f0979f00819f9f00929f9f0036
:10f60400a39f9f00cfb19700678041007100200045
:10f61400050037006f6066004c6add004466de005a
:10f624000c067200c4eede00e00f5600e08f5e00b0
:10f63400050034008100e900e18f4000f5ff3a0045
:10f64400010037000060eb008100e900fdff3b0092
:10f6540067004000c0b79f00dfb297000500e000dc
:10f66400090034006022b8006033b8007f9097002e
:10f674008f9897001f999700af999700ed060700a0
:10f684000000e000c3ff3c0060fb2f008f0040003f
:10f694004fb19700010051000000e9008e0f5000a7
:10f6a40001003d00000778000e00e00003003d006b
:10f6b40073fb2f000f8141002c003700800f57008f
:10f6c40005003d000e80400010409000f3c0b300e0
:10f6d400e74f500001003c008041eb00c4fa2f00ca
:10f6e4000f0242000e0042006a0040008e007800c3
:10f6f400010037000000e9008100e90010417800b2
:10f70400834f5100fbff32000107e800efcf5100a7
:10f7140001003a000248e8000100e000030035005f
:10f7240075fb2f000f814200060037000e07e8002a
:10f734006f90970064004000e0979f0061fb2f00ea
:10f744000f8140008e0041008e01780003003700d5
:10f754001100fb006fb29700e44878008301e900d0
:10f764008100e9000300e000f9ff3d00ffb29700cb
:10f77400550890000000e000f3003d000e00e90091
:10f78400d00a9800f00037007f9497008f9c970070
:10f794001f9d9700af9d97006022b8006033b800aa
:10f7a4000800be000a01be006c0607000000e0006d
:10f7b40005003d000bf0a200f8979f00899f9f0071
:10f7c4009a9f9f00ab9f9f006f90970072592700ec
:10f7d4000280b900026a2800130020009a0607007c
:10f7e400e4005000e1979f0015003b00e380100007
:10f7f400c0ff2f00008460000800ea00e0979f002b
:10f804007f9097008f9897001f999700af99970062
:10f81400294b2100070037000808a3000300320029
:10f824003902be002903be00960607000884d100f1
:10f83400e88444000800e000f7ff3c001b003700a8
:10f844000100e0001d003400c0ff2f0000806000b4
:10f85400e0979f00000478006000b80002002000d8
:10f8640003ff2300294b2100070037000808a300e9
:10f87400030032003902be002903be0081060700de
:10f884000884d100e88444000800e000f7ff3c004d
:10f894000002be000203be007f9097008f9897007d
:10f8a4001f999700af999700eb060700f0979f0008
:10f8b400819f9f00929f9f00a39f9f00ffb097008e
:10f8c4005109900060c6b3008ff1970080cf5100ba
:10f8d400040032006100200060c4b30080cf5100f6
:10f8e40002003a006f929700ea00420001074100cb
:10f8f400f30f5700010034003e01200000c3b300a1
:10f90400e0779f0075fb2f008f824200b5b79f0000
:10f91400330037000800be000a01be0014060700c9
:10f924000006be00680757004240a9000e003400dc
:10f934003b0607000002be000203be000800be0032
:10f944000a01be00390607006022b80046782d007f
:10f95400771924004b060700f0979f00819f9f00b2
:10f96400929f9f00a39f9f003fb0970068044000b0
:10f97400890020000d003700a400200005002000ad
:10f984000c01be00e0fd2f000f004000b302070091
:10f994007fa897008fb097001fb19700afb1970071
:10f9a40004c3b300046441000006be00e00f560027
:10f9b400e08f5e00060034008904e900e18f440012
:10f9c400edff3a000200370000c3b3000064780082
:10f9d4008904e900fcff3b0068044400b8b79f00b9
:10f9e4000e00e0000b0034007f9497008f9c97007a
:10f9f4001f9d9700af9d97006022b8006033b80048
:10fa04000800be000a01be000a0607000000e0006c
:10fa1400c0ff3c00c5fa2f008f8242006a8042007a
:10fa2400bfb09700008050008001e9006f919700fb
:10fa3400e70041006b81420000c3b30001003700be
:10fa44000201e800924f1000fdff320074fb2f000a
:10fa54000f004200808040008280500000804100fe
:10fa640002025000e1979f00ffb29700d509900071
:10fa740060c6b3008ff2970080cf520003003200bb
:10fa840060c4b30080cf520002003a008100e80055
:10fa94000a00370050c6b3008ff0970080cf5000a3
:10faa400050032008000eb0050c4b3008ff29700d1
:10fab40080cf520001003a0011002000018741006c
:10fac4008e0f520001003d00040778000e00e00094
:10fad4001d003500840f570005003d00e2407f0003
:10fae40095c3b30040c3b30080cf500001003c0075
:10faf40005c3b3000e0041008000e9008e017800c8
:10fb0400010037008100e9008301e9001142780017
:10fb1400854f5200fbff32000307e80090c3b30097
:10fb240080cf520001003a008448e8000300e0005e
:10fb340005003d000201e9000e07e8006f90970000
:10fb44000000e800e0979f006f9297008e01780014
:10fb54008ff097007fb097005d0207004f07780091
:10fb64004f06be004f05be004f04be008f04b10017
:10fb7400000006002f03b000889fbe008a9fbe00cd
:10fb84008c9fbe008e1f780000077800d0532100a0
:10fb9400c0b79f0080c5b30080cf5000080032007a
:10fba400c2522100c2b79f007740400080cf50006e
:10fbb40003003a0083002000b3b79f000a00370017
:10fbc40080c7b30080cf500005003200a40020009d
:10fbd400b4b79f0080c5b30080cf500002003a0044
:10fbe40005012000b5b79f003e04be002e05be00ef
:10fbf40040c6b30080cf500003003200654040008f
:10fc040080cf50000b003a00e00f5400e08f5c00fe
:10fc1400e00f5d00e08f5d0006003d006000b8006d
:10fc24006011b80008045000898458000a0559007e
:10fc34008b855900bfb39700e88f5300030032004f
:10fc4400f08f530045003a000200370036002000d0
:10fc54000100370046002000e00f5400e08f5c00f4
:10fc6400e00f5d00e08f5d0005003a005e08900043
:10fc740081012000a1b79f000000e00008003200cd
:10fc84003fb197000200e90008006000cfb197007f
:10fc94006340780090df9f0074012000a4b79f00a8
:10fca400860278008502e900050033008b05d10047
:10fcb4000a85d3008984d3000884d300f9ff370070
:10fcc400089fbe000a97be00afb397000700e90083
:10fcd40021fc2f008f804000008240003fb197003c
:10fce4008202e90012003700afb397008703e900ee
:10fcf400a7b79f0000806200cfb0970061527800e0
:10fd04003e00be002e01be00860378008703e90092
:10fd1400050033008381d1000281d3008180d300a8
:10fd24000080d300f9ff3700009fbe000297be0099
:10fd34003e00be002e01be00e00f5000e08f5800d0
:10fd4400e00f5900e08f5900d6003400afb397009c
:10fd54000700e000e4ff3c00d2003700ae609000f2
:10fd640080c6b30080cf50000b00320006003c0078
:10fd74000104e000080032006640500080cf5000cb
:10fd840073003a0004003700c0c6b30080cf5000af
:10fd94006f003a0031003700080178000800e000e5
:10fda40005003a005e08900081012000a1b79f0081
:10fdb4000000e00009003200bfb197001100090003
:10fdc4000381d8008000fd004fb2970064407800a2
:10fdd40090df9f0075012000a5b79f00bfb3970077
:10fde400110009000781d80080017800afb09700a6
:10fdf4000100e90022fc2f000f0141000002410034
:10fe04000c003700bfb29700110009008501d8002b
:10fe140000017800afb397008703e900a7b79f00fc
:10fe24000590b90000805100cfb09700615278006e
:10fe3400820178000300e000030034002fb1970032
:10fe44000200e000efff3c0003007800cf80de00fa
:10fe540001017800820178003a0037000806be00ec
:10fe6400e00f5400e08f5c0005003a005e0890004b
:10fe740083012000a3b79f000000e00009003200c6
:10fe84003fb297006121b9000c00be00cc05070009
:10fe9400cfb297006540780090df9f007701200083
:10fea400a7b79f003fb297006121b9000c00be00c4
:10feb400c60507000006be00afb297000500e900c2
:10fec40027fc2f008f8343008083430097b79f0054
:10fed400110037003fb197006114b9000801be005a
:10fee4000c00be00d80407000005be00afb19700a7
:10fef4008301e900a3b79f000801be00ff020700c9
:10ff0400000056001fb29700cfb2970065527800e8
:10ff140094b79f000a06be00e00f5600e08f5e0013
:10ff240003003400afb397000700e000e9ff3c0092
:10ff34004feade00cfa2de000c00be000401780010
:10ff440084017800009fbe000297be005500370070
:10ff5400e00f5400e08f5c00e00f5d00e08f5d0077
:10ff640005003a005e08900081012000a1b79f00bf
:10ff74000000e0000d0032003fb19700020278005b
:10ff8400cfa2de0005037800860378000800be00d7
:10ff94000a01be001e0607004fb2970064407800b5
:10ffa40090df9f0075012000a5b79f003fb1970027
:10ffb40002027800cfa2de000503780086037800f1
:10ffc4000800be000a01be000a060700009fbe002a
:10ffd4000297be00afb197000300e90024fc2f0094
:10ffe4000f0242000006420020003700bfb2970013
:10fff40005047800cfc4de00090578008a0578007e
:020000040002f8
:100004000802be000a03be005fa89700efa897008d
:100014007fa997008fb1970001060700d0b79f0012
:10002400e1b79f00f2b79f0083bf9f00afb3970073
:100034008703e900a7b79f000802be000a03be00b9
:100044007d0607005faa970000005200cfb2970018
:10005400655678005fb09700efb097007fb19700c6
:100064008fb99700009fbe000297be003e00be00fd
:100074002e01be00d0af9f00e1af9f00f2af9f0002
:1000840083b79f00e00f5000e08f5800e00f590045
:10009400e08f590003003400afb097000100e00086
:1000a400d2ff3c003fb19700e80f510013003a0023
:1000b4000e1090000038a30010003200afb197007a
:1000c400f78f510006003e0024fc2f000f0242006f
:1000d400e4c0790000c3b30080cf500007003200b1
:1000e400afb297008502e900a5b79f0000c3b30033
:1000f40027fc2f008f83430080f37a00afb1970071
:1001040078811100120f98006e00900024fc2f00db
:100114000f0242008300420003f907001e09900009
:100124005e089000800f510006003d000200500060
:10013400000f98000e1090000040a10000179800d6
:100144000f0037000000e0000d003d000e1090008d
:1001540074006000f00f500009003a007e0890001f
:10016400fe009000010050008e0890000100500035
:10017400020050004240a90001003400000f980022
:100184004f0778004f06be004f05be004f04be0067
:100194002f03b100000006008001eb0004003700cb
:1001a4008301e80090cf1000040032000000e80052
:1001b400828f5100faff3a000000eb0000000600b5
:1001c400889fbe00800478006684400000ff2700fa
:1001d400180060004401de00f07f2000800f510011
:1001e4000e003a00800ceb00180478006f006400e5
:1001f4001c003a00210090000000e00019003a00c1
:10020400110090000000e00016003a0010002000e9
:100214001100e00014003200120037000200e00078
:1002240005003c0001007800dd01070000017800b2
:100234000000e00008003c00f00028001800600006
:1002440001fe2300010c700020c02f00800c41002f
:100254000080eb0004003700800ceb000000eb0092
:1002640001003700200020004f04be0000000600fb
:10027400889fbe008a1f78008c9fbe00000478000f
:100284000206be00e6044000190178000200d00016
:100294004505de008a007800f07f2000800f5500bd
:1002a4000c003a006f00610067003a0028009000db
:1002b4000000e00064003a00180090000000e00034
:1002c40061003a00100020001800e0005f003200d6
:1002d4005d0037000a00e00007003a0008007800db
:1002e400af010700800078000000e0000200340045
:1002f4000a007800550037006108b9000c0140007d
:100304008d814800e07f2000800f5100e08f59006c
:100314000d0034001900e00004003d006000b80046
:100324000200200003ff2f00030037006000b80024
:100334000200200003ff2700009cbe000294be00c0
:100344001000200041003700e00f5100e08f5900f9
:1003540005003400f000280019006000c410dd001e
:10036400810c700036003700190078000100280065
:10037400010360006f0060000040a000800c780062
:1003840061015100e0815900c0fc2f00f1ff2f00f2
:10039400800f5100818f590006003d00860c7800c3
:1003a4000000eb002004980010049800000c780072
:1003b40026003700020078000881e800e4004400c9
:1003c40005003700120c78001109780099087800ac
:1003d400800ceb0070004000f00f4000f9ff340087
:1003e4008002ea00150032008881e8007082120061
:1003f400980078008508de00130078000400dd0012
:10040400008c700064014400930078008508de00cd
:10041400120078000400dd008089700092007800ea
:100424008508de00190078000400dd0000897000f2
:10043400190078000500de00800c7800990c730028
:100444000080eb0001003700200020004f06be00b2
:100454004f0578004f04be00000006000400fa00b7
:10046400889fbe008a9fbe008c1f7800000678001b
:1004740092bf9f00a3bf9f000404be000401be00fe
:100484001fb89700afb897006f0307000005be00c0
:100494000001be000800be00980107001fb99700c4
:1004a400afb99700000051008180590020069800e0
:1004b400310698000a8ebe000c0078004f067800c2
:1004c4004f05be004f04be000080fa000000060085
:1004d4000e00fa00889fbe008a9fbe008c9fbe005b
:1004e400000478000145780002067800830478004f
:1004f400840678000300e00002003c00190020009c
:100504004c57210060c6b300804f55000e003200e6
:1005140060c4b300804f55000b00320070c6b300b6
:10052400804f55000300320070c4b300804f550063
:100534009c003a00e48f4600800035005808900083
:10054400808f56007d003d008d05e80060c6b30035
:10055400804f55001000320060c4b300804f550036
:100564000d003200081090000038a30004003a0087
:1005740058089000808f540001003d00590c9800e9
:10058400580890000b005000500c980002003b00eb
:100594000000eb00500c98000b00e00027003c002a
:1005a400180990006800900001c3b300017079003d
:1005b4008201e800130c9800580890000000e00045
:1005c40003003c00081090000038a300050032002e
:1005d40068009000e1c2b30001f079000280e800f5
:1005e400100c9800d80890000b00ea00808f50008f
:1005f40001003d008105ea000b00ea00200c980090
:1006040001804500500c9800890f500001003d0006
:1006140080047800390c98006800900098089000d5
:1006240001004000090178008c007800bef7070043
:1006340058089000090050001a00370098089000ec
:10064400680090008b8f540018003d0001004000aa
:10065400090178008c007800b3f7070018089000af
:1006640000814400120c980009805500200c980069
:10067400580890000000e00003003c0008109000bf
:100684000038a30006003200e8009000e0c2b30086
:1006940080707900380890000000e800300c980061
:1006a40058089000400c9800a60037000100400054
:1006b4000b0178008c0078009bf707001808900065
:1006c40000814500120c98008b8454005808900057
:1006d4000000e00003003c00081090000038a30074
:1006e4000500320068009000e1c2b3000170790097
:1006f4000200e800100c980058089000890f500080
:1007040001003d0080047800680090009808900083
:10071400010040008b0046000901780082f70700c1
:100724001808900000804400100c980058089000ad
:1007340009005000200c98008200370070c6b300f6
:10074400804f55000300320070c4b300804f550041
:1007540014003a0058089000808f540004003d00b3
:10076400081090000038a30001003a00590c9800ca
:10077400580890000000e900500c980002003b006b
:100784000000eb00500c980070c6b300804f550079
:1007940002003a005ac6b3000b0037005ac4b30033
:1007a4000900370010c6b300804f550002003a001c
:1007b4000ac7b3000400370010c4b300804f5500cb
:1007c40001003a000ac5b3001809900068009000bf
:1007d4003c7079008201e800130c98000c02780048
:1007e400580890000000e00003003c00081090004e
:1007f4000038a30017003200e8009000e0c2b30004
:1008040080f079008280e800110c9800580890006c
:100814000000e0000f0034008904e900890f500053
:1008240001003d00800478006800900000804000d2
:1008340009017800840078003bf70700180890004d
:1008440000804400100c98005808900009005000e3
:10085400200c980068009000980890000100400067
:100864000086e8000a587800800078000d00e00057
:1008740004003500b0c2b300804878008c047800ce
:1008840004003700d0c2b300804878008c0478009c
:100894008d06ea008005eb000a003700a200200064
:1008a4008d00780070805700890007000fb897000a
:1008b4009fb897007a81550001f17f008b05e8000d
:1008c400800678000d00e000f4ff3c00e18f550045
:1008d40009003c0050c6b300804f550003003200ad
:1008e40050c4b300804f550003003a0000c3b30066
:1008f400005e78008c0478000b00e00004003200f5
:100904000b00e900fa805700008040000600370021
:1009140000c3b300805c7800050037008b05e90054
:1009240002c3b300a05c41000b00e000fbff3c00ed
:100934006800900098089000010040000080540076
:10094400300c98000810900074006000f00f500004
:100954000e003a00780090009808900001004000d2
:10096400a808900001004000b80890000100400071
:10097400c80890008100400078089000808f5000e3
:1009840002003d0001005000000c98004f06be001c
:100994004f05be004f04be000080fa0000000600b0
:1009a40000017800e60140001300780001002800ef
:1009b400810360006f0060008009780012003a0033
:1009c400220090000000e0000f003a0012009000a6
:1009d4000000e0000c003a00160020001200e000c5
:1009e4003800320008003700e40041009109780023
:1009f4000280e80090087800120878000009eb00f3
:100a04007003530001003700160020001300e000bb
:100a1400f5ff3200e40241000282e80011003700d1
:100a240080004000150078004f00de0080897000cf
:100a34009500780081804000140078004f00de00ab
:100a4400808a700094007800818040001200780051
:100a54004f00de00008a7000120078000009400098
:100a64000603e90013007800ef0f5000ecff360096
:100a74008282e800640241000e0037009200d10037
:100a8400150078004f00dd00008970009500d1004a
:100a9400140078004f00dd00808a70009400d100bb
:100aa400130078004f00dd00008a70009309d10024
:100ab4000603e80013007800ff0f5000efff3e002c
:100ac400ef096000938973000600780000000600b7
:100ad40002027800809fbe00110009008200d80045
:100ae400000178004f00be0002a2b90084805000cb
:100af400110098000208780000000600020ab900fc
:100b0400001bb9000200b8008100420081004300cc
:100b140000000600889fbe008a9fbe000105780081
:100b24000100e0000400350008003c000000e00083
:100b3400200032000500370060001000e08018003b
:100b440002003b0001f02c001a0037000004be0034
:100b54006011b8006b0920000982cf00020039003f
:100b64000882cf000441b000694252000e003200f6
:100b740008003b0082817100610164008904d10096
:100b84000884d3008b05e8000442e800f9ff3a002a
:100b9400050037000804440089844c008b05e900f3
:100ba4000442e900fbff3a00fa0007000af0a7003c
:100bb40001f0a0004f05be004f04be000000060077
:100bc40003f0a200889fbe008a9fbe008c1f78009d
:100bd400160107001d0133006450e1004f0032008c
:100be4006420e1005200320003826c0007003b00e5
:100bf4000905d0000306d000820f54000c065d00e6
:100c040002003900020032008901780003067800ee
:100c14008582550004003d000003fd008103fd00b2
:100c24008502ea008b854200840f720002003b00bb
:100c340060001000e08018006011b8000005eb00af
:100c44007a28e1000a00390006007800c75ddd005b
:100c5400f707b200878075002d003700828171008c
:100c64000a017800610560008180d1000080d30012
:100c74008502e900f9ff3b00060440008784480030
:100c840002003b0060041400e0841c000988a300f7
:100c9400070032008a817100828171006101640061
:100ca4008904d1000884d3008b05e80017003700bd
:100cb4000978a30013003a000b00e000130034008d
:100cc4008b05e9000804440089844c000a4474003c
:100cd4000978a3000d003a000b00e000070034007f
:100ce4008b05e9000804440089844c0001003a00a3
:100cf4000b0020000978a300f7ff32000001eb008d
:100d040002003700828171000a017800a100070007
:100d14000cf0a70001f0a000d50037006420e1002a
:100d240002003a00838f6c00d50033000801be0036
:100d34000200be00ce003700889fbe008a9fbe001e
:100d44008c1f7800b9000700c000330003866c00d4
:100d54006450e1002e0032006420e10033003200d0
:100d64006150e1002f0032006120e10031003200c7
:100d740085855500eb07b000090020000804200019
:100d8400050037000804440089844c000a0031003f
:100d94000603430087834b000001530081815b00fd
:100da400f8ff33000203be000800a000080444005a
:100db40089844c00f6ff3900c639dd0083017300d5
:100dc40001003200130020008904d1000884d300fc
:100dd4000998a300050032000800a7000300a00042
:100de4008904d1000884d3008b05e8008904d1006c
:100df4000884d3000001eb000281d20065000700e3
:100e040001f0a1000cf0a70001f0a0009800370049
:100e14006420e1009a0032000801be000200be0016
:100e2400f7ff37006120e100950032006000b80050
:100e3400f3ff37000000200001f82700f0ff37001f
:100e4400889fbe008a9fbe008c1f78007700070031
:100e54007e00330003866c006450e10024003200fd
:100e64006420e100270032006150e10022003200da
:100e74006120e100210032008b854200eb07b100c4
:100e84000134b800003ab8000804420089844a00da
:100e9400013ab8000030b8008880400009014a00d7
:100ea4000400330000004000818048000201490032
:100eb4008b05e900c909dd008301700001003200df
:100ec40013002000c814de004814dd004709de00ca
:100ed4001200b200c808de00088470002d0007006c
:100ee40001f0a1000cf0a70001f0a00060003700a1
:100ef4006120e100620032000801be000200be0071
:100f0400f7ff37006150e100fcff3a005c00370056
:100f14000001be005d0007000470a70003f0a100fb
:100f24006509b100160032000d0035006828e100a3
:100f340006003500f0ff2f00f1ff27000300e0005a
:100f440013003b00010028000000050000004000e1
:100f5400818048008502e900fcff3a000800370060
:100f6400f88f420002003c008000eb000000050006
:100f74008100d1000080d3008502e800fcff3a0024
:100f84000300e00002003b0060001000e080180055
:100f94000000060081002000618055000b003d0028
:100fa4000b00200061fe2f000100e1001d00340051
:100fb40082817100610164008904d1000884d30036
:100fc4000000e800faff3a007100200061006400ac
:100fd4000300700002006000090032006104440054
:100fe400e0844c000988a500050032008b05e80068
:100ff4006808e10002003a008904d1000884d300a3
:10100400f20f20000258e10005003d00c75ddd003d
:10101400f907b20089807500080078000000060016
:101024000bf827008b007800000005000004be00c8
:10103400160007000003be000405be000200be0047
:1010440012000700844f7500000006000200be0075
:101054006450e100050036006420e100020036001f
:101064000968a30001003a000800be000160a00066
:101074004f0678004f05be004f04be000000060076
:10108400f0ff2f00f1ff2700f9ff3700c70ade0049
:10109400f107b200f50fb20008003200e1cf4200c0
:1010a400020032000170a00024000500810f7000ce
:1010b400010032000408050044000500810f70009f
:1010c40002003a00140005008502e9000000400017
:1010d40081c04800fcff3b000170a0002400050013
:1010e40081037800e9ff07000001be006000b8003a
:1010f4000478a30013003a006220e10015003e00ca
:101104000d0039008301d1000281d3008180d30016
:101114008301d1000281d3008180d3008301d100f7
:101124000281d3008180d3000538b000c42add00d9
:10113400f300b2008381720007f0a70003f0a0005f
:1011440000000600f3ff2700f2ff2f006110b90032
:10115400fbff370003ff2700f7ff37008f1fd10085
:10116400630207008f87e9000000e000000006002a
:101174001400fa00889fbe008a9fbe008c9fbe00a8
:101184000004be000205be00680047000a90be00cd
:101194000890be007f0207000070a7000bf0a100ba
:1011a400304320009e02900080825200b0fe2f0047
:1011b4000028e10011003d00b0fc2f000028e100f0
:1011c400150034001e0990008e0890007e009000e7
:1011d4000501b0000201d1008180d3000080d3005a
:1011e4008502e800fbff3a000b00e000a4023b008c
:1011f40060001000e0801800a1023700f0ff2f000b
:10120400f1ff27000b00e0009d023b0001002800d5
:10121400000020009a0237006000b80098023700ee
:101224004f89de00820178009a02370007f0a2009d
:10123400cf023700809feb002d0207008f87e90063
:101244000000e00000000600839f68000100e00049
:1012540002003d0060001000e08018000300e00080
:1012640002003d0060011100e0811900d700070071
:101274004f00e00002003b0060001000e080180016
:10128400000006002800fa00889fbe008a9fbe0066
:101294008c9fbe0003866b00650207000028a30034
:1012a40064003a000128a30067003a000008a30084
:1012b40062003a000108a30065003a001e00900095
:1012c400be08900081064000ed3fb100f480570055
:1012d400ee019000111ab8008e099000311bb8007d
:1012e4009e099000311cb800511db800f4855700c8
:1012f40046000700fe0190003a0007008b85e800d5
:101304003e0007008e09900040000700ee019000a7
:10131400340007008b85e800380007008e09900030
:10132400400007009e0990001b18b8008904400083
:101334000a854800fe019000340007008b85e80010
:1013440038000700ee019000300007008e0990007d
:101354001b18b800890440000a8548000a98a300b5
:1013640008003a000402420085824a0006034b004a
:1013740087834b0008044c0089844c000a054d0007
:101384008d06e90084827200850273004c3add0008
:10139400850272000100320015002000443ade008c
:1013a4001400b2004538de00cb45dd000b007000b0
:1013b400c540de00cb4ddd008b8070004549de006a
:1013c400cb55dd000b017100c551de000d03780023
:1013d400e402070003f0a1000cf0a70003f0a00052
:1013e400270237001b18b800850240000683480016
:1013f400e0834b0060044c00070037001b18b80062
:101404000603400087834800faff37001b18b80022
:101414008703400008844800e0844c0060054d00c8
:10142400000006001b18b800080440008984480026
:10143400faff37000108a3000e023a005800be006c
:101444005801be00e3ff37000008a30009023a0078
:1014540009047800f9ff37002800fa00889fbe00cd
:101464008a9fbe008c9fbe0003866b00f0010700bc
:101474006400e100440032006408e1004a003200e4
:101484006100e100460032006108e10049003200d9
:10149400ec0647006000b8003d02be003d03be00fc
:1014a400f48657006011b8003d04be003d05be003f
:1014b4007d0320000b0037000000a0008d06e9002a
:1014c400130032000402420085824a0006034b00e6
:1014d40087834b00000040008180480002014900de
:1014e400838149000802520089825a000a035b0082
:1014f4008b835b00f0ff3b000802420089824a00b4
:101504000a034b008b834b008d06e900edff3a0084
:101514008482720086827200f707b20087827200aa
:1015240001003200150020001e0490003e0b9000c4
:1015340006035400e63fb0000368a300070032002e
:101544000000a7000500a0008301d1000281d300a0
:101554008180d3000080d3000603e8008301d1001a
:101564000281d3008180d3000080d3000002eb000d
:101574000482d2007b02070003f0a1000cf0a70054
:1015840003f0a000be013700640247006408e100d4
:10159400b80132003400be003401be00f6ff37004b
:1015a4006108e100b30132006011b8006000b800c6
:1015b400f1ff370003ff270002002000fbff370084
:1015c400020007000400be00000006006022b8000c
:1015d400060220000000d0008180d2000482d200e4
:1015e4008582d2000000a0000202520083825a00c9
:1015f400030031000202420083824a000000a1007d
:101604000603e900f3ff3a0000000600881f780093
:10161400000478005001be004000be0004004000f9
:10162400858048000601490087814900009cbe006e
:101634000294be000400e1000588e1000690e10088
:101644000798e10002003100680044001008e80037
:101654004f04780000000600f4874700889fbe000e
:101664008a9fbe008c9fbe008e1f78000205be00bc
:101674000004be00d4b79f00e5b79f00f6b79f00f3
:1016840087bf9f000000eb00c0b79f00b0b79f006a
:10169400a0b79f0090b79f0080b79f000d04200063
:1016a400bfb097004fb09700000140000000e00079
:1016b4000f003d004f08de0000007100c0b79f001e
:1016c4009e00070001003d0012002000a100070059
:1016d40001003d0012002000a6000700b100070031
:1016e400b60007000f004000c8ff070022003700c3
:1016f4004f08de0000067100ccb79f008f00070082
:1017040001003d00120020009200070001003d008e
:101714001200200097000700a20007000fb29700f4
:101724009fb297002fb39700bfb39700a90007009b
:101734000000520081805a0002015b0083815b003b
:1017440080b79f0091b79f00a2b79f00b3b79f00d7
:101754000007eb009f0007000020e10001a8e10062
:1017640002b0e10003b8e100010031001e002000d6
:101774000e005600c0b79f004fb297000400e0006f
:101784000700350010002000010020006011b8009f
:1017940008047000898470000a0571008b8571004b
:1017a4008d06e900beff3a000400e00003003d009e
:1017b400820007000f00400094ff07004fa8970025
:1017c4000000e00004003a000fb497009fb49700b3
:1017d4002fb59700bfb59700940007004f07780016
:1017e4004f06be004f05be004f04be004f01b100be
:1017f40000000600881f780018002000881f780069
:1018040095ff07008f87e9004f0478000000060069
:10181400801feb0090ff07008f87e900000006009f
:10182400889fbe008a9fbe008c1f78006e00070050
:1018340007003d0073000700e00f5b00e08f5b00d2
:1018440007003d00320007000006eb0004003700eb
:101854003400070002003d002a0007001c0020009d
:1018640072000700e3ff07000203be000002be008f
:101874000c00e00001003200220007000400be005a
:101884000601be004f0678004f05be004f04be009f
:1018940000000600889fbe008a9fbe008c1f78004f
:1018a4005100070005003d0056000700e00f5b00f3
:1018b400e08f5b0006003d000400370019000700bc
:1018c40003003d006000b8006011b800100007007c
:1018d40056000700ceff07000203be000002be0050
:1018e4000c00e00001003200060007000400be0006
:1018f4000601be004f0678004f05be004f04be002f
:10190400000006006000b8006011b8000000370055
:101914000402500085825800060359008783590049
:10192400000006000006eb00e00f5200e08f5a00b2
:10193400e00f5b00e08f5b000000060001804000c8
:1019440090b79f000001eb008fb097000100e0000a
:10195400000006000200700090b79f000180400064
:1019640080b79f000001eb00ffa897000100e00092
:10197400000006000200700080b79f000180400054
:101984006faa9700cf20de0001007000f0af9f0027
:1019940004024200250007004f18de000002720016
:1019a40000000600e4af9f000804440089844c0052
:1019b4000a054d008b854d00000006003fb29700dc
:1019c400cfb297005fb39700efb3970000fe2f00ec
:1019d400000006003fb09700cfb097005fb19700ba
:1019e400efb19700000006000205be000004be002f
:1019f400e00f5000e08f5800e00f5900e08f5900cd
:101a0400000006006000b8006011b800080450002f
:101a1400898458000a0559008b8559001c00200050
:101a2400e00f5200e08f5a00000006000800be00dc
:101a34000a01be0000000600889fbe008a9fbe0007
:101a44008c1f78000205be000004be000006eb00f7
:101a5400e00f5000e08f5800e00f5900e08f59006c
:101a640007003d006000b8006011b8000804500091
:101a7400898458000a0559008b8559001c002000f0
:101a8400e00f5200e08f5a00e00f5b00e08f5b0034
:101a940002003d000f0007000c00a2000800be0079
:101aa4000a01be005b0107000203be000002be0083
:101ab4000c00e00001003200060007000400be0034
:101ac4000601be004f0678004f05be004f04be005d
:101ad400000006006000b8006011b8000402500065
:101ae40085825800060359008783590000000600c8
:101af400889fbe008a9fbe008c9fbe000404be0067
:101b04000605be00809fbe00829fbe0063010700e1
:101b1400040678000800be000a01be005f01070049
:101b2400840678004f03be004f02be008d4f76003e
:101b34007fb0970013003300f0ff2f008b8f6b00f2
:101b440006003b000d0666000c00a7000a003700e3
:101b540007f0a600100020000a003700880f52008a
:101b6400898f5a008a0f5b008b8f5b00030039005a
:101b74001000200001003e000000200007f0a70034
:101b84000000ea004f06be004f05be004f04be0031
:101b940000000600800078005002be005003be0022
:101ba4004439de00f700b200f37f20000301610036
:101bb400090032000218e10016003a0085017200a3
:101bc40083017300838173000008200015003a002c
:101bd4004000200013003700850172008301730068
:101be4008381730005003a0004a8be0006a8be0065
:101bf400100020000b0037000201e900040242003b
:101c040085824a0006034b0087834b000748a300e4
:101c1400f9ff32000740a00004a8be0006a8be00d9
:101c24002000200080009800920098000000060028
:101c3400680447000294be000094be00fc04470000
:101c44008694be008494be0009007800d1ff07008a
:101c540008007800cfff070099007800814f7000da
:101c64000b003b000800be001e0107004f00b1003e
:101c740003003700f3ff2700f2ff2f006110b900c3
:101c84004f06be004f05be004f04be000080fa00a0
:101c940000000600889fbe00830478000300e00073
:101ca4002c00350003003c00008270000402710027
:101cb4002600320036432000c50020008383cf0075
:101cc4000a0039000541b1008283cf0007003900c2
:101cd4000541b1008183cf00040039000541b10002
:101ce4008083cf00010039000541b10085c3530052
:101cf4006022b800120032000a003b0084827200a5
:101d0400610260008301d1000281d3008180d3008d
:101d14000080d3000603e8008743e800f7ff3a0099
:101d2400070037000000400081804800020149009c
:101d3400838149000603e9008743e900f9ff3a007b
:101d44008800070009f0a70003f0a0004f04be00bc
:101d54000000060060001000e08018006001190017
:101d6400e0811900d3ff3b00033e2c00f7ff37004e
:101d74002800fa00889fbe008a9fbe008c9fbe0088
:101d840007067800878669000c003b00030478008e
:101d94008704780008f0a10009f0a100840f500026
:101da400858f5800860f5900890f5c0003003300ab
:101db4000cf0a20001003a000cf0a1009cff070007
:101dc4006400e1005f003200780147006408e1002c
:101dd400610032006c014700748557003200be0078
:101de4001201be003a04be001a05be001e03900094
:101df400be0a90008503530006003d000004fd0068
:101e04008104fd000205fd008305fd008703ea004f
:101e1400050378000df8a3000400320060041400e8
:101e2400e0841c0060051d00e0851d006022b800f0
:101e34007d0320000d38e1008006eb000b00390023
:101e44004433dd00f300b20083017300390037002e
:101e5400848272000d027800e10664008b85d10053
:101e64000a85d3008984d3000884d3008703e9005a
:101e7400f7ff3b0008004000898048000a01490040
:101e84008b81490004003b0060001000e0801800d2
:101e940060011900e08119000358a3000900320011
:101ea4008d82720084827200610260008301d1001d
:101eb4000281d3008180d3000080d3000603e800b0
:101ec4001b0037000348a30017003a000600e00097
:101ed400170034000603e9000d00a30000004800c9
:101ee4008180480002014900838149000348a3001e
:101ef4000f003a000600e000090034000603e90080
:101f040000004000818048000201490083814900ab
:101f140001003a000003eb000348a300f5ff320080
:101f24006022b80002003700848272006182660079
:101f34000c00070003f0a1000cf0a70003f0a000c0
:101f44004fff3700640147006408e10002003a00d3
:101f54000df8a30047ff3a003200be001201be0094
:101f640047ff3700180020005700200008045300e2
:101f74000d003d000600200097fc2f000740e10003
:101f84001e00340084827200610260008301d1006b
:101f94000281d3008180d3000080d3000804e800cc
:101fa400f8ff3a0047002000610460000504740053
:101fb400040464000d00320061004000e080480029
:101fc40060014900e081490003b8a5000700320020
:101fd4000603e8006538e10004003a008301d100fb
:101fe4000281d3008180d3000080d300f87f2000d9
:101ff4000830e10003003500080378006000b800f1
:102004006011b8004433dd00f300b20083017300b3
:1020140000000600889fbe008a9fbe008c9fbe0001
:102024000404b8000506b8008904460060854e0023
:102034000606b8000a054600e0854e000706b8000b
:102044008b054600040eb800890446000a854e003c
:10205400e0854d00050eb8000a0546008b854e004c
:10206400060eb8008b0546000416b8000a054600a3
:102074008b854e000516b8008b054600041eb8007b
:102084008b0546000800be000a01be004f06be00d4
:102094004f05be004f04be000000060005ff2700e8
:1020a40005826100070032000428e10001003200cb
:1020b400240005000600070001003a004400050062
:1020c4000408050002000700f9ff3a0014000500a7
:1020d4006f826100810270008502710085027200c6
:1020e40000000600e48240001078a30007003200dc
:1020f400640240001178a3003400be001401be0045
:10210400040032000330a700000006003500be00c2
:102114001501be000330a0000000060020c2bf006d
:1021240066406000e64f500002003a003011800023
:102134000000060030118000f00fb200000006001d
:1021440021e2a9009560a9009580a9008560a900f5
:102154008580a90000000600421188000011880053
:1021640011118800010037003011800022c2bf0025
:102174000008a300fcff3a008560a90000000600e7
:102184008560a9008580a900e7416000c419dd00cd
:10219400910a200091407800f2c8b30082c0600028
:1021a40083c070008000fd00a9e0b7008000fd003e
:1021b400800178000307b200c419de00a10a2000e0
:1021c4009140780082cfb30082c0600083c0700069
:1021d4008000fd00aae0b7008000fd0068016000f7
:1021e4004311de004311dd005109200091407800c5
:1021f4000134a10082c070008000fd0095e0b700aa
:102204008000fd000008b2004700de004400dd004d
:1022140051092000914078000144a10080c0700061
:102224000100780095e0b700000006008000780007
:1022340020c2bf0066406000e64f5000010032003b
:10224400f10fb20021118800000006006140600017
:102254004500dd0001742000914078000154a10084
:1022640080c070000100780040e7b700000006005d
:1022740016c2bf000008a300fdff3a0016c2bf004b
:102284000018a300faff3a0016c2bf000028a300fa
:10229400f7ff3a0016c2bf000038a300f4ff3a006b
:1022a40016c2bf000048a300f1ff3a0019c2bf00e4
:1022b4000068a300eeff3a00000006001602a80022
:1022c400000006000080fb009010880018c2bf00c8
:1022d40001c8b300014060000080fb000000e90079
:1022e4004f00de000000e900000006001642a800ce
:1022f400000006001662a80016c2bf000038a30042
:10230400fdff3a0018c2a900801080000080fb0085
:0423140000000600bf
:020000040000fa
:100008003c620100506201006462010078620100f4
:100018008c6201003c6201003c6201003c6201000c
:100028003c6201003c6201003c6201003c6201004c
:100038003c6201003c6201003c6201003c6201003c
:10004800366901003c6201003c6201004868010019
:1000580040680100445a01003c6201003c62010012
:100068003c6201003c6201003c620100e061010069
:100078003c6201003c6201003c6201003c620100fc
:100088003c6201003c6201003c6201004e610100db
:100098003c6201003c6201003c6201003c620100dc
:1000a8003c6201003c6201003c6201003c620100cc
:1000b8003c6201003c6201003c6201003c620100bc
:1000c8003c6201003c6201003c6201003c620100ac
:1000d8003c6201003c6201003c6201003c6201009c
:1000e8003c6201003c6201003c6201003c6201008c
:1000f8003c6201003c6201003c6201003c6201007c
:100108003c6201003c6201003c6201003c6201006b
:100118003c6201003c6201003c6201003c6201005b
:100128003c6201003c6201003c6201003c6201004b
:100138003c6201003c6201003c6201003c6201003b
:100148003c6201003c6201003c6201003c6201002b
:100158003c6201003c6201003c6201003c6201001b
:100168003c6201003c6201003c6201003c6201000b
:100178003c6201003c6201003c6201003c620100fb
:100188003c6201003c6201003c6201003c620100eb
:100198003c6201003c6201003c6201003c620100db
:1001a8003c6201003c6201003c6201003c620100cb
:1001b8003c6201003c6201003c6201003c620100bb
:1001c8003c6201003c6201003c6201003c620100ab
:1001d8003c6201003c6201003c6201003c6201009b
:1001e8003c6201003c6201003c6201003c6201008b
:0801f8003c6201003c620100c1
:020000040000fa
:100208003c620100506201006462010078620100f2
:100218008c6201003c6201003c6201003c6201000a
:100228003c6201003c6201003c6201003c6201004a
:100238003c6201003c6201003c6201003c6201003a
:10024800366901003c6201003c6201004868010017
:1002580040680100445a01003c6201003c62010010
:100268003c6201003c6201003c620100e061010067
:100278003c6201003c6201003c6201003c620100fa
:100288003c6201003c6201003c6201004e610100d9
:100298003c6201003c6201003c6201003c620100da
:1002a8003c6201003c6201003c6201003c620100ca
:1002b8003c6201003c6201003c6201003c620100ba
:1002c8003c6201003c6201003c6201003c620100aa
:1002d8003c6201003c6201003c6201003c6201009a
:1002e8003c6201003c6201003c6201003c6201008a
:1002f8003c6201003c6201003c6201003c6201007a
:100308003c6201003c6201003c6201003c62010069
:100318003c6201003c6201003c6201003c62010059
:100328003c6201003c6201003c6201003c62010049
:100338003c6201003c6201003c6201003c62010039
:100348003c6201003c6201003c6201003c62010029
:100358003c6201003c6201003c6201003c62010019
:100368003c6201003c6201003c6201003c62010009
:100378003c6201003c6201003c6201003c620100f9
:100388003c6201003c6201003c6201003c620100e9
:100398003c6201003c6201003c6201003c620100d9
:1003a8003c6201003c6201003c6201003c620100c9
:1003b8003c6201003c6201003c6201003c620100b9
:1003c8003c6201003c6201003c6201003c620100a9
:1003d8003c6201003c6201003c6201003c62010099
:1003e8003c6201003c6201003c6201003c62010089
:0803f8003c6201003c620100bf
:020000040000fa
:020000040001f9
:10e008000000fa003c6204000100000050620400b5
:10e01800010000006462040001000000786204004e
:10e02800010000008c620400010000003c62040052
:10e03800010000003c620400010000003c62040092
:10e04800010000003c620400010000003c62040082
:10e05800010000003c620400010000003c62040072
:10e068000100000036690400010000003c62040061
:10e07800010000003c620400010000004868040040
:10e08800010000004068040001000000445a040038
:10e09800010000003c620400010000003c62040032
:10e0a800010000003c62040001000000e06104007f
:10e0b800010000003c620400010000003c62040012
:10e0c800010000003c620400010000003c62040002
:10e0d800010000003c620400010000004e610400e1
:10e0e800010000003c620400010000003c620400e2
:10e0f800010000003c620400010000003c620400d2
:10e10800010000003c620400010000003c620400c1
:10e11800010000003c620400010000003c620400b1
:10e12800010000003c620400010000003c620400a1
:10e13800010000003c620400010000003c62040091
:10e14800010000003c620400010000003c62040081
:10e15800010000003c620400010000003c62040071
:10e16800010000003c620400010000003c62040061
:10e17800010000003c620400010000003c62040051
:10e18800010000003c620400010000003c62040041
:10e19800010000003c620400010000003c62040031
:10e1a800010000003c620400010000003c62040021
:10e1b800010000003c620400010000003c62040011
:10e1c800010000003c620400010000003c62040001
:10e1d800010000003c620400010000003c620400f1
:10e1e800010000003c620400010000003c620400e1
:10e1f800010000003c620400010000003c620400d1
:10e20800010000003c620400010000003c620400c0
:0ce21800010000000080fa000000060079
:020000040000fa
:020000040002f8
:102318000d0a00000d0a00000d0a00000d0a000059
:102328000d0a00000d0a00000d0a0000000d000053
:102338000a4400002031000020250000640000004d
:102348000d0a00004420000032200000256400002f
:10235800000d00000a440000203300002025000082
:10236800640000000d0a0000442000003420000032
:1023780025640000000d00000a440000203500001c
:1023880020250000640000000d0a00004420000021
:102398003620000025640000000d00000a440000fb
:1023a8002037000020250000640000000d0a00000e
:1023b800442000003820000025640000000d0000c3
:1023c8000a440000203900002025000064000000b5
:1023d8000d0a000044310000302000002564000090
:1023e800000d00000a4400003131000020250000e3
:1023f800640000000d0a0000443100003220000093
:1024080025640000000d00000a440000313300007c
:1024180020250000640000000d0a0000443100007f
:102428003420000025640000000d00000a4400006c
:102438003135000020250000640000000d0a00006e
:10244800443100003620000025640000000d000023
:102458000a44000031370000202500006400000015
:102468000d0a0000443100003820000025640000f7
:10247800000d00000a44000031390000202500004a
:10248800640000000d0a0000443200003020000003
:1024980025640000000d00000a44000032310000ed
:1024a80020250000640000000d0a000044320000ee
:1024b8003220000025640000000d00000a440000de
:1024c8003233000020250000640000000d0a0000df
:1024d800443200003420000025640000000d000094
:1024e8000a44000032350000202500006400000086
:1024f8000d0a000044320000362000002564000068
:10250800000d00000a4400003237000020250000ba
:10251800640000000d0a000044320000382000006a
:1025280025640000000d00000a4400003239000054
:1025380020250000640000000d0a0000443300005c
:102548003020000025640000000d00000a4400004f
:102558003331000020250000640000000d0a00004f
:10256800443300003220000025640000000d000004
:102578000a440000333300002025000064000000f6
:102588000d0a0000443300003420000025640000d8
:10259800000d00000a44000033350000202500002b
:1025a800640000000d0a00004433000036200000db
:1025b80025640000000d00000a44000033370000c5
:1025c80020250000640000000d0a000044330000cc
:1025d8003820000025640000000d00000a440000b7
:1025e8003339000020250000640000000d0a0000b7
:1025f800443400003020000025640000000d000075
:102608000a44000034310000202500006400000066
:102618000d0a000044340000322000002564000048
:10262800000d00000a0d00000a44000020310000df
:102638003a2500006420000044200000323a0000df
:10264800256400002020000044200000333a0000e8
:10265800256400002020000044200000343a0000d7
:10266800256400002020000044200000353a0000c6
:10267800256400002020000044200000363a0000b5
:10268800256400002020000044200000373a0000a4
:10269800256400002020000044200000383a000093
:1026a800256400002020000044200000393a000082
:1026b800256400002020000044310000303a00006a
:1026c80025640000000d00000a44000031310000bc
:1026d8003a2500006420000044310000323a00002e
:1026e800256400002020000044310000333a000037
:1026f800256400002020000044310000343a000026
:10270800256400002020000044310000353a000014
:10271800256400002020000044310000363a000003
:10272800256400002020000044310000373a0000f2
:1027380025640000203e00003c20000031380000e5
:102748003a250000642000002044000031390000d0
:102758003a250000642000002044000032300000c8
:102768003a250000640000000d0a00004432000011
:10277800313a000025640000204400003232000095
:102788003a25000064200000204400003233000095
:102798003a25000064200000204400003234000084
:1027a8003a25000064200000204400003235000073
:1027b8003a25000064200000204400003236000062
:1027c8003a25000064200000204400003237000051
:1027d8003a25000064200000204400003238000040
:1027e8003a2500006420000020440000323900002f
:1027f8003a25000064200000204400003330000027
:102808003a250000640000000d0a0000443300006f
:10281800313a0000256400002044000033320000f3
:102828003a250000642000002044000033330000f3
:102838003a250000642000002044000033340000e2
:102848003a250000642000002044000033350000d1
:102858003a250000642000002044000033360000c0
:102868003a250000642000002044000033370000af
:102878003a2500006420000020440000333800009e
:102888003a250000642000003e3c0000204400007f
:10289800333900003a25000064200000204400007d
:1028a800343000003a250000640000000d0a0000e2
:1028b80044340000313a0000256400002044000040
:1028c800343200003a250000642000002044000053
:1028d800343300003a250000642000002044000042
:1028e800343400003a250000642000002044000031
:1028f800343500003a250000642000002044000020
:10290800343600003a250000642000003e3c0000f8
:1029180020440000343700003a25000064200000fd
:102928003e3c000020440000343800003a250000f6
:1029380064200000200000000d0a00005b25000054
:10294800635d00005b250000635d00005b250000ff
:10295800635d00005b250000635d00005b250000ef
:10296800635d00005b250000635d0000000d000052
:102978000a250000346400002025000034640000ab
:102988002025000034640000202500003464000085
:102998002025000034640000202500003464000075
:1029a8002025000034640000202500003464000065
:1029b8002025000034640000202500003464000055
:1029c8002025000034640000202500003464000045
:1029d8002025000034640000202500003464000035
:1029e8002025000034640000202500003464000025
:1029f800200000000d0a000053630000616c000015
:102a0800696e0000673a0000000d00000a3c0000f3
:102a180020200000256400003e0000000d0a000090
:102a2800574f0000555400003a250000303400008c
:102a3800580000000d0a0000574f000055540000d0
:102a48002b3100003a250000303400005800000007
:102a58000d0a000053630000616e0000204d000065
:102a68006f640000653a000025640000000d000056
:102a78000a38000030300000303a000025300000ed
:102a880034580000000d00000a3800003030000003
:102a9800323a00002530000034580000000d0000d4
:102aa8000a38000030300000343a000025300000b9
:102ab80034580000000d00000a38000030300000d3
:102ac800363a00002530000034580000000d0000a0
:102ad8000a4200004c6f00006e3a000025640000b6
:102ae800204200004c560000616c00003a250000ae
:102af800640000000d0a000025640000000d0000bd
:102b08000a3000003a0000000d0a000020620000b0
:102b1800746900006f3400003241000070700000da
:102b28002056000065720000736900006f6e000097
:102b38003a20000025640000200000000d0a000073
:102b4800323a0000000d00000a3300003a0000008d
:102b58000d0a0000343a0000000d00000a3500009c
:102b68003a0000000d0a0000363a0000000d00008f
:102b78000a3700003a0000000d0a0000383a000049
:102b8800000d00000a3900003a0000000d0a00009c
:102b98004150000050200000537400006172000092
:102ba800746900006e670000205500007000000086
:102bb8000d0a000053630000616c000065200000ee
:102bc80043680000616e00003a250000640d0000b3
:102bd8000a0000005b0000002535000064200000aa
:102be800005d00002000000020280000256400008f
:102bf800290d00000a0000000d0a00002031000025
:102c08003d4300002d7a0000657200006f2000002f
:102c18000d0a000000430000686100006e3a0000e1
:102c280025640000204300002d5a00006572000052
:102c38006f3a00002564000020520000657600000d
:102c48003a2500006420000052610000773a000035
:102c580025640000204d0000696e00003a25000040
:102c680064200000646200004c6f0000773a0000a6
:102c7800256400002064000062480000693a0000f2
:102c880025640000204d0000617800003a2500000e
:102c9800640d00000a0000000d0a0000432d00002a
:102ca8005a650000726f0000206100006c67000028
:102cb8006f20000063680000616e00003a25000084
:102cc800640000000d0a0000312d00005261000070
:102cd8006e67000065200000616c0000676f0000ef
:102ce80020630000686100006e3a0000256400005f
:102cf800000d00000a500000726f000067720000ab
:102d0800616d0000436100006c43000068610000d1
:102d18006e6e0000656c00003a200000256400001b
:102d2800000d00000a6d0000696e00003a250000e1
:102d3800640000000d0a0000646200004c6f00008f
:102d4800773a000025640000000d00000a640000c6
:102d58006248000069670000683a000025640000c6
:102d6800000d00000a6d0000617800003a2500009f
:102d7800640000000d0a0000666c00006167000036
:102d8800733a0000200000003c5200004157000048
:102d98003e0000003c3100002d520000414e000072
:102da800474500003e0000003c4300002d5a00004b
:102db800657200006f3e0000003c000052450000b4
:102dc8005645000052530000453e0000003c0000fc
:102dd80062750000726e00003e0000000d0a0000df
:102de80070690000642000006c6f00003a25000044
:102df8006420000070690000642000006869000019
:102e08003a2500006400000006000000ff090000e9
:102e180001a100000119000001290000401500006f
:102e28000125000040750000089500004081000061
:102e380000190000012900004091000000c00000b6
:102e48000501000009040000a101000005010000bf
:102e58000509000019010000298000001500000084
:102e68002501000075010000958000008102000026
:102e780009010000a1000000050100000930000060
:102e8800093100000932000009330000093400004c
:102e98000935000009360000093700001600000057
:102ea80000260000ff7f0000751000009508000054
:102eb80081820000c0c00000050100000905000073
:102ec800a10100000501000005090000190100002a
:102ed8002980000015000000250100007501000090
:102ee800958000008102000009010000a100000097
:102ef8000501000009300000093100000932000016
:102f080009330000093400000935000009360000c3
:102f1800093700001600000000260000ff7f0000af
:102f2800751000009508000081820000c0c00000f4
:102f38000d0a0000476100006d650000536900003c
:102f48007a650000000d00000a4a00006f79000051
:102f580020530000697a0000650000000d0a000097
:102f6800432d0000486900006420000053690000f8
:102f78007a650000000000000d0a0000414e0000c4
:102f8800313a00002534000064200000000d0000e4
:102f98000a4100004e3200003a2500003464000067
:102fa800200000000d0a0000414e0000333a0000e6
:102fb8002534000064200000000d00000a410000d4
:102fc8004e3400003a250000346400002000000060
:102fd8000d0a0000414e0000353a0000253400007b
:102fe80064200000000d00000a4100004e36000079
:102ff8003a25000034640000200000000d0a00009b
:10300800414e0000373a00002534000064200000db
:10301800000d00000a4100004e3800003a2500006b
:1030280034640000200000000d0a0000496e000012
:103038006974000020410000440000000d0a0000ef
:103048005049000044200000696e0000207500000f
:10305800736500003a250000303400007820000035
:1030680025640000000d00000a4900006e69000098
:1030780074200000320000000d0a0000476f0000b5
:10308800696e000067200000746f00002053000084
:10309800434100004e0000000d0a00004e4f0000a2
:1030a8005420000073630000616e00006e69000028
:1030b8006e670000000d00000a4600006c61000009
:1030c800677300003a250000303200005800000005
:1030d8000d0a0000205400006573000074200000f1
:1030e80045450000505200004f4d000000200000f0
:1030f80066610000696c0000203100003a20000081
:1031080025300000325800000020000066610000f1
:10311800696c0000203200003a20000025300000d1
:10312800325800000020000066610000696c000051
:10313800203300003a2000002530000032580000fb
:103148000020000066610000696c00002034000067
:103158000020000066610000696c00002035000056
:103168000020000066610000696c00002036000045
:10317800000d00000a54000065730000744500004b
:1031880045500000524f00004d20000053750000cc
:10319800636300006573000073000000256c000085
:1031a80064000000313000003030000000000000f2
:1031b80042540000494f0000343200002053000000
:1031c80054490000434b00002049000046430000da
:1031d800204200004f41000052440000202000001f
:1031e80020200000202000002020000020200000d7
:1031f800000d00000a5b0000256300005d5b000015
:10320800256300005d5b0000256300005d5b000036
:10321800256300005d5b0000256300005d5b000026
:10322800256300005d0000000d0a00005b2500001a
:10323800635d00003c250000633e00000053000071
:103248004947000031300000370000000d0a000037
:1032580045450000505200004f4d0000207200000c
:10326800657700007269000074740000656e0000e4
:10327800000000000d0a000045720000726f000097
:10328800723a00002073000074610000727400003c
:10329800206d000075730000742000006265000056
:1032a80020610000742000006c650000617300005c
:1032b80074200000342000006c6500007373000067
:1032c80020740000686100006e2000007374000024
:1032d8006f700000000d00000a2500003038000063
:1032e8006c780000200000002530000034580000f1
:1032f8002530000034580000200000002020000085
:10330800257300002000000025730000000d000058
:103318000a0000000d0a0000446500007363000005
:1033280020470000616d0000650000000d0a0000e4
:103338004465000073630000204a00006f790000b4
:10334800000d00000a4400006573000063200000bf
:10335800432d000048690000640000000d0a0000c9
:1033680052650000737500006c7400003a2000007c
:1033780061720000793a00002564000020760000a0
:10338800616c00003a25000030340000780000002d
:103398000d0a0000446900006d6900006e740000a9
:1033a800496e000069740000000000000d0a00006a
:1033b80054690000636b0000496e000069740000e6
:1033c800000000003c4700003e0000003c4a0000ae
:0433d8003e000000b3
:020000040000fa
:020000040002f8
:1033dc005400fa00c0182900801f7800b262020065
:1033ec00010000008f87e900d3c2bf000044b20087
:1033fc008000eb00112f98000004e0000200320066
:10340c0010002000102f98009e289000811f78003b
:10341c00b0192900801f7800b26202000100000080
:10342c00e4875700d3c2bf000042b2008000eb001b
:10343c00012f98000004e000020032001000200070
:10344c00002f98008e289000811f7800401a2900c8
:10345c00801f7800b262020001000000e487570070
:10346c00dac2bf00614060008000eb007127980059
:10347c000004e000020032001000200070279800c9
:10348c00fe209000811f7800d01a2900801f780040
:10349c00b262020001000000e4875700dbc2bf00eb
:1034ac00684060008000eb00612798000004e00099
:1034bc00020032001000200060279800ee209000df
:1034cc00811f7800601b2900801f7800b262020007
:1034dc0001000000e4875700dbc2bf0064406000bd
:1034ec008000eb00512798000004e000020032003d
:1034fc001000200050279800de209000811f7800db
:10350c00f01b2900801f7800b2620200010000004d
:10351c00e4875700dbc2bf00624060008000eb0014
:10352c00412798000004e000020032001000200047
:10353c0040279800ce209000811f7800801c290025
:10354c00801f7800b262020001000000e48757007f
:10355c00dbc2bf00614060008000eb0031279800a7
:10356c000004e00002003200100020003027980018
:10357c00be209000811f7800101d2900801f78004c
:10358c00b262020001000000e4875700dac2bf00fb
:10359c00644060008000eb00212798000004e000ec
:1035ac00020032001000200020279800ae2090006e
:1035bc00811f7800a01d2900801f7800b2620200d4
:1035cc0001000000e4875700dac2bf0062406000cf
:1035dc008000eb00112798000004e000020032008c
:1035ec0010002000102798009e209000811f78006a
:1035fc00301e2900801f7800b2620200010000001a
:10360c00e4875700ebc2bf00614060008000eb0014
:10361c00012798000004e000020032001000200096
:10362c00002798008e209000811f7800c01e290072
:10363c00801f7800b262020001000000e48757008e
:10364c00eac2bf00644060008000eb00711f98006c
:10365c000004e0000200320010002000701f9800ef
:10366c00fe189000811f7800501f2900801f7800e1
:10367c00b262020001000000e4875700cbc2bf0019
:10368c00644060008000eb00611f98000004e000c3
:10369c000200320010002000601f9800ee1890000d
:1036ac00811f7800e01f2900801f7800b2620200a1
:1036bc0001000000e4875700b12d200091407800f4
:1036cc0000c8b30000c060008000eb00511f9800e0
:1036dc000004e0000200320010002000501f98008f
:1036ec00de189000811f780070202900801f780060
:1036fc00b262020001000000e4875700eac2bf007a
:10370c00704060008000eb00411f98000004e00056
:10371c000200320010002000401f9800ce189000cc
:10372c00811f780000212900801f7800b2620200fe
:10373c0001000000e4875700eac2bf000042b2005b
:10374c008000eb00311f98000004e0000200320002
:10375c0010002000301f9800be189000811f7800c8
:10376c0090212900801f7800b26202000100000045
:10377c00e4875700dbc2bf000044b2008000eb00be
:10378c00211f98000004e00002003200100020000d
:10379c00201f9800ae189000811f7800202229006d
:1037ac00801f7800b262020001000000e48757001d
:1037bc00cbc2bf000042b2008000eb00111f98008a
:1037cc000004e0000200320010002000101f9800de
:1037dc009e189000811f7800b0222900801f78006d
:1037ec00b262020001000000e4875700cbc2bf00a8
:1037fc00704060008000eb00011f98000004e000a6
:10380c000200320010002000001f98008e1890005b
:10381c00811f780040232900801f7800b2620200cb
:10382c0001000000e4875700c3c2bf006240600083
:10383c008000eb00711798000004e00002003200d9
:10384c001000200070179800fe109000811f780067
:10385c00d0232900801f7800b26202000100000012
:10386c00e4875700c3c2bf00644060008000eb00d7
:10387c00611798000004e0000200320010002000e4
:10388c0060179800ee109000811f780060242900ca
:10389c00801f7800b262020001000000e48757002c
:1038ac00e3c2bf00614060008000eb00511798003c
:1038bc000004e000020032001000200050179800b5
:1038cc00de109000811f7800f0242900801f780002
:1038dc00b262020001000000e4875700e3c2bf009f
:1038ec00624060008000eb00411798000004e0008b
:1038fc00020032001000200040179800ce109000fb
:10390c00811f780080252900801f7800b262020098
:10391c0001000000e4875700f3c2bf006140600063
:10392c008000eb00311798000004e0000200320028
:10393c001000200030179800be109000811f7800f6
:10394c0010262900801f7800b262020001000000de
:10395c00e4875700f3c2bf00624060008000eb00b8
:10396c00211798000004e000020032001000200033
:10397c0020179800ae109000811f7800a026290017
:10398c00801f7800b262020001000000e48757003b
:10399c00f2c2bf000044b2008000eb001117980087
:1039ac000004e00002003200100020001017980004
:1039bc009e109000811f780030272900801f78000e
:1039cc00b262020001000000e4875700212f2000a2
:1039dc009140780000c8b30000c060008000eb008c
:1039ec00011798000004e0000200320010002000d3
:1039fc00001798008e109000811f7800c0272900b6
:103a0c00801f7800b262020001000000e4875700ba
:103a1c00d2c2bf00624060008000eb00710f9800c2
:103a2c000004e0000200320010002000700f98002b
:103a3c00fe089000811f780050282900801f780014
:103a4c00b262020001000000e4875700d2c2bf003e
:103a5c00684060008000eb00610f98000004e000fb
:103a6c000200320010002000600f9800ee08900059
:103a7c00811f7800e0282900801f7800b2620200c4
:103a8c0001000000e4875700e2c2bf000044b2000e
:103a9c008000eb00510f98000004e000020032009f
:103aac0010002000500f9800de089000811f780055
:103abc0070292900801f7800b2620200010000000a
:103acc00e4875700212e20009140780000c8b300f5
:103adc0000c060008000eb00410f98000004e00083
:103aec000200320010002000400f9800ce08900019
:103afc00811f7800002a2900801f7800b262020022
:103b0c0001000000e4875700e2c2bf00644060007f
:103b1c008000eb00310f98000004e000020032003e
:103b2c0010002000300f9800be089000811f780014
:103b3c00902a2900801f7800b26202000100000068
:103b4c00e4875700e2c2bf000042b2008000eb00e5
:103b5c00210f98000004e000020032001000200049
:103b6c00200f9800ae089000811f7800202b2900b0
:103b7c00801f7800b262020001000000e487570049
:103b8c00e2c2bf00704060008000eb00110f980093
:103b9c000004e0000200320010002000100f98001a
:103bac009e089000811f7800b02b2900801f7800a0
:103bbc00b262020001000000e4875700e2c2bf00bd
:103bcc00684060008000eb00010f98000004e000ea
:103bdc000200320010002000000f98008e089000a8
:103bec00811f7800402c2900801f7800b2620200ef
:103bfc0001000000e4875700e2c2bf006140600092
:103c0c008000eb00710798000004e0000200320015
:103c1c001000200070079800fe009000811f7800b3
:103c2c00d02c2900801f7800b26202000100000035
:103c3c00e4875700e2c2bf00624060008000eb00e6
:103c4c00610798000004e000020032001000200020
:103c5c0060079800ee009000811f7800602d29000d
:103c6c00801f7800b262020001000000e487570058
:103c7c00f2c2bf00624060008000eb005107980068
:103c8c000004e000020032001000200050079800f1
:103c9c00de009000811f7800f02d2900801f780035
:103cac00b262020001000000e4875700f2c2bf00bc
:103cbc00614060008000eb00410798000004e000c8
:103ccc00020032001000200040079800ce00900047
:103cdc00811f7800802e2900801f7800b2620200bc
:103cec0001000000e4875700eac2bf006240600098
:103cfc008000eb00310798000004e0000200320065
:103d0c001000200030079800be009000811f780042
:103d1c00102f2900801f7800b26202000100000001
:103d2c00e4875700eac2bf00614060008000eb00ee
:103d3c00210798000004e00002003200100020006f
:103d4c0020079800ae009000811f7800a02f29005a
:103d5c00801f7800b262020001000000e487570067
:103d6c00dac2bf000044b2008000eb0011079800db
:103d7c000004e00002003200100020001007980040
:103d8c009e009000811f780030302900801f780041
:103d9c00b262020001000000e4875700a12d200050
:103dac009140780000c8b30000c060008000eb00b8
:103dbc00010f78000004e000020032001000200027
:103dcc00000f78009e007800811f7800c030290019
:103ddc00801f7800b262020001000000e4875700e7
:103dec000080fa00000006000000fa00889fbe0068
:103dfc009fd0bf008080fb009ed0bf000081fb00e5
:103e0c009dd0bf008081fb009cd0bf000082fb00d6
:103e1c009bd0bf008082fb009ad0bf000083fb00c8
:103e2c0099d0bf008083fb0098d0bf000084fb00ba
:103e3c0097d0bf008084fb0096d0bf000080fb00b1
:103e4c00811f7800821f7800831f7800841f780000
:103e5c00851f7800861f7800871f7800881f7800e0
:103e6c00891f7800801f780050312900801f78004e
:103e7c00b262020001000000f6875700a9d0bf0013
:103e8c008080fb00a8d0bf000081fb00a7d0bf0042
:103e9c008081fb00a6d0bf000082fb00a5d0bf0034
:103eac008082fb00a4d0bf000083fb00a3d0bf0026
:103ebc008083fb00a2d0bf000084fb00a1d0bf0018
:103ecc008084fb00a0d0bf000080fb00811f780025
:103edc00821f7800831f7800841f7800851f78006c
:103eec00861f7800871f7800881f7800891f78004c
:103efc00801f780070362900801f7800b2620200a3
:103f0c0001000000f6875700b3d0bf008080fb0093
:103f1c00b2d0bf000081fb00b1d0bf008081fb009c
:103f2c00b0d0bf000082fb00afd0bf008082fb008e
:103f3c00aed0bf000083fb00add0bf008083fb0080
:103f4c00acd0bf000084fb00abd0bf008084fb0072
:103f5c00aad0bf000080fb00811f7800821f780070
:103f6c00831f7800841f7800851f7800861f7800d7
:103f7c00871f7800881f7800891f7800801f7800c1
:103f8c00803b2900801f7800b26202000100000013
:103f9c00f6875700bdd0bf008080fb00bcd0bf00af
:103fac000081fb00bbd0bf008081fb00bad0bf00fa
:103fbc000082fb00b9d0bf008082fb00b8d0bf00ec
:103fcc000083fb00b7d0bf008083fb00b6d0bf00de
:103fdc000084fb00b5d0bf008084fb00b4d0bf00d0
:103fec000080fb00811f7800821f7800831f7800ff
:103ffc00841f7800851f7800861f7800871f780043
:10400c00881f7800891f7800801f78008040290065
:10401c00801f7800b262020001000000f687570092
:10402c00c5d0bf008081fb00c4d0bf000082fb0064
:10403c00c3d0bf008082fb00c2d0bf000083fb0056
:10404c00c1d0bf008083fb00c0d0bf008080fb00cc
:10405c00bfd0bf000081fb00bed0bf000080fb00c2
:10406c00831f7800841f7800851f7800861f7800d6
:10407c00871f7800811f7800821f7800801f7800ce
:10408c00a0452900801f7800b262020001000000e8
:10409c00f28757004f04be000080fa0000000600b3
:1040ac000600fa00100798000000eb00000f7800e3
:1040bc001e009000200798002e009000e20f500088
:1040cc001a0032002e009000e20f500007003c0056
:1040dc002e0090000000e0000e0032002e00900038
:1040ec00e10f50000e0032001b0037002e00900034
:1040fc00e40f5000130032002e009000e40f50002b
:10410c000d0035002e009000e50f5000100032001d
:10411c00110037000000eb00000f78000e00370094
:10412c0080002000000f78000b00370000012000f9
:10413c00000f78000800370080012000000f780085
:10414c000500370000022000000f78000200370045
:10415c0080022000000f78009e007800600921008a
:10416c0000804000104078000004e000060032009f
:10417c009e009000000c21008080400010c0b30015
:10418c0080487800050037009e009000000c21004c
:10419c00808040000040eb00804878009e00e800e2
:1041ac006009210000804000104078000004e0000d
:1041bc000b0032001e0190009e009000000c2100ac
:1041cc000080400010407800804078000114a0006e
:1041dc00000c210000004100014878000a00370063
:1041ec001e0190009e009000000c210000804000f9
:1041fc0090407800d0cfb30080c06000000c21004c
:10420c0000004100014878009e80e8006009210010
:10421c0000804000104078000004e0000b003200e9
:10422c001e0190009e009000000c210000804000b8
:10423c0010407800804078000124a000000c210080
:10424c0000004100014878000a0037001e01900070
:10425c009e009000000c21000080400090407800ef
:10426c00b0cfb30080c06000000c21000000410002
:10427c00014878001e007800e3004000600921002e
:10428c0000804000104078000004e0000b00320079
:10429c001e0190009e009000000c21000080400048
:1042ac0010407800804078000134a000000c210000
:1042bc0000004100014878000a0037001e01900000
:1042cc009e009000000c210000804000904078007f
:1042dc0070cfb30080c06000000c210000004100d2
:1042ec00014878001e007800e400400060092100bd
:1042fc0000804000104078000004e0000b00320009
:10430c001e0190009e009000000c210000804000d7
:10431c0010407800804078000144a000000c21007f
:10432c0000004100014878000a0037001e0190008f
:10433c009e009000000c210000804000904078000e
:10434c00f0ceb30080c06000000c210000004100e2
:10435c00014878001e007800e5004000600921004b
:10436c0000804000104078000004e0000b00320098
:10437c001e0190009e009000000c21000080400067
:10438c009040780000c2b30080c07000000c210087
:10439c0000004100014878000a0037001e0190001f
:1043ac009e009000000c210000804000904078009e
:1043bc00f0cdb30080c06000000c21000000410073
:1043cc00014878001e007800e600400060092100da
:1043dc0000804000104078000004e0000b00320028
:1043ec001e0190009e009000000c210000804000f7
:1043fc009040780000c4b30080c07000000c210015
:10440c0000004100014878000a0037001e019000ae
:10441c009e009000000c210000804000904078002d
:10442c00f0cbb30080c06000000c21000000410004
:10443c00014878001e007800e70040006009210068
:10444c0000804000104078000004e0000b003200b7
:10445c001e0190009e009000000c21000080400086
:10446c009040780000c8b30080c07000000c2100a0
:10447c0000004100014878000a0037001e0190003e
:10448c009e009000000c21000080400090407800bd
:10449c00f0c7b30080c06000000c21000000410098
:1044ac00014878000080fa00000006000600fa00bf
:1044bc00000f7800214798001e007800104078000b
:1044cc00e24f5000030036000000eb00200798007c
:1044dc00110037001e007800104078008040e80082
:1044ec001e007800014878001e007800104078000b
:1044fc00e24f5000060036002e4090000000fb00fa
:10450c00e7fe07001000200020079800020037008b
:10451c000000eb00200798002e0090000080fa00ad
:10452c00000006000600fa00000f780021479800f2
:10453c001e007800104078000004e00003003a00f0
:10454c000000eb0020079800110037001e007800d7
:10455c00104078008040e9001e0078000148780087
:10456c001e007800104078000004e00006003a00bd
:10457c002e4090000000fb00c9fe07001000200038
:10458c0020079800020037000000eb00200798007d
:10459c002e0090000080fa00000006000200fa00d5
:1045ac000040eb00004f7800d3c2bf000044b200c3
:1045bc000004e000050032008040eb00600921009f
:1045cc00d8ff07001e4f7000040037008040eb003e
:1045dc0060092100b5ff07001e4f7000d3c2bf0059
:1045ec000042b2000004e000050032007009210016
:1045fc008040eb00cbff07001e4f7000040037001b
:10460c00700921008040eb00a8ff07001e4f7000ce
:10461c00dac2bf00614060000004e0000500320017
:10462c00800921008040eb00beff07001e4f700088
:10463c0004003700800921008040eb009bff07003d
:10464c001e4f7000dbc2bf00684060000004e00039
:10465c0005003200900921008040eb00b1ff0700fb
:10466c001e4f700004003700900921008040eb00c1
:10467c008eff07001e4f7000dbc2bf00644060005d
:10468c000004e00005003200a00921008040eb008e
:10469c00a4ff07001e4f700004003700a009210082
:1046ac008040eb0081ff07001e4f7000dbc2bf0093
:1046bc00624060000004e00005003200b0092100f7
:1046cc008040eb0097ff07001e4f7000040037007e
:1046dc00b00921008040eb0074ff07001e4f7000f2
:1046ec00dbc2bf00614060000004e0000500320046
:1046fc00c00921008040eb008aff07001e4f7000ac
:10470c0004003700c00921008040eb0067ff070060
:10471c001e4f7000dac2bf00644060000004e0006d
:10472c0005003200d00921008040eb007dff07001e
:10473c001e4f700004003700d00921008040eb00b0
:10474c005aff07001e4f7000dac2bf0062406000c3
:10475c000004e00005003200e009210011c0b300a4
:10476c0070ff07001e4f700004003700e0092100a5
:10477c0011c0b3004dff07001e4f7000ebc2bf000d
:10478c00614060000004e00005003200f0092100e7
:10479c0011c0b30063ff07001e4f70000400370008
:1047ac00f009210011c0b30040ff07001e4f70003c
:1047bc00eac2bf00644060000004e0000500320063
:1047cc00000a210011c0b30056ff07001e4f7000f5
:1047dc0004003700000a210011c0b30033ff0700aa
:1047ec001e4f7000cbc2bf00644060000004e000ac
:1047fc0005003200100a210011c0b30049ff070068
:10480c001e4f700004003700100a210011c0b300c5
:10481c0026ff07001e4f7000dbc2bf0001c8b300ab
:10482c00014060000004e00005003200200a210075
:10483c0011c0b3003bff07001e4f7000040037008f
:10484c00200a210011c0b30018ff07001e4f700092
:10485c00eac2bf00704060000004e00005003200b6
:10486c00300a210011c0b3002eff07001e4f70004c
:10487c0004003700300a210011c0b3000bff070001
:10488c001e4f7000eac2bf000042b2000004e000fc
:10489c0005003200400a210011c0b30021ff0700bf
:1048ac001e4f700004003700400a210011c0b300f5
:1048bc00fefe07001e4f7000dbc2bf000044b200ba
:1048cc000004e00005003200500a210011c0b300c2
:1048dc0014ff07001e4f700004003700500a21001f
:1048ec0011c0b300f1fe07001e4f7000cbc2bf0019
:1048fc000042b2000004e00005003200600a210012
:10490c0021c0b30007ff07001e4f700004003700e2
:10491c00600a210021c0b300e4fe07001e4f7000a6
:10492c00cbc2bf00704060000004e0000500320004
:10493c00700a210021c0b300fafe07001e4f700060
:10494c0004003700700a210021c0b300d7fe070015
:10495c001e4f7000c3c2bf00624060000004e00044
:10496c0005003200800a210021c0b300edfe0700d3
:10497c001e4f700004003700800a210021c0b300d4
:10498c00cafe07001e4f7000c3c2bf006440600027
:10499c000004e00005003200900a210021c0b300a1
:1049ac00e0fe07001e4f700004003700900a210043
:1049bc0021c0b300bdfe07001e4f7000e3c2bf0054
:1049cc00614060000004e00005003200a00a2100f4
:1049dc0021c0b300d3fe07001e4f70000400370047
:1049ec00a00a210021c0b300b0fe07001e4f7000ca
:1049fc00e3c2bf00624060000004e000050032002a
:104a0c00b00a210021c0b300c6fe07001e4f700083
:104a1c0004003700b00a210021c0b300a3fe070038
:104a2c001e4f7000f3c2bf00614060000004e00044
:104a3c0005003200c00a210021c0b300b9fe0700f6
:104a4c001e4f700004003700c00a210021c0b300c3
:104a5c0096fe07001e4f7000f3c2bf00624060005c
:104a6c000004e00005003200d00a210021c0b30090
:104a7c00acfe07001e4f700004003700d00a210066
:104a8c0021c0b30089fe07001e4f7000f2c2bf00a8
:104a9c000044b2000004e00005003200e00a2100ee
:104aac0031c0b3009ffe07001e4f7000040037009a
:104abc00e00a210031c0b3007cfe07001e4f7000dd
:104acc00f2c2bf0001c8b300014060000004e00066
:104adc0005003200f00a210031c0b30091fe07003e
:104aec001e4f700004003700f00a210031c0b300e3
:104afc006efe07001e4f7000d2c2bf006240600005
:104b0c000004e00005003200000b210031c0b300ae
:104b1c0084fe07001e4f700004003700000b2100bc
:104b2c0031c0b30061fe07001e4f7000d2c2bf003f
:104b3c00684060000004e00005003200100b21000a
:104b4c0031c0b30077fe07001e4f70000400370021
:104b5c00100b210031c0b30054fe07001e4f700033
:104b6c0093d3bf000004e000b8003a00e2c2bf00db
:104b7c000044b2000004e00005003200200b2100cc
:104b8c0031c0b30067fe07001e4f700004003700f1
:104b9c00200b210031c0b30044fe07001e4f7000f3
:104bac00e2c2bf0001c8b300014060000004e00095
:104bbc0005003200300b210031c0b30059fe070054
:104bcc001e4f700004003700300b210031c0b300c1
:104bdc0036fe07001e4f7000e2c2bf00644060004a
:104bec000004e00005003200400b210031c0b3008e
:104bfc004cfe07001e4f700004003700400b2100d4
:104c0c0031c0b30029fe07001e4f7000e2c2bf0086
:104c1c000042b2000004e00005003200500b2100fd
:104c2c0031c0b3003ffe07001e4f70000400370078
:104c3c00500b210031c0b3001cfe07001e4f70004a
:104c4c00e2c2bf00704060000004e00005003200ca
:104c5c00600b210041c0b30032fe07001e4f7000f4
:104c6c0004003700600b210041c0b3000ffe0700a9
:104c7c001e4f7000e2c2bf00684060000004e000fc
:104c8c0005003200700b210041c0b30025fe070067
:104c9c001e4f700004003700700b210041c0b300a0
:104cac0002fe07001e4f7000e2c2bf0061406000b0
:104cbc000004e00005003200800b210041c0b3006d
:104ccc0018fe07001e4f700004003700800b2100f7
:104cdc0041c0b300f5fd07001e4f7000e2c2bf00db
:104cec00624060000004e00005003200900b2100df
:104cfc0041c0b3000bfe07001e4f700004003700cc
:104d0c00900b210041c0b300e8fd07001e4f70005e
:104d1c00f2c2bf00624060000004e00005003200f7
:104d2c00a00b210041c0b300fefd07001e4f700018
:104d3c0004003700a00b210041c0b300dbfd0700cd
:104d4c001e4f7000f2c2bf00614060000004e00022
:104d5c0005003200b00b210041c0b300f1fd07008b
:104d6c001e4f700004003700b00b210041c0b3008f
:104d7c00cefd07001e4f7000eac2bf00624060000b
:104d8c000004e00005003200c00b210041c0b3005c
:104d9c00e4fd07001e4f700004003700c00b21001b
:104dac0041c0b300c1fd07001e4f7000eac2bf0036
:104dbc00614060000004e00005003200d00b2100cf
:104dcc0041c0b300d7fd07001e4f70000400370030
:104ddc00d00b210041c0b300b4fd07001e4f700082
:104dec00dac2bf000044b2000004e000050032004b
:104dfc00e00b210051c0b300cafd07001e4f70002c
:104e0c0004003700e00b210051c0b300a7fd0700e0
:104e1c001e4f7000dac2bf0001c8b3000140600031
:104e2c000004e00005003200f00b210051c0b3007b
:104e3c00bcfd07001e4f700004003700f00b210072
:104e4c0051c0b30099fd07001e4f70000080fa009e
:104e5c00000006000000fa000080fa0000000600c6
:104e6c000200fa00a0002000865d02000100000094
:104e7c008040780020c4b30080cf50000a003a0074
:104e8c00b0002000865d0200010000008040780028
:104e9c00c0c4b30080cf500003003a0010002000c3
:104eac00000f7800020037000000eb00000f7800c4
:104ebc001e0078000080fa00000006000000fa00d6
:104ecc0021c4b300a0002000825d0200010000009c
:104edc00c1c4b300b0002000825d020001000000dc
:104eec000080fa00000006000000fa0001c2b300c6
:104efc00a0002000825d02000100000001c2b3008e
:104f0c00b0002000825d0200010000000080fa0069
:104f1c00000006000600fa00100798002107980010
:104f2c000000eb00000f78000b0037001e0078002b
:104f3c00800078001e009000008040001040780037
:104f4c0080407800c20820001e004100825d0200f3
:104f5c00010000001e0fe8002e0090009e0f1000b4
:104f6c00f2ff35000080fa00000006000400fa0091
:104f7c00881f7800100798000000eb00000f7800e5
:104f8c000a0037001e007800800078001e00900098
:104f9c0000844000c10820001e804000865d020095
:104fac0001000000004c78001e0fe800f00120000a
:104fbc009e0f1000f3ff34001e0078008000780074
:104fcc001e009000808040000040eb00804878007c
:104fdc001e0090004f0478000080fa0000000600cc
:104fec000200fa00004f78009e407800600220001a
:104ffc00825d0200010000000080fa000000060043
:10500c000000fa0060022000865d02000100000032
:10501c000080fb000080fa00000006000800fa0087
:10502c0010079800210798002e009000000f7800c0
:10503c001e0078004800de00000f78001e00900073
:10504c00300798003e009000e30f50003b00320008
:10505c003e009000e30f50000a003c003e00900020
:10506c00e10f50001f0032003e009000e10f500095
:10507c0027003c003e0090000000e0000e003200d3
:10508c00640037003e009000e50f500041003200f4
:10509c003e009000e50f5000330035003e009000bc
:1050ac00e60f5000460032003e009000e70f500023
:1050bc004e003200570037001e0078008040780008
:1050cc0080022000825d0200010000002e00900092
:1050dc008040780090022000825d020001000000f8
:1050ec004c0037001e007800804078002003200020
:1050fc00825d0200010000002e00900080407800cc
:10510c0030032000825d02000100000041003700e6
:10511c001e00780080407800c0032000825d0200f1
:10512c00010000002e00900080407800d003200089
:10513c00825d020001000000360037001e0078007e
:10514c008040780060042000825d020001000000b5
:10515c002e0090008040780070042000825d0200d8
:10516c00010000002b0037001e0078008040780002
:10517c0000052000825d0200010000002e0090005e
:10518c008040780010052000825d020001000000c4
:10519c00200037001e00780080407800a005200019
:1051ac00825d0200010000002e009000804078001b
:1051bc00b0052000825d02000100000015003700e0
:1051cc001e0078008040780040062000825d0200be
:1051dc00010000002e009000804078005006200056
:1051ec00825d0200010000000a0037001e007800fa
:1051fc0080407800e0062000825d02000100000083
:10520c002e00900080407800f0062000825d0200a5
:10521c00010000000080fa00000006000600fa0001
:10522c00100798000000eb00000f78001e009000a3
:10523c00200798002e009000e30f50003e00320033
:10524c002e009000e30f50000a003c002e0090004e
:10525c00e10f5000200032002e009000e10f5000b2
:10526c0029003c002e0090000000e0000e003200ef
:10527c006c0037002e009000e50f50004600320005
:10528c002e009000e50f5000370035002e009000e6
:10529c00e60f50004c0032002e009000e70f50003b
:1052ac00550032005f00370080022000865d02004e
:1052bc00010000000080fb004800dd00000f7800ba
:1052cc0090022000865d0200010000000080fb00bf
:1052dc001e0f40005300370020032000865d0200a3
:1052ec00010000000080fb004800dd00000f78008a
:1052fc0030032000865d0200010000000080fb00ee
:10530c001e0f400047003700c0032000865d0200de
:10531c00010000000080fb004800dd00000f780059
:10532c00d0032000865d0200010000000080fb001d
:10533c001e0f40003b00370060042000865d020019
:10534c00010000000080fb004800dd00000f780029
:10535c0070042000865d0200010000000080fb004c
:10536c001e0f40002f00370000052000865d020054
:10537c00010000000080fb004800dd00000f7800f9
:10538c0010052000865d0200010000000080fb007b
:10539c001e0f400023003700a0052000865d020090
:1053ac00010000000080fb004800dd00000f7800c9
:1053bc00b0052000865d0200010000000080fb00ab
:1053cc001e0f40001700370040062000865d0200cb
:1053dc00010000000080fb004800dd00000f780099
:1053ec0050062000865d0200010000000080fb00da
:1053fc001e0f40000b003700e0062000865d020007
:10540c00010000000080fb004800dd00000f780068
:10541c00f0062000865d0200010000000080fb0009
:10542c001e0f40001e0078000080fa0000000600ed
:10543c000800fa0010079800210798002e00900031
:10544c00000f78001e0078004800de00000f780086
:10545c001e009000300798003e009000e30f5000b3
:10546c003b0032003e009000e30f50000a003c006d
:10547c003e009000e10f50001f0032003e009000f3
:10548c00e10f500027003c003e0090000000e000bf
:10549c000e003200640037003e009000e50f500013
:1054ac00410032003e009000e50f50003300350003
:1054bc003e009000e60f5000460032003e00900087
:1054cc00e70f50004e003200570037001e007800e6
:1054dc0080407800a0022000825d020001000000e4
:1054ec002e00900080407800b0022000825d020007
:1054fc00010000004c0037001e007800804078004e
:10550c0040032000825d0200010000002e0090008c
:10551c008040780050032000825d020001000000f2
:10552c00410037001e00780080407800e003200026
:10553c00825d0200010000002e0090008040780087
:10554c00f0032000825d02000100000036003700ed
:10555c001e0078008040780080042000825d0200ec
:10556c00010000002e009000804078009004200084
:10557c00825d0200010000002b0037001e00780045
:10558c008040780020052000825d020001000000b0
:10559c002e0090008040780030052000825d0200d3
:1055ac0001000000200037001e00780080407800c9
:1055bc00c0052000825d0200010000002e0090005a
:1055cc0080407800d0052000825d020001000000c0
:1055dc00150037001e00780080407800600620001f
:1055ec00825d0200010000002e00900080407800d7
:1055fc0070062000825d0200010000000a003700e6
:10560c001e0078008040780000072000825d0200b8
:10561c00010000002e009000804078001007200050
:10562c00825d0200010000000080fa00000006000c
:10563c000600fa00100798000000eb00000f78003d
:10564c001e009000200798002e009000e30f5000e1
:10565c003e0032002e009000e30f50000a003c0088
:10566c002e009000e10f5000200032002e00900020
:10567c00e10f500029003c002e0090000000e000db
:10568c000e0032006c0037002e009000e50f500029
:10569c00460032002e009000e50f50003700350018
:1056ac002e009000e60f50004c0032002e009000af
:1056bc00e70f5000550032005f003700a0022000b9
:1056cc00865d0200010000000080fb004800dd0048
:1056dc00000f7800b0022000865d0200010000007f
:1056ec000080fb001e0f40005300370040032000d9
:1056fc00865d0200010000000080fb004800dd0018
:10570c00000f780050032000865d020001000000ad
:10571c000080fb001e0f400047003700e003200014
:10572c00865d0200010000000080fb004800dd00e7
:10573c00000f7800f0032000865d020001000000dd
:10574c000080fb001e0f40003b003700800420004f
:10575c00865d0200010000000080fb004800dd00b7
:10576c00000f780090042000865d0200010000000c
:10577c000080fb001e0f40002f003700200520008a
:10578c00865d0200010000000080fb004800dd0087
:10579c00000f780030052000865d0200010000003b
:1057ac000080fb001e0f400023003700c0052000c6
:1057bc00865d0200010000000080fb004800dd0057
:1057cc00000f7800d0052000865d0200010000006b
:1057dc000080fb001e0f4000170037006006200001
:1057ec00865d0200010000000080fb004800dd0027
:1057fc00000f780070062000865d0200010000009a
:10580c000080fb001e0f40000b003700000720003b
:10581c00865d0200010000000080fb004800dd00f6
:10582c00000f780010072000865d020001000000c8
:10583c000080fb001e0f40001e0078000080fa0064
:10584c00000006000800fa001007980021079800d5
:10585c002e009000000f78001e0078004800de003b
:10586c00000f78001e009000300798003e0090005a
:10587c00e30f50003b0032003e009000e30f50005d
:10588c000a003c003e009000e10f50001f00320067
:10589c003e009000e10f500027003c003e009000bd
:1058ac000000e0000e003200640037003e00900063
:1058bc00e50f5000410032003e009000e50f500013
:1058cc00330035003e009000e60f500046003200d9
:1058dc003e009000e70f50004e003200570037009a
:1058ec001e00780080407800c0022000825d02001b
:1058fc00010000002e00900080407800d0022000b3
:10590c00825d0200010000004c0037001e00780090
:10591c008040780060032000825d020001000000de
:10592c002e0090008040780070032000825d020001
:10593c0001000000410037001e0078008040780014
:10594c0000042000825d0200010000002e00900087
:10595c008040780010042000825d020001000000ed
:10596c00360037001e00780080407800a00420002c
:10597c00825d0200010000002e0090008040780043
:10598c00b0042000825d0200010000002b003700f3
:10599c001e0078008040780040052000825d0200e7
:1059ac00010000002e00900080407800500520007f
:1059bc00825d020001000000200037001e0078000c
:1059cc0080407800e0052000825d020001000000ac
:1059dc002e00900080407800f0052000825d0200cf
:1059ec0001000000150037001e0078008040780090
:1059fc0080062000825d0200010000002e00900055
:105a0c008040780090062000825d020001000000ba
:105a1c000a0037001e007800804078002007200024
:105a2c00825d0200010000002e0090008040780092
:105a3c0030072000825d0200010000000080fa00a7
:105a4c00000006000600fa00100798000000eb00aa
:105a5c00000f78001e009000200798002e00900088
:105a6c00e30f50003e0032002e009000e30f500078
:105a7c000a003c002e009000e10f50002000320084
:105a8c002e009000e10f500029003c002e009000e9
:105a9c000000e0000e0032006c0037002e00900079
:105aac00e50f5000460032002e009000e50f50002c
:105abc00370035002e009000e60f50004c003200ed
:105acc002e009000e70f5000550032005f003700a9
:105adc00c0022000865d0200010000000080fb0077
:105aec004800dd00000f7800d0022000865d020027
:105afc00010000000080fb001e0f40005300370027
:105b0c0060032000865d0200010000000080fb00a5
:105b1c004800dd00000f780070032000865d020055
:105b2c00010000000080fb001e0f40004700370002
:105b3c0000042000865d0200010000000080fb00d4
:105b4c004800dd00000f780010042000865d020084
:105b5c00010000000080fb001e0f40003b003700de
:105b6c00a0042000865d0200010000000080fb0004
:105b7c004800dd00000f7800b0042000865d0200b4
:105b8c00010000000080fb001e0f40002f003700ba
:105b9c0040052000865d0200010000000080fb0033
:105bac004800dd00000f780050052000865d0200e3
:105bbc00010000000080fb001e0f40002300370096
:105bcc00e0052000865d0200010000000080fb0063
:105bdc004800dd00000f7800f0052000865d020013
:105bec00010000000080fb001e0f40001700370072
:105bfc0080062000865d0200010000000080fb0092
:105c0c004800dd00000f780090062000865d020041
:105c1c00010000000080fb001e0f40000b0037004d
:105c2c0020072000865d0200010000000080fb00c0
:105c3c004800dd00000f780030072000865d020070
:105c4c00010000000080fb001e0f40001e007800c9
:105c5c000080fa00000006000800fa001007980007
:105c6c00210798002e009000000f78001e0078008d
:105c7c004800de00000f78001e00900030079800ee
:105c8c003e009000e30f50003b0032003e009000bd
:105c9c00e30f50000a003c003e009000e10f500062
:105cac001f0032003e009000e10f500027003c0026
:105cbc003e0090000000e0000e003200640037004f
:105ccc003e009000e50f5000410032003e00900075
:105cdc00e50f5000330035003e009000e60f5000f9
:105cec00460032003e009000e70f50004e0032009c
:105cfc00570037001e00780080407800e00220003a
:105d0c00825d0200010000002e00900080407800af
:105d1c00f0022000825d0200010000004c00370000
:105d2c001e0078008040780080032000825d020015
:105d3c00010000002e0090008040780090032000ad
:105d4c00825d020001000000410037001e00780057
:105d5c008040780020042000825d020001000000d9
:105d6c002e0090008040780030042000825d0200fc
:105d7c0001000000360037001e00780080407800db
:105d8c00c0042000825d0200010000002e00900083
:105d9c0080407800d0042000825d020001000000e9
:105dac002b0037001e007800804078006005200032
:105dbc00825d0200010000002e00900080407800ff
:105dcc0070052000825d02000100000020003700f9
:105ddc001e0078008040780000062000825d0200e2
:105dec00010000002e00900080407800100620007a
:105dfc00825d020001000000150037001e007800d3
:105e0c0080407800a0062000825d020001000000a6
:105e1c002e00900080407800b0062000825d0200c9
:105e2c00010000000a0037001e0078008040780056
:105e3c0040072000825d0200010000002e0090004f
:105e4c008040780050072000825d020001000000b5
:105e5c000080fa00000006000600fa001007980007
:105e6c000000eb00000f78001e0090002007980047
:105e7c002e009000e30f50003e0032002e009000e8
:105e8c00e30f50000a003c002e009000e10f500080
:105e9c00200032002e009000e10f500029003c0041
:105eac002e0090000000e0000e0032006c00370065
:105ebc002e009000e50f5000460032002e0090009e
:105ecc00e50f5000370035002e009000e60f500013
:105edc004c0032002e009000e70f500055003200ad
:105eec005f003700e0022000865d02000100000028
:105efc000080fb004800dd00000f7800f00220005d
:105f0c00865d0200010000000080fb001e0f4000b7
:105f1c005300370080032000865d02000100000062
:105f2c000080fb004800dd00000f7800900320008b
:105f3c00865d0200010000000080fb001e0f400087
:105f4c004700370020042000865d0200010000009d
:105f5c000080fb004800dd00000f780030042000ba
:105f6c00865d0200010000000080fb001e0f400057
:105f7c003b003700c0042000865d020001000000d9
:105f8c000080fb004800dd00000f7800d0042000ea
:105f9c00865d0200010000000080fb001e0f400027
:105fac002f00370060052000865d02000100000014
:105fbc000080fb004800dd00000f78007005200019
:105fcc00865d0200010000000080fb001e0f4000f7
:105fdc002300370000062000865d0200010000004f
:105fec000080fb004800dd00000f78001006200048
:105ffc00865d0200010000000080fb001e0f4000c7
:10600c0017003700a0062000865d0200010000008a
:10601c000080fb004800dd00000f7800b006200077
:10602c00865d0200010000000080fb001e0f400096
:10603c000b00370040072000865d020001000000c5
:10604c000080fb004800dd00000f780050072000a6
:10605c00865d0200010000000080fb001e0f400066
:10606c001e0078000080fa00000006000600fa000e
:10607c00000f7800214798001e0078002007980038
:10608c002e009000e30f5000290032002e009000eb
:10609c00e30f50000a003c002e009000e10f50006e
:1060ac00190032002e009000e10f50001b003c0044
:1060bc002e0090000000e0000e003200340037008b
:1060cc002e009000e50f5000230032002e009000af
:1060dc00e50f50001b0035002e009000e60f50001d
:1060ec00220032002e009000e70f500024003200f6
:1060fc0027003700ae40900060072000825d020050
:10610c000100000022003700ae4090007007200014
:10611c00825d0200010000001d003700ae409000bf
:10612c0080072000825d020001000000180037008b
:10613c00ae40900090072000825d0200010000003c
:10614c0013003700ae409000a0072000825d0200d3
:10615c00010000000e003700ae409000b007200098
:10616c00825d02000100000009003700ae40900083
:10617c00c0072000825d020001000000040037000f
:10618c00ae409000d0072000825d020001000000ac
:10619c000080fa00000006000600fa00000f7800ec
:1061ac001e007800200798002e009000e30f50008e
:1061bc002c0032002e009000e30f50000a003c002f
:1061cc002e009000e10f50001a0032002e009000bb
:1061dc00e10f50001d003c002e0090000000e0007c
:1061ec000e0032003d0037002e009000e50f5000ed
:1061fc00280032002e009000e50f50001f003500e3
:10620c002e009000e60f5000280032002e00900067
:10621c00e70f50002b0032003000370060072000e1
:10622c00865d0200010000000080fb001007980052
:10623c002c00370070072000865d02000100000072
:10624c000080fb0010079800260037008007200014
:10625c00865d0200010000000080fb001007980022
:10626c002000370090072000865d0200010000002e
:10627c000080fb00100798001a003700a0072000d0
:10628c00865d0200010000000080fb0010079800f2
:10629c0014003700b0072000865d020001000000ea
:1062ac000080fb00100798000e003700c00720008c
:1062bc00865d0200010000000080fb0010079800c2
:1062cc0008003700d0072000865d020001000000a6
:1062dc000080fb0010079800020037000000eb0064
:1062ec00100798001e0090000080fa0000000600c5
:1062fc000400fa00100798000000eb00000f780073
:10630c000b0037001e007800800078001e00900003
:10631c00008040001040780080407800420b200044
:10632c001e004100825d0200010000001e0fe8000b
:10633c00500020009e0f1000f2ff34000080fa0085
:10634c00000006000400fa00881f7800100798006f
:10635c000000eb00000f78000a0037001e007800e8
:10636c00800078001e00900000844000410b20004b
:10637c001e804000865d020001000000004c780089
:10638c001e0fe800500020009e0f1000f3ff340099
:10639c001e009000e60040000040eb0080487800b2
:1063ac001e0090004f0478000080fa0000000600e8
:1063bc000400fa000000eb00000f78000000eb0076
:1063cc00100798001b0037009e0078006a80400080
:1063dc00800078001e00900010fb0700b104200024
:1063ec001e804000800078001e00900010fc07000a
:1063fc00d10720001e804000800078001e00900015
:10640c0010fd0700c13f20001e8040008000780076
:10641c001e00900010fe07008040eb001e00900054
:10642c0012ff07001e0fe8001e0090000000e8009d
:10643c00100798001e009000e70f5000e2ff340098
:10644c000080fa00000006000000fa0070c0b300e3
:10645c002f00070000cbb300350007000080fa00c6
:10646c00000006000000fa000040eb0092f3b700b9
:10647c000080fa00000006000000fa000102200073
:10648c00c08d2900a3fa07000080fa000000060066
:10649c000200fa00004f78009e407800e00b2000cc
:1064ac00825d0200010000000080fa00000006007e
:1064bc000200fa00e00b2000865d020001000000e3
:1064cc00004f78001e80fb000080fa0000000600e0
:1064dc000200fa00004f78009e407800000c20006b
:1064ec00825d0200010000000080fa00000006003e
:1064fc000200fa00000c2000865d02000100000082
:10650c00004f78001e80fb000080fa00000006009f
:10651c000200fa00004f78009e407800800c2000aa
:10652c00825d0200010000000080fa0000000600fd
:10653c000200fa00004f78009e407800900c20007a
:10654c00825d0200010000000080fa0000000600dd
:10655c000000fa00800c2000865d020001000000a3
:10656c000080fb000080fa00000006000000fa002a
:10657c00900c2000865d0200010000000080fb00f2
:10658c000080fa00000006000a00fa00881f78005c
:10659c000e80e8006bff07000e80e8005040900072
:1065ac008001fb000e80e800404090000002fb00e0
:1065bc000e80e800304090008002fb000e80e80066
:1065cc00204090008000fb000e80e80010409000fe
:1065dc000001fb000e80e800104078000000fb007a
:1065ec00831f7800841f7800851f7800811f780036
:1065fc00821f7800801f7800d08f2900801f7800c0
:10660c00b262020001000000ee8757000e80e80025
:10661c009040780030c5b30080cf500019003a008c
:10662c000e80e8009040900090c4b30080cf5000e2
:10663c0014003a000e80e800a040900070c4b30033
:10664c0080cf50000f003a000e80e800b040900060
:10665c0010c3b30080cf50000a003a000e80e8004f
:10666c00c040900000c3b30080cf500005003a003a
:10667c000e80e800d040900070c3b30080cf500073
:10668c006b00320030c5b3008000fb000e80e800c8
:10669c00104078000000fb00811f7800801f7800fc
:1066ac0080912900801f7800b26202000100000076
:1066bc00e687570090c4b3008000fb000e80e80012
:1066cc00104090000000fb00811f7800801f7800b4
:1066dc0080912900801f7800b26202000100000046
:1066ec00e687570070c4b3008000fb000e80e80002
:1066fc00204090000000fb00811f7800801f780074
:10670c0080912900801f7800b26202000100000015
:10671c00e687570010c3b3008000fb000e80e80032
:10672c00304090000000fb00811f7800801f780033
:10673c0080912900801f7800b262020001000000e5
:10674c00e687570000c3b3008000fb000e80e80012
:10675c00404090000000fb00811f7800801f7800f3
:10676c0080912900801f7800b262020001000000b5
:10677c00e687570070c3b3008000fb000e80e80072
:10678c00504090000000fb00811f7800801f7800b3
:10679c0080912900801f7800b26202000100000085
:1067ac00e687570002ff070027ff07002dff0700b1
:1067bc0031ff070030922900cdfe07000000eb00ee
:1067cc00fc4402000100000010002000fc44020008
:1067dc000100000020002000fc4402000100000029
:1067ec0030002000fc4402000100000040002000aa
:1067fc00fc4402000100000050002000fc44020098
:10680c000100000060002000fc44020001000000b8
:10681c0070002000fc44020001000000a09229003e
:10682c00801f7800b2620200010000008f87e9002f
:10683c000000eb00000f7800080037001e04780001
:10684c001e00780054fe070080407800600c210088
:10685c0000004400014878001e0fe8007000200082
:10686c009e0f1000f5ff3400e00c2100bff907006b
:10687c00e3f9070092f3b7000dff070080407800a2
:10688c00e0c6b30080cf50000200360070c1b300e8
:10689c00fffe070016ff0700e14f400002003a0020
:1068ac000040eb000aff070001ff07000080fb001f
:1068bc0000a1880000a18000f0a088000cff070058
:1068cc0095f3b70095d3bf0096f3b7004f0478004b
:1068dc000080fa00000006009ec0a9008ea4ef0004
:1068ec008aa4ef00aa24ef00ac24ef0020002000c3
:1068fc0030258800a824ef008644a900f009200068
:10690c0080248800602488008804a80001202100cd
:10691c004808de00c02488000000eb008018eb0063
:10692c008018eb000000e800e80f5000fbff3a0075
:10693c009424a8009624ef0094a4a9009424a90000
:10694c0021382100914078000001780005003700c3
:10695c00522488007473ef007573ef007673ef00a8
:10696c008040eb008ac4bf000038a300f8ff3a0057
:10697c000100780082f3b70010002000a09a880074
:10698c00909a88008633ef008a33ef007c33ef0057
:10699c000000eb00a4362100e236210080007800d4
:1069ac009535210073352100001aeb000019eb001e
:1069bc0001f07a0001f079000000e800e20f5000cd
:1069cc00f9ff3a0080202100509b8800d000200065
:1069dc0050258800a03421001090880080c0b3009e
:1069ec0000f2b70040c8b30001f2b7000100780014
:1069fc0079f3b7007a33ef00000006005413e2007d
:106a0c0020003a0014002000a49a8800919a80007b
:106a1c000100e0001b003a00949a880062d3bf008a
:106a2c00e24f500006003a00509b8000014878006d
:106a3c0081ccb300509b80001140980000000600f0
:106a4c00e14f50000f003a0083c0b300309b800030
:106a5c0003487800319b8000a234210092009800fa
:106a6c0040c8b30090409800e49a8800209b8000b6
:106a7c0003487800219b80009200980000c8b30066
:106a8c0090409800000006000080fb008001400050
:106a9c000180fb00008041004300dd00022021004a
:106aac0002014000124090000070a10010419800bb
:106abc00e03621000104e00001003200a036210084
:106acc0082317800124090000060a10010419800c3
:106adc00e4004100114090000060a000904098003c
:106aec0000000600889fbe008a1f780000447800d2
:106afc00014578008184fb000938a30002003200b4
:106b0c008040eb00e0ff07000928a30003003200df
:106b1c0011c0b30008407800dbff07000880fb00c1
:106b2c0000004000a14a20000af078004f057800d0
:106b3c004f04be0000000600004378000082fb00fa
:106b4c00814378000104e00003003200840042001d
:106b5c00a03621000200370084004200e0362100fc
:106b6c00e10278000500e00002003a000500780020
:106b7c00000006000682fb0092029800834a78000f
:106b8c00154090000044b2009042980015409000cf
:106b9c0081c8b30001407000904298000704e000e7
:106bac000300320004004200a1362100020037002d
:106bbc0004004200e1362100010040001024a20034
:106bcc000500780000000600014178000004e00098
:106bdc000c003a0081c0b300209b80000148780073
:106bec00219b8000a034210090009800c0c8b30005
:106bfc009040980041c8b300509b80001140980011
:106c0c00000006008080fb00818040000280fb00b9
:106c1c0080804000c308dd0002202100028140007a
:106c2c001240900043c8b30003407000104198001c
:106c3c0040202100808040001140900003407000f3
:106c4c0090409800000006008040780094c4bf007b
:106c5c000058a300180032000181fb000201410022
:106c6c00a4362100e2017a001300be0005042000c6
:106c7c0000806200010020008089be00e2017a00e1
:106c8c000004200001002000931968009391680013
:106c9c00040141001224a2009200780011409000df
:106cac000044b2009040980092007800114090008f
:106cbc00054068009040980000000600219c800070
:106ccc0083c0b300e78f500009003e00814178007b
:106cdc0063d3bf0002003a0010c0b30003003700ba
:106cec00e14f500002003a0020c0b30063f3b7003c
:106cfc000380fb0000805000209c8800509b80008b
:106d0c000348780020342100009b88008213ab00dc
:106d1c000200320003417800120037000341780072
:106d2c008041eb0006003700009b8000019c800036
:106d3c0031587800009b8800019c88000241e900d2
:106d4c00834f5100f8ff3a0000000600009b8000c2
:106d5c00019c800031587800009b8800019c8800c1
:106d6c000241e9000204e000f8ff3a0000000600ce
:106d7c008633ef008a33ef002036210021c0b300a8
:106d8c0090cf100009003a0081c0b300209b800016
:106d9c0001487800219b800020342100900098004d
:106dac0080ccb300904098000000060050d3bf0088
:106dbc000080fb001135210091407800c808dd00ef
:106dcc0080807000209c8000808f50000700310074
:106ddc0001352100914078008180fb0051d3bf0028
:106dec004800dd0001007000209c8800b3ff070004
:106dfc0021342100509b80001100980081ccb300fd
:106e0c00509b800011409800000006000200fa0020
:106e1c00889fbe008a1f78007a13e20010003a00a7
:106e2c009424ef008c24ef002000200030258800f3
:106e3c00a824ef008644a900f009200080248800d3
:106e4c0060248800010037009404a80094c4bf009b
:106e5c000008a300fcff320010002000d09b88002b
:106e6c00d09b8000e10f500009003a0094c4bf0091
:106e7c000068a30006003a008aa4ef008c24ef00ff
:106e8c008c04a8008c84a80020002000d09b8800d3
:106e9c0080c4bf000048a3000d00320082c4bf00b4
:106eac000048a3000a0032000801200008248800d2
:106ebc007c33ef000001eb008000eb00400720006a
:106ecc00d84e0200010000008284a900082488002a
:106edc0088c4bf000018a300ca023a008ac4bf00cd
:106eec000008a300080032008cc4bf000008a300f7
:106efc000500320078fe070040002000d09b88007f
:106f0c0010002000502488008ac4bf000048a30051
:106f1c000e0032008cc4bf000048a3000b003200ee
:106f2c008284a8000801200058248800100020004a
:106f3c00e09b88000001eb008000eb005007200074
:106f4c00d84e020001000000582488008ac4bf00fb
:106f5c000028a300100032008cc4bf000028a3003e
:106f6c0005003200120020008000eb0030072000ea
:106f7c00d84e020001000000400020005024880080
:106f8c0056d3bf00030032000040e90056f3b700af
:106f9c0001003a0099fe07008a44e20014003d000b
:106fac008c44e20012003d00aac4bf000018a300ec
:106fbc000d003200329b80009240900000c8b3005c
:106fcc0080cf500007003a00509b8000904090000a
:106fdc0040c8b30080cf500002003a006840400027
:106fec0010419800aa24a900000820005024880011
:106ffc008ac4bf000018a3000b0032008cc4bf0071
:10700c000018a30008003200120020008000eb00e2
:10701c00f0ff2700d84e0200010000008ea4ef0004
:10702c002000200050248800d09b8000e30f5000eb
:10703c00740236008cc4bf000038a3007102320009
:10704c000045eb008ac4bf000038a3006d0232007b
:10705c00902480005ff3b7008080fb00c409de0041
:10706c008001fd005ef3b7008001fd00810020006f
:10707c0051248800723521000038a3000100320031
:10708c009235210063407900e14060000104a200c8
:10709c000004a10001407000807179005e53e20091
:1070ac0050023a00d0c2b30056f3b7005fd3bf0012
:1070bc008080fb00810178000320a1000300e00028
:1070cc0011023a00c10fb2000020210000814000e3
:1070dc00329b8800229b88006453aa0012409000c7
:1070ec00c043b20041c3b300814f5000ab013a0022
:1070fc0082007800a23421001100900010f1790078
:10710c00110090000000e800900098008301e80056
:10711c00e88f5100f8ff3a00920098006373ef007b
:10712c008833ef008633ef008a33ef005c33ef00d7
:10713c006273ef00519b8000114090000074a1001d
:10714c00904098006a53aa00519b80001140900017
:10715c000074a100904098006a53aa00219b800003
:10716c00114090000074a100904098008273ef00d1
:10717c008433ef007473ef007573ef007673ef00d8
:10718c004ad3bf000046b20051013a004bd3bf00b6
:10719c000080fb0001002000eb0f5000e08f580036
:1071ac004b013e0000600100640037009100370085
:1071bc00470137008f0037004501370006003700c4
:1071cc00080037003d0137005a0037003300370004
:1071dc00280137003101370082f3a800800020001d
:1071ec004b003700a13421009140780000c8b30057
:1071fc0080cf500036013a0000ccb30082f3b700c8
:10720c004dd3bf00e24f500008003200e34f500056
:10721c0012003200e14f50001e003a00a011210074
:10722c00009c880020012000180037004cd3bf00c0
:10723c000080fb000000400001412100e08078004c
:10724c00019c8800019c80002140900084f3b700d1
:10725c003140900085f3b7001d0137004cd3bf00bf
:10726c00e24f50000b003e004cd3bf000080fb00ef
:10727c00000040002141210060807800009c8800c3
:10728c00009c8000104078000080fb00209c88004f
:10729c000f0137008273ef000d01370082f3a80055
:1072ac00ac24ef00020220008000eb000020210043
:1072bc0088f20200000000009424a8000000eb00fb
:1072cc0093352100804078007235210001f079005f
:1072dc00017079000000e800e20f5000fbff3a005b
:1072ec000100780068f3b7009424a90080202100e5
:1072fc00509b880000202100309b8800209b880038
:10730c004cd3bf0079f3b70003003a000001200012
:10731c00d09b8800ee00370012002000913721002e
:10732c0010002000d84e02000100000000022000d6
:10733c00f7ff370090372100d20037004273ef007f
:10734c004373ef004ad3bf007f006000e10f500091
:10735c000b003200e20f50000b0032000000e00086
:10736c001c003a0082f3a8004213a800f09b800096
:10737c00e10f500017003a004233a8001500370007
:10738c0082f3a8001300370082f3a8004e53e200ea
:10739c00050035004ed3bf006f00600000004000b8
:1073ac00e1362100040037004ed3bf006f006000af
:1073bc0000004000a13621006080780001402800c8
:1073cc0010806000810f500002003a0010c0b30022
:1073dc0042f3b70082f3ab00bd0032002034210031
:1073ec00009c88008213a80020c0b30084f3b7006f
:1073fc00b70037004cd3bf00e14f50000b003a00f0
:10740c004ad3bf007f40600008003a0082f3a80016
:10741c004bd3bf00e34f500003003a001000200094
:10742c00f09b8800010037007e33ef004c53e200e4
:10743c00a7003a004ad3bf007f406000e24f5000e3
:10744c00a3003a004ed3bf006f406000a000320092
:10745c004ed3bf006f006000e10f50009c003c0059
:10746c00d19b800000022000808f500098003a00d1
:10747c0082f3a8004e53e2000a0035004ed3bf0041
:10748c006f00600000004000e13621006080780051
:10749c00c0bf9f004ed3bf006f006000713521004c
:1074ac00090037004ed3bf006f00600000004000a1
:1074bc00a136210060807800c0bf9f004ed3bf0072
:1074cc006f0060009135210060c478000808a300ab
:1074dc0004003a008ff897000124a10081ff9f005f
:1074ec00030037000ff997000224a00082ff9f00d1
:1074fc004e53e200050035004ed3bf006f00600014
:10750c0000004000e1362100040037004ed3bf00dc
:10751c006f00600000004000a13621004fb99700b9
:10752c0002b078004bd3bf00e34f500015003a0077
:10753c004fb897001000e0000c003d004e53e200e5
:10754c00040035004ed3bf006f006000723521007f
:10755c00030037004ed3bf006f006000923521004e
:10756c00e04079000114a000017079004fb8970039
:10757c009040900042c8b30082c070001140980047
:10758c0053003700e88457000ff897000024a2003e
:10759c0080ff9f00cfb89700114090001100e000d1
:1075ac000c003d000074a10090409800cfb89700eb
:1075bc00114090000064a000904098002200200030
:1075cc00cfb8970050002000d84e020001000000f8
:1075dc00020037000064a000904098001924a2001b
:1075ec000818a30003003a00cfb897001100e00080
:1075fc0016003d004e53e200040035004ed3bf0090
:10760c006f00600072352100030037004ed3bf00bd
:10761c006f00600092352100e04079000114a10058
:10762c0001707900cfb8970011409000b043b200c0
:10763c009040980022002000cfb897005000200006
:10764c00d84e0200010000000300370011409000ea
:10765c00b043b200904098004ed3bf006f00600062
:10766c0000004000a14a2000010040001014a100bd
:10767c00170037004ed3bf000080fb00813621007d
:10768c0001004000009c88008213a80010c0b300c9
:10769c0084f3b70082f3a8000d00370082f3a80032
:1076ac004ed3bf000080fb0081362100c234210084
:1076bc001241780002f07800050037000001eb0061
:1076cc008000eb0020002000d84e020001000000da
:1076dc000001eb008000eb0030002000d84e0200cf
:1076ec000100000094a4a900189c80000808b200b6
:1076fc0013003a007453e20008003d0020c0b300b0
:10770c0062f3b7008a13e20001003a0098fd07000b
:10771c00989a8800a89a8800b700370081c0b300f7
:10772c00209b800001487800219b8000a034210020
:10773c0090009800c0c8b3009040980090003700ab
:10774c004a53e20006003d0010c0b30062f3b700dc
:10775c008613e2000c003a0085fd07000a00370092
:10776c0020c0b30062f3b70081c0b300209b80003f
:10777c0001487800219b8000a034210090009800e3
:10778c0040c8b300904098005233ef005433ef00e0
:10779c008813e20098003a004a0037002036210096
:1077ac0021c0b30090cf100048003a00124278007c
:1077bc0075d3bf000080fb00613721009140780039
:1077cc00c808dd00808070000480fb00810f500031
:1077dc0001003600014278000480fb00008050005c
:1077ec0075f3b7004800de0076f3b70025342100ae
:1077fc000e00370072d3bf000080fb003137210030
:10780c0091407800c808dd00808070000280fb0089
:10781c00e0d87a000100780072f3b700c808de00e7
:10782c000100780073f3b7008301e800034178008e
:10783c0084cf5100efff3900229b8000513721008b
:10784c00914078008180fb0076d3bf004800dd00ba
:10785c00010070000a00320080c0b30000497800bb
:10786c00219b80002034210090009800309b8000e8
:10787c00104090000068a300480032004900370017
:10788c0080c0b30000497800219b8000a034210007
:10789c009000980040c8b3009040980071372100c8
:1078ac00914078008180fb0078d3bf004800dd0058
:1078bc0001007000010032000000010074f3a90007
:1078cc00b3ff37004dfc07004b0037008001fd0073
:1078dc0062f3b7008001fd005c13e20008003a007f
:1078ec0081c0b300209b800001487800219b800060
:1078fc00a034210090009800c0c8b3002a003700c3
:10790c00e39a88003c003700e88f51003a003a00b7
:10791c00509b8000104090004600de006104600027
:10792c006a53aa00d09b8000e80f500008003a0070
:10793c004cd3bf000080fb00b02488000001200065
:10794c009604e20001003a0040002000d09b880021
:10795c002036210012c0b300904f110014003a00e1
:10796c0020342100519b800090009800d3fc07002c
:10797c003036210021c0b30090cf100004003a0033
:10798c0041c8b300509b8000114098001a0037008a
:10799c00519b80000804e00002003a0080ccb30048
:1079ac000100370080c8b3009040980012003700e7
:1079bc007453e20009003d007137210091407800ba
:1079cc008180fb0078d3bf004800dd00010070000f
:1079dc00010032000000010074f3a9006273ef0093
:1079ec00050037000001eb00f135210020072000d5
:1079fc00d84e0200010000000a45e800e44f550093
:107a0c0090fd3a008ec0a9004f0578004f04be00cf
:107a1c000080fa00000006001c00fa00889fbe00df
:107a2c008a9fbe008c9fbe00005798000e5090009d
:107a3c000000fb006101b90000fe2f00f1ff2f00d8
:107a4c000201400083814800320f9800430f9800d8
:107a5c00a0052000010020003e099000ce099000f6
:107a6c00800f5100818f59008a023e003e08900021
:107a7c00ce089000006001005202370085023700ea
:107a8c0084023700830237008202370081023700fc
:107a9c00800237007f0237007e0237007d023700fc
:107aac007c0237007b0237007a02370079023700fc
:107abc0078023700770237004a0037005000370051
:107acc00530037005600370076003700a20037000d
:107adc00a4003700bc003700be0037006d02370031
:107aec006c0237006b0237006a02370069023700fc
:107afc00680237003302370066023700cf003700c8
:107b0c00d2003700d5003700d8003700da00370034
:107b1c00dc003700e4003700ea003700f0003700e3
:107b2c00f6003700fc00370014013700b4013700b1
:107b3c00be01370057023700c9013700f101370089
:107b4c00f401370007023700090237000b02370037
:107b5c000d0237000f0237001102370013023700f5
:107b6c00150237004b0237004a0237004902370032
:107b7c00480237004702370046023700af00370093
:107b8c00b2003700b5003700b8003700ba00370034
:107b9c00bc003700c4003700ca003700d0003700e3
:107bac00d6003700dc003700f400370094013700b2
:107bbc009e01370037023700a9013700d101370089
:107bcc00d4013700e7013700e9013700eb0137003a
:107bdc00ed013700ef013700f1013700f3013700f9
:107bec00f50137000040eb000661020001000000c7
:107bfc000040eb001a610200010000002502370072
:107c0c0010c0b3001a63020001000000210237000b
:107c1c000040eb001a630200010000001d02370057
:107c2c0068004700a831020001000000680047000e
:107c3c00504090008001fb006800470040409000dd
:107c4c000002fb0068004700304090008002fb00ff
:107c5c0068004700204090008000fb00680047004f
:107c6c00104090000001fb006800470010407800b5
:107c7c000000fb00831f7800841f7800851f7800ac
:107c8c00811f7800821f7800801f7800004a29002d
:107c9c00801f7800b262020001000000ee875700de
:107cac00fc01370001848000510f9800f1838000a3
:107cbc00e2838000d3838000c4838000b58380007e
:107ccc00a68380009783800088838000798380005e
:107cdc006a8380005b8380004c8380003d8380003e
:107cec0020838000200f980010838000100f9800d4
:107cfc005e089000801f7800811f7800821f78003a
:107d0c00831f7800841f7800851f7800861f7800f9
:107d1c00871f7800881f7800891f78008a1f7800d9
:107d2c008b1f78008c1f78008d1f7800ae08900098
:107d3c00811f78001e099000821f7800b04b29002b
:107d4c00801f7800b262020001000000e0fd2f00ed
:107d5c0080874700cf013700ee430200010000008e
:107d6c00cc013700e04f2900801f7800b26202007e
:107d7c00010000008f87e9000000eb00300798003d
:107d8c000d003700be019000831f78009050290031
:107d9c00801f7800b262020001000000e4875700e7
:107dac003e00900054430200010000003e00900091
:107dbc000000e800300798003e009000e70f5000ec
:107dcc00f0ff3400b3013700ee190200010000008f
:107ddc00b001370080022000865d02000100000027
:107dec000080fb004800dd00200798002e0090006a
:107dfc00801f780020512900801f7800b262020099
:107e0c0001000000e487570090022000865d02000c
:107e1c00010000000080fb0020079800ae009000dd
:107e2c00811f7800e0512900801f7800b2620200a7
:107e3c0001000000e4875700960137000040eb007a
:107e4c00f6270200010000009201370010c0b300b9
:107e5c00f6270200010000008e01370020c0b3009d
:107e6c00f6270200010000008a01370010c0b300a1
:107e7c0093f3b700870137000040eb0093f3b70092
:107e8c008401370093d3bf000000fb00801f7800f3
:107e9c00c0522900801f7800b2620200010000006d
:107eac00e48757007b013700f20029000300200013
:107ebc0000002800010020006a55020001000000ab
:107ecc0074013700028f29000300200000002900f4
:107edc00010020006a550200010000006d0137000e
:107eec00020f2a000300200000ff290001002000df
:107efc006a5502000100000066013700020f2f00d6
:107f0c000300200000002f00010020006a55020031
:107f1c00010000005f013700020f27000300200062
:107f2c0000002700010020006a550200010000003b
:107f3c00020f280003002000000028000100200090
:107f4c006a55020001000000020f29000300200006
:107f5c0000002900010020006a5502000100000009
:107f6c00020f2f000300200000002e000100200053
:107f7c006a55020001000000460137000001eb00c9
:107f8c000000270001002000105802000100000032
:107f9c0012002000200027000100200010580200d1
:107fac0001000000220020004000270001002000fa
:107fbc001058020001000000320020006000270071
:107fcc0001002000105802000100000042002000b7
:107fdc008000270001002000105802000100000062
:107fec0052002000a00027000100200010580200c1
:107ffc000100000062002000c000270001002000ea
:10800c00105802000100000072002000e000270060
:10801c00010020001058020001000000a200200006
:10802c000000280001002000105802000100000090
:10803c00b20020002000280001002000105802008f
:10804c0001000000c20020004000280001002000b8
:10805c001058020001000000d2002000600028002f
:10806c00010020001058020001000000e200200076
:10807c0080002800010020001058020001000000c0
:10808c00f2002000a000280001002000105802007f
:10809c000100000002012000c000280001002000a7
:1080ac00105802000100000012012000e00028001e
:1080bc0001002000105802000100000042012000c5
:1080cc0000002900010020001058020001000000ef
:1080dc00520120002000290001002000105802004d
:1080ec000100000062012000400029000100200076
:1080fc0010580200010000007201200060002900ed
:10810c000100200010580200010000008201200034
:10811c00800029000100200010580200010000001e
:10812c0092012000a000290001002000105802003c
:10813c0001000000a2012000c00029000100200065
:10814c001058020001000000b2012000e0002900dc
:10815c00010020001058020001000000e201200084
:10816c0000ff2e000100200010580200010000004a
:10817c00f201200020ff2e00010020001058020008
:10818c00010000000202200040ff2e000100200030
:10819c0010580200010000001202200060ff2e00a7
:1081ac0001002000105802000100000022022000f3
:1081bc0080ff2e000100200010580200010000007a
:1081cc0032022000a0ff2e000100200010580200f7
:1081dc000100000042022000c0ff2e000100200020
:1081ec00105802000100000052022000e0ff2e0097
:1081fc00010020001058020001000000a50037000b
:10820c00d09f800001002000008fbe0000002100e4
:10821c00010020003e014000ae8148001e00be005f
:10822c002a550200010000009a0037000000eb0004
:10823c00fc4402000100000010002000fc4402007d
:10824c000100000020002000fc440200010000009e
:10825c0070002000fc440200010000008d0037007b
:10826c000000280001002000ec5702000100000073
:10827c00801f7800b0532900801f7800b262020082
:10828c0001000000e48757002000280001002000b6
:10829c00ec57020001000000801f78007054290088
:1082ac00801f7800b262020001000000e4875700d2
:1082bc004000280001002000ec57020001000000e3
:1082cc00801f780030552900801f7800b2620200b0
:1082dc0001000000e4875700600028000100200026
:1082ec00ec57020001000000801f7800f0552900b7
:1082fc00801f7800b262020001000000e487570082
:10830c00640037000000eb00544302000100000041
:10831c006000370001a1800022d4bf000000fb00e8
:10832c00811f7800801f7800b0562900801f7800cc
:10833c00b262020001000000e68757007e320200a4
:10834c00010000000080fb00801f7800e05729002e
:10835c00801f7800b262020001000000e487570021
:10836c004c0037004000200000a188004900370075
:10837c00b000200000a188004600370060012000fa
:10838c0000a18800430037001002200000a18800e3
:10839c0040003700c002200000a188003d003700db
:1083ac007003200000a188003a003700d0042000a0
:1083bc0000a18800370037003006200000a188009b
:1083cc003400370030582900801f7800b262020058
:1083dc00010000008f87e9000000eb00801f78008f
:1083ec0080582900801f7800b26202000100000052
:1083fc00e4875700205a2900801f7800b2620200df
:10840c00010000008f87e900705a2900801f780056
:10841c00b2620200010000008f87e900c05a2900f7
:10842c00801f7800b2620200010000008f87e90013
:10843c00105b2900801f7800b2620200010000006e
:10844c008f87e900605b2900801f7800b262020010
:10845c00010000008f87e900b05b2900801f7800c5
:10846c00b2620200010000008f87e900005c290065
:10847c00801f7800b2620200010000008f87e900c3
:10848c00505c2900801f7800b262020001000000dd
:10849c008f87e9004f06be004f05be004f04be009b
:1084ac000080fa00000006000200fa000040eb0019
:1084bc00004f780010c0b300f3f3b70001e6a90039
:1084cc0007e2a9005c00a90000c02f006019880019
:1084dc00c122a800c142a800c1c2a800c1e2a800e4
:1084ec00c802a800c822a800c842a800c862a800f8
:1084fc00c882a800c8a2a800c8c2a900c8e2a900e6
:10850c00c902a800c922a800c942a800c962a900d2
:10851c00c982a800c9a2a800c9c2a900c9e2a800c2
:10852c00cd62a900d022a800d062a800d1a2a800d8
:10853c00d1c2a800d802a800d822a800d842a8000e
:10854c00d862a800d882a800d8a2a800d8c2a800d7
:10855c00d8e2a800d902a800d922a800d942a800c4
:10856c00d962a800d982a900d9a2a900d9c2a800b1
:10857c00d9e2a800dd82a800dda2a900e002a800d3
:10858c00e022a800e042a800e062a800e082a80077
:10859c00e0a2a800e0c2a800e0e2a800e102a80066
:1085ac00e122a800e802a800e822a800e842a800fe
:1085bc00e862a900e882a800e8a2a800e902a800e5
:1085cc00ec62a900f002a800f022a800f0c2a800fa
:1085dc00f0e2a800f102a800f122a8000000eb00d4
:1085ec00003a8800f068020001000000a05c29003d
:1085fc00801f7800b2620200010000008f87e90042
:10860c002e610200010000003a630200010000002c
:10861c0010c0b3001a61020001000000fc600200ef
:10862c000100000010c0b300066102000100000050
:10863c00a05c2900801f7800b262020001000000db
:10864c008f87e900100020002811020001000000b3
:10865c000040eb001a610200010000000040eb003a
:10866c0006610200010000006458020001000000d5
:10867c00b468020001000000004f78001e04e00006
:10868c00020032001e407800e3fc07008c5f020001
:10869c00010000000060fe00f5ff37000e00fa003c
:1086ac00600798000000eb00400798006e009000f7
:1086bc0080004000803f21000080400010007800c6
:1086cc000100200020079800310798006e009000f0
:1086dc00801f7800c05d2900801f7800b262020004
:1086ec0001000000e48757000000eb0050079800e1
:1086fc002e009000be009000008fbe0029003700b5
:10870c00e05e2900801f7800b262020001000000c8
:10871c008f87e9001e00be00ec570200010000002c
:10872c00801f7800005f2900801f7800b262020071
:10873c0001000000e4875700505f2900801f78007b
:10874c00b2620200010000008f87e9005e00900019
:10875c000000e800500798004e0090000000e80070
:10876c00400798005e009000ef0f500009003400a5
:10877c000000eb0050079800ce009000811f78009d
:10878c00805f2900801f7800b262020001000000a7
:10879c00e487570020002000010020001e0f40003d
:1087ac005e9748002e009000be00900002802000d2
:1087bc00030020000000410081804900be0f5000e2
:1087cc00ae8f5800ceff3c000080fa00000006007f
:1087dc001000fa0000602900801f7800b2620200cd
:1087ec00010000008f87e9000000eb007007980083
:1087fc003f003700fe009000600c2100008040001c
:10880c00104078000080fb004300de006100600037
:10881c0060079800fe009000600c21000080400072
:10882c00104078000080fb00610060005007980049
:10883c00fe009000600c2100008040001040780089
:10884c000080fb004200de006100600040079800e1
:10885c007e009000142902000100000030079800ef
:10886c007e0090001e2b02000100000020079800e3
:10887c007e009000282d02000100000010079800d7
:10888c007e009000322f020001000000000f7800e3
:10889c001e007800801f78001e009000801f78005a
:1088ac002e009000801f78003e009000801f780002
:1088bc005e009000801f78006e009000801f780092
:1088cc004e009000801f78007e009000801f780082
:1088dc00f0602900801f7800b262020001000000e5
:1088ec00f28757007e0090000000e80070079800a7
:1088fc007e009000e70f5000beff34000080fa00ad
:10890c00000006000c00fa00500798005e00900072
:10891c000000e00002003d000000eb005007980052
:10892c005e009000e70f5000020034007000200041
:10893c00500798005e00900080004000803f2100ae
:10894c000080400010007800010020001007980003
:10895c00210798001e019000ae019000000021003c
:10896c000100200002014000838148001e0090009d
:10897c00ae0090002a550200010000001e0090007d
:10898c00ae00900030079800410798000000eb0003
:10899c00000f7800100037001e00780080004000a7
:1089ac002080200000804000100178003e009000e4
:1089bc00ce00900010580200010000003e00900014
:1089cc00ce00900062004000e08048003007980024
:1089dc00410798001e0fe800f03f20009e0f10008a
:1089ec00edff34000080fa00000006004800fa0099
:1089fc00701798007e1090001429020001000000ee
:108a0c00300798007e1090001e2b02000100000021
:108a1c00200798007e109000282d02000100000015
:108a2c00100798007e109000322f02000100000009
:108a3c00000f7800fe109000600c210000804000b8
:108a4c0090407800414f98004e4890000080fb0009
:108a5c004200de00610060000004e000ea00320029
:108a6c007e109000801f780000652900801f780020
:108a7c00b262020001000000e48757003e00900043
:108a8c00cf80de008c05020001000000001f980062
:108a9c00111f98003e0090000000e00008003d000f
:108aac0002002000037824000e1890009e189000fd
:108abc00e405020001000000001f9800111f98003f
:108acc000e1890009e1890003017980041179800cf
:108adc002e009000cf80de008c050200010000000b
:108aec00201f9800311f98002e0090000000e0001d
:108afc0008003d0002002000037824002e1890008e
:108b0c00be189000e405020001000000201f980030
:108b1c00311f98002e189000be1890005017980026
:108b2c00611798001e009000cf80de008c050200bb
:108b3c0001000000401f9800511f98001e0090007b
:108b4c000000e00008003d00020020000378240033
:108b5c004e189000de189000e405020001000000a1
:108b6c00401f9800511f98004e189000de1890007e
:108b7c00700f9800011798001e007800cf80de005f
:108b8c008c05020001000000601f9800711f980006
:108b9c001e00e00008003d000200200003782400c5
:108bac006e189000fe189000e40502000100000011
:108bbc00601f9800711f98006e189000fe189000ae
:108bcc0010179800211798003e119000ce119000bc
:108bdc005e109000ee109000e20502000100000013
:108bec000001be0000002000016824009e06020067
:108bfc0001000000500f9800610f98007e09900052
:108c0c008e1190001e109000ae109000e205020034
:108c1c00010000000001be000000200001682400db
:108c2c009e06020001000000300f9800410f9800d2
:108c3c000000eb00000f9800090037000e089000b0
:108c4c008000400020802000808040000000eb006d
:108c5c00800878000e0890000000e800000f9800d3
:108c6c008e0890003e009000808f5000f3ff39007a
:108c7c00ae0090003e0090000080500070079800fd
:108c8c000000eb00000f9800160037000e08900053
:108c9c00cf80de008c050200010000005e09900010
:108cac00ee09900022070200010000008a07020072
:108cbc0001000000500798008e0890003e009000c4
:108ccc000080400080004000208020000080400098
:108cdc00de009000010878000e0890000000e8000b
:108cec00000f98008e0890007e009000808f50003e
:108cfc00e6ff35002e009000000f980009003700a9
:108d0c000e08900080004000208020000080400071
:108d1c00de009000010878000e0890000000e800ca
:108d2c00000f98008e0890001e009000808f50005d
:108d3c00f3ff39005e009000400798001e00900081
:108d4c001e001000700798000000eb00000f980048
:108d5c00180037000e089000cf80de008c05020052
:108d6c00010000003e099000ce099000220702008d
:108d7c00010000008a070200010000005007980063
:108d8c008e0890001e00900000814000de009000d4
:108d9c004e00900080814000820041002080200025
:108dac0000804000030878000e0890000000e800e6
:108dbc00000f98008e0890007e009000808f50006d
:108dcc00e4ff35009e007800010f98000900370081
:108ddc000e08900080004000208020008080400021
:108dec00f0ff2700800878000e0890000000e800d3
:108dfc00000f98008e089000f03f2000808f5000ec
:108e0c00f3ff3400780037007e109000801f78004c
:108e1c0060662900801f7800b26202000100000029
:108e2c00e48757001e007800cf80de008c0502001e
:108e3c000100000000279800112798001e00e00098
:108e4c0008003d0002002000037824000e20900052
:108e5c009e209000e405020001000000002798000d
:108e6c00112798000e2090009e209000501798001b
:108e7c00611798001e009000cf80de008c05020068
:108e8c000100000020279800312798001e00900058
:108e9c000000e00008003d000200200003782400e0
:108eac002e209000be209000e4050200010000007e
:108ebc0020279800312798002e209000be2090008b
:108ecc0030179800411798003e119000ce11900079
:108edc005e109000ee109000e20502000100000010
:108eec000001be0000e02f00f16f24009e0602007e
:108efc0001000000500f9800610f98005e0990006f
:108f0c00ee0990003e109000ce1090002207020057
:108f1c0001000000100f9800210f98000000eb00da
:108f2c00000f98002c0037008e0890003e00900037
:108f3c00808f5000030031000000eb0050079800b8
:108f4c001c0037008e0890001e009000808f50008f
:108f5c00030031000000eb005007980015003700ab
:108f6c000e0890009e0f500003003600f0ff270003
:108f7c00500798000f0037000e089000cf80de00dd
:108f8c008c050200010000005e099000ee099000c3
:108f9c0022070200010000001e099000ae0990009b
:108fac00e2050200010000008a0702000100000037
:108fbc00500798000e089000800040002080200090
:108fcc0000804000de009000010878000e08900040
:108fdc000000e800000f98008e089000f03f200081
:108fec00808f5000d0ff34007e10900045fe0700ab
:108ffc000080fa00000006000e00fa00881f7800be
:10900c0010079800640047000108780012009800cf
:10901c002300980034009800450098000040eb00b5
:10902c00004f78001e009000801f7800d067290048
:10903c00801f7800b262020001000000e487570034
:10904c006400470010007800801f780050692900e8
:10905c00801f7800b262020001000000e487570014
:10906c006400470010009000801f7800e069290020
:10907c00801f7800b262020001000000e4875700f4
:10908c006400470020009000801f7800906a29003f
:10909c00801f7800b262020001000000e4875700d4
:1090ac006400470030009000801f7800506b29004e
:1090bc00801f7800b262020001000000e4875700b4
:1090cc00e06b2900801f7800b262020001000000f2
:1090dc008f87e90064004700004890000080fb0087
:1090ec00610060000004e00005003200806c290083
:1090fc00801f7800b2620200010000008f87e90037
:10910c0064004700004890000080fb000000d10084
:10911c00610060000004e00005003200e06c2900f2
:10912c00801f7800b2620200010000008f87e90006
:10913c0064004700004890000080fb004200de0005
:10914c00610060000004e00005003200806d290021
:10915c00801f7800b2620200010000008f87e900d6
:10916c0064004700004890000080fb004300de00d4
:10917c00610060000004e00005003200106e290060
:10918c00801f7800b2620200010000008f87e900a6
:10919c0064004700100478001e009000142902009f
:1091ac0001000000800f54000700320010c0b30013
:1091bc00004f780064004700900078001e0090007b
:1091cc001428020001000000640047001004900005
:1091dc001e0090001e2b020001000000800f5400a6
:1091ec000700320010c0b300004f78006400470045
:1091fc00900090001e0090001e2a0200010000004a
:10920c0064004700200490001e009000282d0200ee
:10921c0001000000800f54000700320010c0b300a2
:10922c00004f780064004700a00090001e009000e2
:10923c00282c02000100000064004700300490005c
:10924c001e009000322f020001000000800f54001d
:10925c000700320010c0b300004f780064004700d4
:10926c00b00090001e009000322e020001000000a1
:10927c0064004700004c90001e009000d2300200a9
:10928c0001000000804f54000b00320064004700c6
:10929c00804890001e0090003c300200010000004d
:1092ac001e0190006400470080489000600c210073
:1092bc0000004100014878001e04e0000700320065
:1092cc00b06e2900801f7800b2620200010000001d
:1092dc008f87e9001e009000c4fd07004f04780042
:1092ec000080fa00000006000000fa000080fa007e
:1092fc00000006000000fa000400070072340200af
:10930c00010000000080fa00000006000000fa00d6
:10931c000000eb00b08f88000000eb00c08f8800cd
:10932c0010002000d08f88000080fa00000006009a
:10933c000400fa00000f7800110798001e00780056
:10934c004800de00804078001e0090000148780044
:10935c001e0090008000e8001e0078008048780015
:10936c000080fa00000006000400fa0010079800c4
:10937c001e009000104078000080fb004800dd00cb
:10938c00000f78001e0090000000e80010407800ec
:10939c000080fb001e0f40001e0078000080fa00c9
:1093ac00000006000600fa00881f7800b08f8000cd
:1093bc000000e00006003200b08f8000904090006a
:1093cc0000c8b30000c060000004e00039013a009e
:1093dc00b0cab30001f3b700d0ccb30002f3b700ae
:1093ec0030c4b30003f3b70010c2b30004f3b700ea
:1093fc0003c4b300f22f210011c0b30010c0b3009e
:10940c00a235020001000000c08f880003c4b30025
:10941c00f22b21008040eb0010c0b300a2350200fb
:10942c0001000000b08f8800bfd2bf002047980019
:10943c002e4090000004e0001e013200c0d2bf009c
:10944c00e64f40001b013a00112c2100914078009e
:10945c00a0cdb30080cf500016013a00212c210082
:10946c0091407800a0cbb30080cf500011013a009e
:10947c00312c210091407800a0cbb30080cf50005c
:10948c000c013a00c5d2bf0093f3b700c4d2bf00a1
:10949c00104798001e4090000000fb002007980029
:1094ac0030022000ae009000808f5000c3003200cc
:1094bc0030022000ae009000808f500012003c0063
:1094cc002e009000fe0f5000fa003200ae0090000b
:1094dc00fe8f500004003c002e009000ea0f50005c
:1094ec00d7003200f3003700ae009000ff8f500021
:1094fc001b00320010022000ae009000808f500044
:10950c0062003200eb00370060022000ae009000d9
:10951c00808f5000c700320060022000ae00900027
:10952c00808f500005003c0040022000ae009000ef
:10953c00808f500089003200de003700800220004e
:10954c00ae009000808f5000c0003200a0022000be
:10955c00ae009000808f5000c9003200d50037005b
:10956c0000c2b30005f3b700683021000000eb0027
:10957c002c59020001000000880078006cff0700e5
:10958c0088302100100020002c590200010000003e
:10959c008800780066ff0700a8302100200020001a
:1095ac002c590200010000008800780060ff0700c1
:1095bc00c8302100300020002c59020001000000ae
:1095cc00880078005aff0700e83021004000200096
:1095dc002c590200010000008800780054ff07009d
:1095ec0008312100500020002c590200010000001d
:1095fc00880078004eff0700283121006000200011
:10960c002c590200010000008800780048ff070078
:10961c0048312100700020002c590200010000008c
:10962c008800780042ff0700c0d0bf0016f3b700d7
:10963c00c1d0bf0017f3b700c2d0bf0018f3b700fa
:10964c00c3d0bf0019f3b700c4d0bf001af3b700e2
:10965c00c5d0bf001bf3b700a09e80001cf3b70061
:10966c00b09e80001df3b700c09e80001ef3b700b3
:10967c00d09e80001ff3b700e09e800020f3b7005f
:10968c0010c0b30000f3b7008a0037002c6302004f
:10969c0001000000c5d2bf000080fb000040880024
:1096ac0020c2b30005f3b7000040800006f3b700fa
:1096bc0000408000d23002000100000007f3b70028
:1096cc008830210000408000c859020001000000d1
:1096dc008800780016ff0700a830210000408000a9
:1096ec002c590200010000008800780010ff0700d0
:1096fc00c830210000408000142902000100000045
:10970c00880078000aff0700e83021000040800044
:10971c001e2b0200010000008800780004ff0700e7
:10972c000831210000408000282d020001000000bb
:10973c0088007800fefe07002831210000408000e0
:10974c00322f02000100000088007800f8fe0700ac
:10975c0010c0b30000f3b700560037002c630200b2
:10976c0001000000c5d2bf000080fb000040880053
:10977c0050c2b30005f3b7000040800006f3b700f9
:10978c007830210000408000c85902000100000020
:10979c0088007800e6fe0700983021000040800029
:1097ac002c5902000100000088007800e0fe070040
:1097bc0010c0b30000f3b7003e0037002c6302006a
:1097cc0001000000c5d2bf000080fb0000408800f3
:1097dc00c6d2bf000af0b700702c2100e2fe0700d1
:1097ec0010808800902c2100dffe0700208088006c
:1097fc00b02c2100dcfe070030808800d02c21002a
:10980c00d9fe070040808800004080001180800055
:10981c00228080003380800044808000558080004e
:10982c00024802000100000010c0b300bef2b700f5
:10983c00200037000040eb0000f3b7001d0037009c
:10984c0010c0b300bef2b7001a0037002c63020040
:10985c000100000090c2b30005f3b70000a1800026
:10986c0006f3b7000040eb0007f3b70095d3bf0039
:10987c0008f3b70010c0b30000f3b7000d003700b9
:10988c002c63020001000000c5d2bf00004f78001d
:10989c001e80fb0000a18800612c21009140780003
:1098ac00014f78001e40780095f3b70010c0b3004c
:1098bc00bef2b7004f0478000080fa0000000600ea
:1098cc000400fa00000f7800110798001e007800c1
:1098dc00804078001e009000014878001e00900027
:1098ec008000e8001e0078004800de008048780008
:1098fc000080fa00000006000000fa00881f7800c3
:10990c00c0d0bf00fff2b700c1d0bf0000f3b7005a
:10991c00c2d0bf0001f3b700c3d0bf0002f3b70041
:10992c00c4d0bf0003f3b700c5d0bf0004f3b70029
:10993c00a09e800005f3b700b09e800006f3b70030
:10994c00c09e800007f3b700d09e800008f3b700dc
:10995c00e09e800009f3b70000c0eb000af3b700eb
:10996c0000c0eb000bf3b70000c0eb000cf3b7002a
:10997c0000c0eb000df3b70000c0eb000ef3b70016
:10998c00f83021000000eb002c590200010000000f
:10999c0088007800caff0700183121001000200051
:1099ac002c5902000100000088007800c4ff070059
:1099bc0038312100200020002c5902000100000049
:1099cc0088007800beff07005831210030002000cd
:1099dc002c5902000100000088007800b8ff070035
:1099ec0078312100400020002c59020001000000b9
:1099fc0088007800b2ff0700983121005000200049
:109a0c002c5902000100000088007800acff070010
:109a1c00b8312100600020002c5902000100000028
:109a2c0088007800a6ff0700d831210070002000c4
:109a3c002c5902000100000088007800a0ff0700ec
:109a4c004f0478000080fa00000006000000fa00c5
:109a5c00881f7800c0d0bf00fff2b700c1d0bf0094
:109a6c0000f3b700c2d0bf0001f3b700c3d0bf00f2
:109a7c0002f3b700c4d0bf0003f3b700c5d0bf00da
:109a8c0004f3b700a09e800005f3b700b09e8000e1
:109a9c0006f3b700c09e800007f3b700d09e80008d
:109aac0008f3b700e09e800009f3b70000c0eb009c
:109abc000af3b70000c0eb000bf3b70000c0eb00db
:109acc000cf3b70000c0eb000df3b70000c0eb00c7
:109adc000ef3b700f83021000000eb002c59020007
:109aec00010000008800780075ff07001831210084
:109afc00100020002c5902000100000088007800a2
:109b0c006fff070038312100200020002c59020083
:109b1c00010000008800780069ff0700583121001f
:109b2c00300020002c590200010000008800780051
:109b3c0063ff070078312100400020002c590200ff
:109b4c0001000000880078005dff070098312100bb
:109b5c00500020002c590200010000008800780001
:109b6c0057ff0700b8312100600020002c5902007b
:109b7c00010000008800780051ff0700d831210057
:109b8c00700020002c5902000100000088007800b1
:109b9c004bff07004f0478000080fa00000006001d
:109bac000200fa00000f7800009a80000000e0002c
:109bbc0036003a00c0082000009a8800c08f800050
:109bcc000000e00006003200c08f80009040900042
:109bdc0000c8b30000c060000004e0002b003a0095
:109bec00100020009e0f100011003a0042ff0700e9
:109bfc00e28f8000f38f8000009f24002100200062
:109c0c00800f5100818f5900190034006000b8009a
:109c1c00e08f8800f18f8800609e2900801f7800fb
:109c2c00b2620200010000008f87e90010003700cb
:109c3c0086ff0700e28f8000f38f8000009f2400d6
:109c4c0021002000800f5100818f59000800340042
:109c5c006000b800e08f8800f18f8800a09e29007a
:109c6c00801f7800b2620200010000008f87e900bb
:109c7c0003c2b300f22f210011c0b30010c0b30017
:109c8c00a235020001000000c08f8800009a8000fd
:109c9c000000e900009a88000080fa00000006002d
:109cac000000fa000080fa00000006000000fa0034
:109cbc000080fa00000006000000fa000080fa00a4
:109ccc00000006000000fa000080fa000000060008
:109cdc000000fa003e670200010000000080fa005c
:109cec00000006000000fa000080fa0000000600e8
:109cfc000000fa00d1c1b30010c0b30078350200e7
:109d0c000100000003c4b300f22b21008040eb00e3
:109d1c0010c0b300a235020001000000b08f880013
:109d2c000080fa00000006000000fa00f09b8000a2
:109d3c00e10f500019003a00e09b8000e10f500049
:109d4c0016003a00d9ff07008824a9000000eb0098
:109d5c00e09b880000e12000e0958800e095800001
:109d6c000000e900e0958800e09580000000e0002c
:109d7c00faff3a009444a80080702000e095880017
:109d8c00e09580000000e900e0958800e0958000f7
:109d9c000000e000faff3a009444a9000080fa00a9
:109dac00000006000800fa00000f78001107980068
:109dbc00220798001e00780030079800200720002a
:109dcc00be009000808f50002c0032002007200035
:109ddc00be009000808f50000a003c003e009000b6
:109dec00e20f500020003200be009000e38f5000c4
:109dfc001f0032003e009000e10f500018003200ae
:109e0c001e00370040072000be009000808f5000dd
:109e1c001100320040072000be009000808f5000df
:109e2c000900350050072000be009000808f5000c4
:109e3c0007003200f0ff2700be009000808f50001a
:109e4c000d0032000d0037009bff07000b003700a0
:109e5c0093ff07000900370094ff07000700370045
:109e6c00a3ff0700050037009eff07000300370023
:109e7c0097ff07000100370092ff07001000200039
:109e8c000080fa00000006000000fa000c37020007
:109e9c0001000000d09b8000ff0f5000180036001e
:109eac0088c4bf00624060000004e0000100320082
:109ebc0013003700e08f8000f18f800061004000bc
:109ecc00e0804800e08f8800f18f880092d3bf00bb
:109edc00e14f500003003a001000200030ff070053
:109eec000700370092d3bf00e24f500003003a0046
:109efc000000eb002aff07000100370029fd0700d6
:109f0c000080fa00000006000000fa00f9fc0700cf
:109f1c000080fa00000006000200fa000000eb00ce
:109f2c00000f7800240037001e00780080004000ed
:109f3c00403d210000804000100178001e00780098
:109f4c0080004000e03d21000080400010007800bf
:109f5c00800f5100170032001e0178001e0078009f
:109f6c0080004000403d21000080400090017800be
:109f7c0082004100e03d2100008040000308780091
:109f8c001e00780080004000403d21000080400011
:109f9c0010007800801f78001e007800801f780069
:109fac00209b2900801f7800b26202000100000093
:109fbc00e68757001e0fe800400020009e0f10009f
:109fcc00d9ff34000080fa00000006000200fa00fd
:109fdc00004f7800e4c2a800e4e2a800e442a80024
:109fec00e4a2a8001e04e00002003a00e4c2a900aa
:109ffc000b00370010c0b3009e4f100002003a0057
:10a00c00e4e2a9000600370020c0b3009e4f100008
:10a01c0002003a00e442a90001003700e4a2a900c2
:10a02c000080fa00000006001400fa000000eb00ab
:10a03c00000f7800e2c2bf00f04060000000eb00af
:10a04c00000f78000104e00002003a00100020002c
:10a05c00000f7800e2c2bf00684060000004e0001e
:10a06c0003003a0020002000100f98000200370077
:10a07c000000eb00100f98001e0890001e0f40000f
:10a08c00e2c2bf00614060000004e00003003a003f
:10a09c0040002000000f9800020037000000eb0089
:10a0ac00000f98000e0890001e0f4000e2c2bf0087
:10a0bc00624060000004e00003003a0080002000d1
:10a0cc0070079800020037000000eb007007980042
:10a0dc007e0090001e0f4000f2c2bf006240600084
:10a0ec000004e00003003a00000120006007980023
:10a0fc00020037000000eb00600798006e00900033
:10a10c001e0f4000f2c2bf00614060000004e0007e
:10a11c0003003a00000220005007980002003700ac
:10a12c000000eb00500798005e0090001e0f4000ee
:10a13c00eac2bf00624060000004e00003003a0085
:10a14c000004200040079800020037000000eb00dc
:10a15c00400798004e0090001e0f4000eac2bf005e
:10a16c00614060000004e00003003a000008200099
:10a17c0030079800020037000000eb003007980011
:10a18c003e0090001e0f4000dac2bf000044b20037
:10a19c000004e00003003a000010200020079800a3
:10a1ac00020037000000eb00200798002e00900002
:10a1bc001e0f4000dac2bf0001c8b30001406000ae
:10a1cc000004e00003003a00002020001007980073
:10a1dc00020037000000eb00100798001e009000f2
:10a1ec001e0f40001e0078000080fa0000000600e0
:10a1fc000600fa00000f780011079800220798005b
:10a20c001e0078001e0190006a00b9000200400098
:10a21c0080004000200121000080400010007800e8
:10a22c00e20f500004003400ae009000100020003b
:10a23c00800878000f0037001e0178009e01900006
:10a24c006a10b9000300400080004000200121008a
:10a25c0000804000100078000002e8006a10b9008d
:10a26c0003004000800040002001210000804000dd
:10a27c00040878000080fa00000006000600fa00ce
:10a28c00000f780011079800220798001e00780034
:10a29c001e0190006a00b9000200400080004000de
:10a2ac002001210000804000100078000000e00038
:10a2bc0004003c00ae0090000000eb008008780029
:10a2cc000f0037001e0178009e0190006a10b90043
:10a2dc00030040008000400020012100008040006d
:10a2ec00100078000002e9006a10b9000300400079
:10a2fc00800040002001210000804000040878000c
:10a30c000080fa00000006000e00fa00100798000a
:10a31c0021079800320798004307980054079800cb
:10a32c00650798009e0090003e00900080806000c1
:10a33c003e009000808f500005003a000e0178001e
:10a34c00ce0090002e009000a9ff070004003700fb
:10a35c000e017800ce0090002e009000c7ff070081
:10a36c001e0078000000e0000d003200de019000bd
:10a37c005e00900080004000403d210000804000c5
:10a38c00900078006e009000008170008380410086
:10a39c00403d210000804000020878000e0037008c
:10a3ac00de0190005e00900080004000403d2100e6
:10a3bc0000804000100178006e0090000080ea00e0
:10a3cc008180ea000001610083804100403d210052
:10a3dc0000804000020878000080fa0000000600af
:10a3ec000400fa00100798000000eb00000f780042
:10a3fc000dff0700000f7800f03f20001e0f6000db
:10a40c001e0090000000e00047003a0015002000fc
:10a41c000002eb008001eb00120020009e00900077
:10a42c001e007800b8ff0700250020000002eb009a
:10a43c0013002000220020009e0090001e007800d7
:10a44c00b1ff0700450020000002eb0023002000b4
:10a45c00420020009e0090001e007800aaff07001a
:10a46c00850020000002eb00330020008200200059
:10a47c009e0090001e007800a3ff0700050120003d
:10a48c000002eb0043002000020120009e0090001f
:10a49c001e0078009cff0700050220000002eb0064
:10a4ac0053002000020220009e0090001e00780045
:10a4bc0095ff0700050420000002eb00630020005c
:10a4cc00020420009e0090001e0078008eff070002
:10a4dc00050820000002eb00730020000208200099
:10a4ec009e0090001e00780087ff070015002000da
:10a4fc001400200083002000021020009e00900019
:10a50c001e00780080ff07002500200014002000aa
:10a51c0093002000022020009e0090001e00780076
:10a52c0079ff0700dd0037001e009000e10f50009e
:10a53c0047003a0045002000140020008001eb0089
:10a54c00120020009e0090001e0078006eff070095
:10a55c0085002000140020001300200022002000a1
:10a56c009e0090001e00780067ff07000501200088
:10a57c001400200023002000420020009e009000c8
:10a58c001e00780060ff0700050220001400200068
:10a59c0033002000820020009e0090001e007800f6
:10a5ac0059ff070005042000140020004300200080
:10a5bc00020120009e0090001e00780052ff070050
:10a5cc000508200014002000530020000202200087
:10a5dc009e0090001e0078004bff07001500200025
:10a5ec002400200063002000020420009e00900044
:10a5fc001e00780044ff07002500200024002000e6
:10a60c0073002000020820009e0090001e007800bd
:10a61c003dff07004500200024002000830020009f
:10a62c00021020009e0090001e00780036ff0700ec
:10a63c008500200024002000930020000220200030
:10a64c009e0090001e0078002fff0700930037003b
:10a65c001e009000e20f500047003a000501200058
:10a66c00240020008001eb00120020009e009000ce
:10a67c001e00780024ff07000502200024002000a3
:10a68c0013002000220020009e0090001e00780085
:10a69c001dff0700050420002400200023002000db
:10a6ac00420020009e0090001e00780016ff07005c
:10a6bc000508200024002000330020008200200028
:10a6cc009e0090001e0078000fff07001500200070
:10a6dc003400200043002000020120009e00900066
:10a6ec001e00780008ff0700250020003400200021
:10a6fc0053002000020220009e0090001e007800f3
:10a70c0001ff0700450020003400200063002000fa
:10a71c00020420009e0090001e007800fafe070044
:10a72c008500200034002000730020000208200067
:10a73c009e0090001e007800f3fe0700050120002b
:10a74c003400200083002000021020009e009000a6
:10a75c001e007800ecfe07000502200034002000eb
:10a76c0093002000022020009e0090001e00780024
:10a77c00e5fe0700490037001e009000e30f500073
:10a78c0046003a0005042000340020008001eb0054
:10a79c00120020009e0090001e007800dafe0700d8
:10a7ac0005082000340020001300200022002000a7
:10a7bc009e0090001e007800d3fe070015002000bc
:10a7cc004400200023002000420020009e00900046
:10a7dc001e007800ccfe070025002000440020005d
:10a7ec0033002000820020009e0090001e007800a4
:10a7fc00c5fe070045002000440020004300200057
:10a80c00020120009e0090001e007800befe070092
:10a81c00850020004400200053002000020220008c
:10a82c009e0090001e007800b7fe07000501200076
:10a83c004400200063002000020420009e009000d1
:10a84c001e007800b0fe0700050220004400200026
:10a85c0073002000020820009e0090001e0078006b
:10a86c00a9fe0700050420004400200083002000fe
:10a87c00021020009e0090001e007800a2fe07002f
:10a88c000508200044002000930020000220200036
:10a89c009e0090001e0078009bfe07000080fa00ce
:10a8ac00000006000000fa0093d3bf000004e00093
:10a8bc002300320094d3bf000004e00003003a00f0
:10a8cc0010c0b30094f3b70025000700608080002f
:10a8dc007180800061004000e0804800608088004a
:10a8ec00718088006280800073808000800c200062
:10a8fc0001002000800f5100818f59001600340098
:10a90c006000b800608088007180880080808000c2
:10a91c00aefd070080808000b1fe070080808000c3
:10a92c000000e8008080880080808000e30f5000e9
:10a93c00090034000000eb0080808800060037001e
:10a94c0094d3bf000004e000030032000b000700aa
:10a95c000040eb0094f3b7000080fa000000060002
:10a96c000000fa00e0c2a900e0e2a900e042a90060
:10a97c00e0a2a9000080fa00000006000000fa0026
:10a98c00e4c2a800e0c2a800e4e2a800e0e2a8004b
:10a99c00e442a800e042a800e4a2a800e0a2a800bb
:10a9ac000080fa00000006000000fa000040eb00f6
:10a9bc0094f3b70094d3bf0093f3b7000080fa0070
:10a9cc00000006000c00fa003007980041079800c0
:10a9dc003e009000ce0090004088de00cf80de006c
:10a9ec0010079800be0090000080eb000080600013
:10a9fc002007980020042400003b8800ae00900043
:10aa0c0000f02f00008f60001e0090009001880065
:10aa1c009e0078000000eb008008bb000500fc00e5
:10aa2c005e00900050052000303b8800a00a2000fa
:10aa3c00303b880061e7a800000000000000000027
:10aa4c000080fa00000006001000fa004007980091
:10aa5c005107980062079800730798006e019000e8
:10aa6c00fe01900000f02f00f1ff2f00001f4100ad
:10aa7c00019749004e009000de00900020079800de
:10aa8c0031079800090037002e009000be0090009e
:10aa9c00ccff07002e009000be0090000010b0000c
:10aaac000180b00020079800310798002e0090001c
:10aabc00be009000be0f5000ae8f5800f2ff350064
:10aacc000080fa00000006004c00fa0020279800d5
:10aadc00312798004227980053279800ce209000e9
:10aaec002e20900000805000100798001e0090004f
:10aafc00e30f500006003c00e0932900801f780013
:10ab0c00b2620200010000008f87e900a10037004b
:10ab1c001e00900022002000110009000200d80045
:10ab2c00100798002e209000be209000002798005f
:10ab3c00112798001e209000900188000000eb0067
:10ab4c00600798002e209000be209000809fbe00d1
:10ab5c00f0962900801f7800b2620200010000000c
:10ab6c00e68757000000eb00400798008000370094
:10ab7c000e2090001000ba00300798000e209000b4
:10ab8c001080ba0020079800be009000811f78004a
:10ab9c002e009000801f780080972900801f78007d
:10abac00b262020001000000e68757006e019000bf
:10abbc002e0090004800de00804078006e004700b8
:10abcc00017178006e0090000000e80060079800aa
:10abdc006e0190002e009000804078006e004700bf
:10abec00017178006e0090000000e800600798008a
:10abfc006e0190003e0090004800de00804078001e
:10ac0c006e004700017178006e0090000000e800b3
:10ac1c00600798006e0190003e0090008040780024
:10ac2c006e004700017178006e0090000000e80093
:10ac3c00600798000e2090009e209000620040005b
:10ac4c00e080480000279800112798001e209000f3
:10ac5c00900188006e009000f00f500041003a0007
:10ac6c000000eb005007980013003700de00900046
:10ac7c006e004700e140780000c2b30080cf500066
:10ac8c0006003400de0090006e004700e1407800c2
:10ac9c00d0c7b30080cf5000040034005e01900098
:10acac00ee004700e0c2b30000f178005e009000b7
:10acbc000000e80050079800de0090006e00900045
:10accc00808f5000e9ff35005e019000ee004700d8
:10acdc000040eb0000f178006e00470080489000c7
:10acec00014f7800ee0047000040eb0080489800d0
:10acfc006e004700801f780020982900801f780084
:10ad0c00b262020001000000e48757006e004700a9
:10ad1c009e407800014898006e0047006800400093
:10ad2c00801f780080982900801f7800b262020092
:10ad3c0001000000e48757000e2090009e20900038
:10ad4c00809fbe00f0962900801f7800b26202003e
:10ad5c0001000000e68757000000eb006007980038
:10ad6c000060fe004e0090000000e80040079800d4
:10ad7c00ce0090001e009000808f50007cff3500ac
:10ad8c00b0982900801f7800b26202000100000018
:10ad9c008f87e9000080fa00000006002400fa000a
:10adac00200f9800310f9800420f9800530f980015
:10adbc004e099000de0990002e089000be0890000d
:10adcc00000051008180590020079800310798003d
:10addc006000b800008fbe002e019000be019000f4
:10adec003000200001002000800f5100818f59009d
:10adfc0009003c00e0932900801f7800b262020039
:10ae0c00010000008f87e9006000b800600f980017
:10ae1c00710f98005b0037002e019000be0190006e
:10ae2c006118b9004f08de0001002000000041004d
:10ae3c00818049008180d1000080d30020079800d8
:10ae4c00310798002e089000be089000000f980063
:10ae5c00110f98001e089000900188006000b80047
:10ae6c0060079800710798003c0037000e089000ae
:10ae7c001000ba00500798000e0890001080ba001d
:10ae8c00400798004e009000010020001e0f40006b
:10ae9c005e9748005e0090004800de000100200034
:10aeac001e0f40005e9748005e00900001002000dd
:10aebc00f20f2000030020000002780081027800cd
:10aecc0002007800830078000001620001806200bb
:10aedc006102b80004179800151798000e10900026
:10aeec009e109000c000dd000000200000179800ac
:10aefc00111798000e1090009e1090006112b8006f
:10af0c0004179800151798000e1190009e119000d0
:10af1c0002007000838070001e0f40005e97480096
:10af2c000e0890009e08900062004000e0804800ef
:10af3c00000f9800110f98001e08900090018800d7
:10af4c000060fe006e009000fe009000610040006a
:10af5c00e080480060079800710798006e0190002f
:10af6c00fe0190002e009000be009000800f51005a
:10af7c00818f5900bdff35001e02be00640f980082
:10af8c00750f98006e089000fe0890000080fa0083
:10af9c00000006000c00fa0020079800310798000a
:10afac0042079800530798004e019000de01900074
:10afbc002e009000be00900078ff0700008fbe00ae
:10afcc001e0078000080fa00000006000c00fa0059
:10afdc0040079800510798004e009000de0090004a
:10afec0020079800310798003e00900090018800df
:10affc002e0090001000ba00100798002e00900050
:10b00c001080ba00000f78001e0090000080fa003b
:10b01c00000006000e00fa00300798004107980067
:10b02c00520798003e009000ce0090001007980048
:10b03c002107980030002400003b88002e0090006f
:10b04c00900188009e0090005e0090008008bb007c
:10b05c00f00f2000000f78001e0090001e88bb002f
:10b06c001000fc00ee00900051052000313b8800e0
:10b07c00a10a2000313b880061e7a8000000000015
:10b08c000000000061c7bf0001c8b30001406000b0
:10b09c000004e000fbff3a000000eb000080fa0027
:10b0ac00000006000200fa00004f78001e80fb0032
:10b0bc00a00188000080fa00000006000000fa00e1
:10b0cc004440a8000080fa00000006000a00fa00c4
:10b0dc002007980031079800be0090000040200027
:10b0ec00808f50000300360000402000400798007d
:10b0fc001a0037002e0090000000e00002003d0016
:10b10c000000eb00200798002e009000e70f500085
:10b11c000200340070002000200798003e009000d0
:10b12c000000400001002000008fbe002e009000a7
:10b13c0080004000803f210000804000100078001b
:10b14c00010020001e0f40005e9748001e00be004c
:10b15c00ec57020001000000400798004e009000e0
:10b16c000080fa00000006000600fa00000f7800cc
:10b17c00110798009e009000f03f2000808f500037
:10b18c0002003600f03f2000100798009e00780067
:10b19c00600c210000804000104078000080fb0013
:10b1ac004300de00610060000004e0001500320086
:10b1bc009e007800600c2100008040001040780058
:10b1cc000080fb00610060000004e000050032001c
:10b1dc00014020001e009000808050002107980044
:10b1ec00170037009e0090001e007800b7ff070084
:10b1fc0080007800f0ff2700010050002007980025
:10b20c000f0037009e007800600c21000080400089
:10b21c00104078000080fb00610060000004e0003a
:10b22c00030032001e009000200798000400370035
:10b23c009e0090001e007800a4ff070020079800d5
:10b24c002e0090000080fa00000006000600fa00b4
:10b25c00000f78001e007800200798002e00900048
:10b26c00e30f5000290032002e009000e30f500035
:10b27c000a003c002e009000e10f50001900320033
:10b28c002e009000e10f50001b003c002e0090009f
:10b29c000000e0000e003200350037002e00900058
:10b2ac00e50f5000230032002e009000e50f5000f7
:10b2bc001b0035002e009000e60f500022003200db
:10b2cc002e009000e70f50002400320028003700b9
:10b2dc00618380001e007800a3ff07001007980010
:10b2ec0025003700518380001e0078009eff070068
:10b2fc001007980020003700418380001e00780062
:10b30c0099ff0700100798001b003700318380005d
:10b31c001e00780094ff07001007980016003700f5
:10b32c00218380001e0078008fff07001007980013
:10b33c0011003700118380001e0078008aff07007f
:10b34c00100798000c003700918380001e007800d5
:10b35c0085ff07001007980007003700a1838000c5
:10b36c001e00780080ff07001007980002003700cd
:10b37c000000eb00100798001e0090000080fa00ff
:10b38c00000006000600fa00000f78001e0078008e
:10b39c00200798002e009000e30f5000230032008d
:10b3ac002e009000e30f50000a003c002e0090008d
:10b3bc00e10f5000170032002e009000e10f5000fa
:10b3cc0017003c002e0090000000e0000e00320040
:10b3dc00250037002e009000e50f500019003200b8
:10b3ec002e009000e50f5000130035002e00900049
:10b3fc00e60f5000160032002e009000e70f5000b0
:10b40c001600320018003700608380001007980087
:10b41c001700370050838000100798001400370085
:10b42c0040838000100798001100370030838000a3
:10b43c00100798000e00370020838000100798003a
:10b44c000b003700108380001007980008003700ad
:10b45c00908380001007980005003700a0838000bf
:10b46c0010079800020037000000eb00100798004e
:10b47c001e0090000080fa0000000600809fbe00b5
:10b48c00829fbe00841f78000800fa0085a0a900e6
:10b49c00001880006101b800f09d8000019e8000c2
:10b4ac000200400083804800f09d8800019e8800c7
:10b4bc00101880006101b800109e8000219e800051
:10b4cc000200400083804800109e8800219e880066
:10b4dc00319e80002018800000804000309e880043
:10b4ec00419e80003018800000804000409e880003
:10b4fc00519e80004018800000804000509e8800c3
:10b50c00619e80005018800000804000609e880082
:10b51c006018800070838800701880008083880019
:10b52c00719e80008018800000804000709e880012
:10b53c00819e80009018800000804000809e8800d2
:10b54c00a0188000b0838800b0188000c0838800e9
:10b55c00c0188000d0838800d0188000e083880059
:10b56c00e0188000f0838800f018800000848800c8
:10b57c00909e80000000e800909e8800909e8000c5
:10b58c00e70f50004f003400f09d8000019e8000ba
:10b59c00008fbe001e00be00e00f5000e08f580070
:10b5ac0004003d001e01be0067014100e08149001e
:10b5bc00028fbe001e01be004d1add004310de00de
:10b5cc0000007200c398de0010838800109e80007b
:10b5dc00219e800020079800310798002e009000d3
:10b5ec00be009000e00f5000e08f580006003d00b8
:10b5fc002e019000be01900067014100e0814900de
:10b60c0022079800330798002e019000be0190008d
:10b61c004d1add004310de0000007200c398de00fe
:10b62c0020838800309e80004300de003083880039
:10b63c00409e80004300de0040838800509e8000c6
:10b64c004300de0050838800609e80004300de00d3
:10b65c0060838800709e80004300de009083880029
:10b66c00809e80004300de00a08388000000eb0079
:10b67c00809e8800809e8000709e8800709e800056
:10b68c00609e8800609e8000509e8800509e8000c6
:10b69c00409e8800409e8000309e8800309e800036
:10b6ac0001002000109e8800219e8800109e8000c2
:10b6bc00219e8000f09d8800019e88000000eb0018
:10b6cc00909e88000080fa004f0278004f01be0067
:10b6dc004f00be00004006000000fa0011322000ae
:10b6ec0091407800c0cfb30000c0600021e3b700e8
:10b6fc00013220009140780000ceb30000c07000f1
:10b70c0020e3b7002043a8002132200091407800ac
:10b71c00c0c3b30000c0700022e3b70023c3bf0056
:10b72c007f40600023e3b7002343a800f0c3b300bd
:10b73c0024e3b70025e3a9005132200091407800a2
:10b74c0000ceb30000c060009041b30025e3b70009
:10b75c000000eb0050198800f03f20008019880091
:10b76c000000eb009019880085a0a90095a0a80006
:10b77c002003a9002023a90021e3a8000080fa00df
:10b78c0000000600619f8000808f50000200320094
:10b79c0080007800fcff3700619f880002003700b2
:10b7ac00a062020001000000ec13e200fcff3a0072
:10b7bc0000000600889fbe000004780081447800d9
:10b7cc003a110200010000006011020001000000ab
:10b7dc003a1102000100000000cab300641102001b
:10b7ec00010000003a110200010000004840de0098
:10b7fc0064110200010000003a1102000100000077
:10b80c000840780064110200010000003a110200a7
:10b81c0001000000094078006411020001000000e2
:10b82c003a11020001000000781102000100000032
:10b83c003a1102000100000090012000d1ff070026
:10b84c004f04be0000000600881f7800000478003a
:10b85c003a1102000100000060110200010000001a
:10b86c003a1102000100000000cab300641102008a
:10b87c00010000003a110200010000004840de0007
:10b88c0064110200010000003a11020001000000e6
:10b89c000840780064110200010000003a11020017
:10b8ac000100000060110200010000003a110200ca
:10b8bc000100000010cab300641102000100000076
:10b8cc003a110200010000007c110200010000008e
:10b8dc00004478003a1102000100000078110200c7
:10b8ec00010000003a110200010000000884fb0076
:10b8fc00080078004f04780000000600889fbe0006
:10b90c008a9fbe00c0862900801f7800b2620200a8
:10b91c0001000000dd82a90060012000caff0700c1
:10b92c0000447800a1c5b30060012000a1ff07000e
:10b93c0060012000c4ff0700004578008f87e900f4
:10b94c00a0c5b300804f5500080032000a80fb00f0
:10b95c00801f7800b0872900801f7800b262020037
:10b96c0001000000100020001000370051cab30085
:10b97c00600120008fff070060012000b2ff07006c
:10b98c008044780050cab30080cf540009003200c4
:10b99c000980fb00801f780090882900801f7800a8
:10b9ac00b26202000100000020002000e487570072
:10b9bc004e00370088407800600120007dff0700b2
:10b9cc00e00d2000a0ff0700804578008a40780039
:10b9dc00e00d200077ff0700e00d20009aff070024
:10b9ec00004478008a4f5000080032000080fb00b1
:10b9fc00801f780070892900801f7800b2620200d5
:10ba0c000100000030002000e8ff3700894078007a
:10ba1c00e00d200067ff0700e00d20008aff070003
:10ba2c0000457800894f500006003200508a2900ea
:10ba3c00801f7800b262020001000000400020006c
:10ba4c00290037008b407800e00d200059ff0700db
:10ba5c00e08a20007cff0700804478008840780052
:10ba6c00e08a200053ff0700e08a200076ff0700e1
:10ba7c00884f500006003200d08a2900801f7800c1
:10ba8c00b2620200010000005000200016003700d6
:10ba9c008a407800e08a200046ff0700e08a2000f8
:10baac0069ff07008a4f500006003200508b2900b6
:10babc00801f7800b26202000100000060002000cc
:10bacc000900370089407800e08a200039ff070020
:10badc00d08b2900801f7800b262020001000000a8
:10baec00dd82a8000000eb008f87e9004f05be0047
:10bafc004f04be00000006002eff070000000500ea
:10bb0c0051ff07000080fb00000006000a00fa004d
:10bb1c00881f78000004780080fb27004aff07008c
:10bb2c00c0f79f0090fb270047ff0700d0f79f004e
:10bb3c00a0fb270044ff0700e0f79f00b0fb2700a5
:10bb4c0041ff0700f0f79f00c0fb27003eff0700f6
:10bb5c0080ff9f00d0fb27003bff070090ff9f005a
:10bb6c00e0fb270038ff0700a0ff9f00f0fb270039
:10bb7c0035ff0700b0ff9f000081fb002ff89700f6
:10bb8c004800dd000100200002014000e081480077
:10bb9c001ff897000080fb0001002000c000dd00b2
:10bbac000000200002014000838148000ff897003c
:10bbbc000080fb0001002000c800dd000000200018
:10bbcc00801f4100819f4900208d2900801f780033
:10bbdc007280570010f2020000000000f280570043
:10bbec0001007800d4f1020000000000e687570045
:10bbfc00e40f50000a0036006c81570080004100b1
:10bc0c00e4805000420020000800780032f202006c
:10bc1c00000000000040eb00404498000400370096
:10bc2c00618d29000800780054f202000000000029
:10bc3c00080078004f0478000080fa00000006002d
:10bc4c000c00fa00889fbe008a1f78000004780060
:10bc5c006c8557000a007800acff07007280570013
:10bc6c00aaff070072805700800078000a00780055
:10bc7c0064f2020000000000800478000000e00084
:10bc8c00f3ff3a00420020008a0078000800780098
:10bc9c0032f20200000000004944980008007800cd
:10bcac004f0578004f04be000080fa00000006002b
:10bcbc00dd82a80017e2a90020022000a010880055
:10bccc00000a2000d01088001902a9001722a90030
:10bcdc008a40a90017e2a800000006000c00fa0038
:10bcec0030079800410798003e0090006500400026
:10bcfc00200798003e009000650050001007980047
:10bd0c004e009000000f78002e0090009e0f100047
:10bd1c0003003c001e0090009e0f100003003d002d
:10bd2c001000200050079800020037000000eb00c4
:10bd3c00500798005e0090000080fa00000006009a
:10bd4c000000fa0061838000109d8000e3ff070073
:10bd5c000004e0000900320060838000109d880020
:10bd6c0060838000801f7800007c2900801f780091
:10bd7c00b262020001000000e4875700518380008a
:10bd8c00009d8000d5ff07000004e0000900320090
:10bd9c0050838000009d880050838000801f7800b5
:10bdac00b07c2900801f7800b26202000100000004
:10bdbc00e487570041838000f09c8000c7ff070098
:10bdcc000004e0000900320040838000f09c8800f1
:10bddc0040838000801f7800607d2900801f7800e0
:10bdec00b262020001000000e4875700318380003a
:10bdfc00e09c8000b9ff07000004e000090032005d
:10be0c0030838000e09c880030838000801f7800a5
:10be1c00107e2900801f7800b26202000100000031
:10be2c00e487570021838000d09c8000abff070083
:10be3c000004e0000900320020838000d09c8800c0
:10be4c0020838000801f7800c07e2900801f78002e
:10be5c00b262020001000000e487570011838000e9
:10be6c00c09c80009dff07000004e0000900320028
:10be7c0010838000c09c880010838000801f780095
:10be8c00707f2900801f7800b26202000100000060
:10be9c00e487570091838000409d80008fff07004e
:10beac000004e0000900320090838000409d88006f
:10bebc0090838000801f780020802900801f7800ec
:10becc00b262020001000000e4875700a1838000e9
:10bedc00509d800081ff07000004e0000900320043
:10beec00a0838000509d8800a0838000801f780074
:10befc00d0802900801f7800b2620200010000008f
:10bf0c00e48757000080fa00000006000400fa00e5
:10bf1c00609c8000100798001e009000e20f5000fb
:10bf2c006f0032001e009000e20f500007003c0032
:10bf3c001e0090000000e0000b0032001e0090007c
:10bf4c00e10f500038003200a40037001e009000b2
:10bf5c00e30f5000980032001e009000e40f5000d8
:10bf6c009c0032009d0037000040eb001a63020079
:10bf7c000100000010c0b3001a61020001000000b3
:10bf8c000040eb00066102000100000030062000ba
:10bf9c00e2f102000000000010c0b30024f4b7006e
:10bfac0030002000609c880080382100709c880044
:10bfbc005e5e02000100000080812900801f780075
:10bfcc00b2620200010000008f87e900ca32020051
:10bfdc00010000007a49020001000000725b0200bf
:10bfec00010000004863020001000000809c8800f2
:10bffc00809c8000819c8000801f7800811f7800cd
:10c00c0020822900801f7800b2620200010000002b
:10c01c00e687570080630200010000008a4f02008f
:10c02c00010000006d00370070832900801f78002c
:10c03c00b2620200010000008f87e900200020009e
:10c04c00609c88000040eb001a61020001000000b7
:10c05c00da540200010000007869020001000000bf
:10c06c005e320200010000000080fb0000a188008d
:10c07c0010c0b30022f4b7007e32020001000000b1
:10c08c00004f78001e80fb00610060000004e0009f
:10c09c000800320000842900801f7800b262020080
:10c0ac00010000008f87e90010c0b30093f3b700c4
:10c0bc000700370000852900801f7800b26202005b
:10c0cc00010000008f87e9000040eb0093f3b700fc
:10c0dc0010c0b3001a630200010000003f003700db
:10c0ec00f1a0800000a18000808f5000050032007c
:10c0fc0000a18000f0a0880000a180004e32020058
:10c10c0001000000613921009140780095d3bf00f7
:10c11c0080cf50002100320095d3bf0096f3b700ba
:10c12c0095d3bf000080fb00801f7800f0852900ac
:10c13c00801f7800b262020001000000e487570003
:10c14c0095d3bf006e3202000100000095d3bf00f2
:10c15c000080fb00610060000004e0000800320079
:10c16c0000842900801f7800b262020001000000e8
:10c17c008f87e90010c0b30093f3b70007003700b6
:10c18c0000852900801f7800b262020001000000c7
:10c19c008f87e9000040eb0093f3b700d422020034
:10c1ac00010000004a4f0200010000005854020038
:10c1bc000100000009003700709c80000000e000c6
:10c1cc0006003a0024d4bf000000fb00609c8800ed
:10c1dc00020037000000eb00609c8800a0620200a7
:10c1ec00010000000080fa00000006000000fa00c8
:10c1fc000000eb00609c88000080fa000000060044
:10c20c000200fa00004f7800d8a2a800d862a8005b
:10c21c001e04e00002003200d8a2a900dca2a90092
:10c22c000080fa00000006000200fa00004f7800bf
:10c23c00d8a2a800d862a8001e04e00002003200b8
:10c24c00d862a900dc62a9000080fa000000060098
:10c25c000000fa00a09d2900801f7800be00070096
:10c26c008f87e9000000eb00a0088800803e2000ca
:10c27c00d008880000012a00f00888008760a90017
:10c28c009760a8001fe1a8000080fa0000000600db
:10c29c0000a0fe003600f800849fbe00869fbe0002
:10c2ac003400f80024002000a40188000000fa00eb
:10c2bc008760a900f2d3bf000004e0001500320033
:10c2cc0050a080000000e80050a0880051a0800021
:10c2dc0040062000808f50000e0034000000eb0060
:10c2ec0050a088000cd4bf000004e0000500320010
:10c2fc000040eb000cf4b7000cd4bf00caff0700e1
:10c30c000400370010c0b3000cf4b7000cd4bf000d
:10c31c00c5ff070040a080000000e00003003200d1
:10c32c0040a080000000e90040a08800709c8000c4
:10c33c000000e00003003200709c80000000e90067
:10c34c00709c8800609f80000000e00003003200b9
:10c35c00609f80000000e900609f880070a0800052
:10c36c000000e0000a00320070a080000000e9002c
:10c37c0070a0880070a08000e10f500004003a000b
:10c38c000040eb00a8ff07000000eb0070a0880045
:10c39c0010c0b300e8f3b7000080fa003400f900d5
:10c3ac004f03be004f02be003600f9000080fe00b5
:10c3bc00004006003400f800881f78002800200098
:10c3cc00a80188004f0478000000fa008660a900dc
:10c3dc000080fa003400f900004006000600fa0064
:10c3ec00200798000000eb00100798000e003700a3
:10c3fc000000eb00000f7800050037001e009000d5
:10c40c001e004000209188000060fe001e0fe80016
:10c41c00309c20009e0f1000f8ff34001e0090008e
:10c42c000000e800100798009e0090002e0090007d
:10c43c00808f5000eeff35000080fa0000000600ef
:10c44c000200fa00000f78001e00780040a088005f
:10c45c00010037003700070040a080000000e0001a
:10c46c00fcff3a000080fa00000006003400f800df
:10c47c00881f780028002000a80188004f0478004d
:10c48c000000fa0081e0a9000080fa003400f900f5
:10c49c00004006003400f800881f780028002000b7
:10c4ac00a80188004f0478000000fa008020a90041
:10c4bc000080fa003400f900004006003400f80057
:10c4cc00881f780028002000a80188004f047800fd
:10c4dc000000fa008060a9000080fa003400f90026
:10c4ec00004006003400f800881f78002800200067
:10c4fc00a80188004f0478000000fa008040a900d1
:10c50c000080fa003400f900004006003400f80006
:10c51c00881f780028002000a80188004f047800ac
:10c52c000000fa008080a9000080fa003400f900b5
:10c53c00004006000000fa00e8d3bf000004e00051
:10c54c00030032000060fe000040eb00e8f3b7008f
:10c55c000080fa00000006000600fa00f3d3bf00ca
:10c56c000004e0002100320068005700000f780042
:10c57c004eb89700800078001e01780060222100e0
:10c58c00b6f102000000000060222100d4f102008c
:10c59c0000000000200798000000eb001007980036
:10c5ac000e00370023c2bf00624060000004e000b0
:10c5bc00fcff3a009e0090006022210000804000a9
:10c5cc00104078000000fb0020118800d9ff070004
:10c5dc001e0090000000e800100798009e009000dc
:10c5ec002e009000808f5000eeff35000080fa0086
:10c5fc00000006000200fa00dac2bf0070406000c2
:10c60c000004e000030032000000eb00000f780093
:10c61c000200370010002000000f78001e00780088
:10c62c000080fa00000006000200fa00004f7800bb
:10c63c001e04e00002003200ec62a800010037008a
:10c64c00ec62a9000080fa00000006000000fa006d
:10c65c0010c0b300f4fe07004006200070a0880054
:10c66c000080fa00000006000000fa000040eb0019
:10c67c00e8f3b7000040eb00f2f3b7000080fa00db
:10c68c00000006000400fa00bc32020001000000a9
:10c69c0030479800ae32020001000000204798009d
:10c6ac002e4090008080fb003e4090000080fb00fc
:10c6bc00811f7800801f7800206f2900801f780070
:10c6cc00b262020001000000e68757003e40900075
:10c6dc000080fb00000f78002e4090000080fb00d3
:10c6ec004800dd001e0f40001e0078000080fa009c
:10c6fc00000006000200fa0030c0b3002cf1b700b5
:10c70c0030c0b3002df1b700904020007089880034
:10c71c0070c1b30030f1b70030c0b30031f1b700d5
:10c72c00200420009089880050072000a0898800f0
:10c73c0070062000b089880050062000c08988004f
:10c74c0090072000d089880050062000e0898800de
:10c75c0000022000f089880040052000008a880033
:10c76c0050062000108a880030062000208a88009d
:10c77c0080062000308a8800e0062000408a88006d
:10c78c00f0062000508a8800c0062000608a8800cd
:10c79c00f0062000708a880070062000808a8800cd
:10c7ac0090072000908a880000022000a08a880050
:10c7bc0090042000b08a8800e0062000c08a88001f
:10c7cc0030062000d08a8800e0022000e08a880031
:10c7dc000000eb00000f78000c0037001e01780001
:10c7ec009e007800e00c2100008040001040780092
:10c7fc008001fb00020041008080e800e015210070
:10c80c0000804000030878001e0fe800f0012000b3
:10c81c009e0f1000f1ff340030c0b3005ff1b70081
:10c82c0010c2b3005ef1b70020c1b3001af1b7001b
:10c83c0010c0b3001bf1b7001cd1bf0060406000fa
:10c84c001cf1b7001dd1bf00604060000014a000b7
:10c85c001df1b7000040eb001ef1b7000040eb00eb
:10c86c001ff1b7000040eb0020f1b70080c0b3000f
:10c87c0021f1b70022d1bf006040600051c7b30066
:10c88c000140700022f1b70023d1bf00604060006e
:10c89c0041c3b3000140700023f1b700829c8000bb
:10c8ac00f00f20008000610024d1bf0060406000c8
:10c8bc000140700024f1b700c810de0025d1bf0084
:10c8cc00604060000140700025f1b70026d1bf0028
:10c8dc00604060000014a00026f1b70027d1bf0013
:10c8ec006040600027f1b70010c0b30028f1b7001a
:10c8fc0020c0b30029f1b7000040eb002af1b700cb
:10c90c0010c0b3002bf1b70090c0b300f0f0b7002b
:10c91c0020c0b300f1f0b70090c2b300f2f0b70042
:10c92c000040eb00f3f0b70010c0b300f4f0b70018
:10c93c0010c0b300f5f0b7000040eb00f6f0b70004
:10c94c0000ccb300f7f0b700a0cfb300f8f0b700fd
:10c95c0090c0b300f9f0b70040c0b300faf0b700d4
:10c96c000040eb00fbf0b7000040eb00fcf0b70020
:10c97c0020c0b300fdf0b70030c0b300fef0b7002c
:10c98c000040eb00fff0b7000040eb0000f1b700f7
:10c99c000040eb0001f1b70090c0b30002f1b7000a
:10c9ac0010c2b30003f1b70010c1b30004f1b7001b
:10c9bc0010c0b30005f1b7000040eb0006f1b70062
:10c9cc0010c0b30007f1b70020c2b30008f1b700e4
:10c9dc0092d3bf00e14f50000a003a00c0c3b3002d
:10c9ec0009f1b7000040eb000af1b700c07929004b
:10c9fc00801f7800b2620200010000008f87e900fe
:10ca0c001600370092d3bf00e24f50000a003a00e4
:10ca1c00c0c3b30009f1b7000040eb000af1b70046
:10ca2c00707a2900801f7800b262020001000000b9
:10ca3c008f87e90009003700c0c1b30009f1b700c6
:10ca4c000040eb000af1b700207b2900801f780022
:10ca5c00b2620200010000008f87e90070c0b300d1
:10ca6c000bf1b70050c0b3000cf1b70010c8b30005
:10ca7c000df1b70030c0b3000ef1b70000c4b30025
:10ca8c000ff1b7000040eb0010f1b70010c0b3007d
:10ca9c0011f1b70070c0b30012f1b70050c0b30071
:10caac0013f1b70010c0b30014f1b70030c0b300dd
:10cabc0015f1b70000c4b30016f1b7000040eb004d
:10cacc0017f1b70010c0b30018f1b7000080fa00de
:04cadc000000060050
:020000040000fa
:020000040002f8
:10cae0001814000006000000020000000000000012
:10caf000000000009e11000058000000000000002f
:10cb0000e8130000100000000000000008140000fe
:10cb1000080000000200000000000000000000000b
:10cb200000000000201200009c0000000000000037
:10cb300024140000020000000200000000000000b9
:10cb40008c1300002c0000000000000010140000f6
:10cb50000800000002000000f0102c00113011004d
:10cb60005e110000f0100000ae00000000000000a8
:10cb7000261400000200000000000000f611000072
:10cb80000a00000002000000000000000001000098
:10cb90000000000000000000bc1200008600000041
:10cba00000000000421300004a00000000000000e6
:10cbb000001200002000000000000000b813000078
:10cbc0001c00000002000000000000000000000047
:10cbd0000000000000000000000000000000000055
:10cbe0000000000000000000000000000000000045
:10cbf00062100000340000000000000096100000e9
:10cc000030000000000000000c1000005600000082
:10cc10000200000000000000000000000000000012
:10cc20000000000000000000000000000000000004
:10cc300000000000000000000000000000000000f4
:10cc400000000000000000000000000000000000e4
:10cc500000000000000000000000000000000000d4
:10cc600000000000000000000000000000000000c4
:10cc700000000000000000000000000000000000b4
:10cc80000000000000000000d413000014000000a9
:10cc900000000000f8130000100000000200000077
:10cca000007000008000900000a00000b000c000f4
:10ccb00000d00000e0000000000800000c080000a8
:10ccc00000000000c61000002a0000000000000064
:10ccd0002814000002000000020000000000000014
:10cce0001e14000006000000000000004e150000a9
:10ccf0001200000002000000010002000004000019
:10cd00000800100000000000202b2d002330000040
:10cd10006a1500000800000002000000686a6c004c
:10cd2000747a4c0000000000601500000a0000004a
:10cd300002000000000001000000000000000000f0
:10cd4000000000002a14000088000000000000001d
:10cd5000b2140000480000000200000000000000c3
:10cd60000000000024400000000000000000590006
:10cd7000400000000000000088c3400000000000e8
:10cd80000084d7009741000080e0370079c341005c
:10cd900043176e0005b5b500b8934600f5f93f009e
:10cda000e9034f00384d32001d30f900487782000a
:10cdb0005a3cbf00737fdd004f157500fa14000068
:10cdc00032000000020000004e414e00006e610083
:10cdd0006e0049004e460000696e6600003031006a
:10cde000323334003536370038396100626364000d
:10cdf0006566000030313200333435003637380094
:10ce00003941420043444500460000002c15000013
:10ce100022000000020000003031320033343500bf
:10ce2000363738003961620063646500660030009f
:10ce3000313233003435360037383900414243004f
:10ce4000444546000000000072150000020000008a
:10ce50000200000000000000741500000200000045
:10ce60000200000030000000761500000200000003
:0cce7000020000000000000000000000b4
:020000040000fa
:020000040002f8
:10ce7c000400fa004ad3bf007f406000e14f50002d
:10ce8c007a003a004ed3bf000004e00077003a006d
:10ce9c004bd3bf00e64f500040003a004dd3bf00cb
:10ceac000080fb0010079800100220009e009000ec
:10cebc00808f500005003200200220001e019000df
:10cecc00800f51000c0032003400370079d3bf00c2
:10cedc00e14f500031003a00000f21007200400079
:10ceec00009c880090002000209c880000ccb3009f
:10cefc0082f3b7002900370092d3bf00e14f5000f6
:10cf0c000c003a00e0982900801f7800b262020001
:10cf1c00010000008f87e90000762900009c880042
:10cf2c00c0032000209c880000ccb30082f3b70023
:10cf3c001a00370092d3bf00e24f50000c003a00a9
:10cf4c00a0992900801f7800b26202000100000045
:10cf5c008f87e90040722900009c8800c0032000e4
:10cf6c00209c880000ccb30082f3b7000b00370084
:10cf7c00509a2900801f7800b26202000100000064
:10cf8c008f87e90080702900009c8800c001200078
:10cf9c00209c880000ccb30082f3b7004ad3bf00ba
:10cfac0002c6b3008240600000c2b30080cf5000c4
:10cfbc002e003a004bd3bf000080fb00000f78001e
:10cfcc001e007800e30f50001d0032009e00780018
:10cfdc00e38f500007003c001e017800e10f510068
:10cfec00220032001e007800e20f500008003200d0
:10cffc001e0037009e007800ea8f50000b003200b4
:10d00c001e017800eb0f510014003200170037009e
:10d01c0060422100009c880010002000209c8800a9
:10d02c0010ccb30082f3b7001000370000c8b30077
:10d03c0082f3b7004dd3bf0026f4b7000b003700c6
:10d04c0070422100009c880010002000209c880069
:10d05c0010c8b30082f3b7000400370000c8b30057
:10d06c0082f3b7004cd3bf0027f4b7000080fa005e
:10d07c00000006000000fa008580a9000080fa007c
:10d08c00004006003600f800809fbe00829fbe0064
:10d09c00849fbe00869fbe00881f78000000fa00a7
:10d0ac008560a900c1a08000d0a08000808f5000b6
:10d0bc0004003a000000eb00d0a08800d0a0800053
:10d0cc00c0a08800c0a080000000e800c0a08800bc
:10d0dc00c1a08000f0042000808f500003003400b9
:10d0ec00c0a080000000e900c0a08800c8a080009b
:10d0fc00901002000100000080407800e01921002f
:10d10c0000004400014878000080fa004f047800c9
:10d11c004f03be004f02be004f01be004f00be00c9
:10d12c003600f900004006000200fa00c1a08000a1
:10d13c00d0a08000808f500003003200100020002f
:10d14c00000f7800020037000000eb00000f7800a1
:10d15c001e0078000080fa00000006000400fa00af
:10d16c000040eb00004f7800c1a08000d0a08000f0
:10d17c00808f500003003a001e00fb00100798003f
:10d18c0011003700d0a080008000e800e0192100d9
:10d19c000080400010407800004f7800d0a0800044
:10d1ac000000e800d0a08800d1a08000f00420008e
:10d1bc00808f5000020034000000eb00d0a08800eb
:10d1cc001e00fb00100798001e0090000080fa0063
:10d1dc00000006000200fa00a2100200010000008c
:10d1ec0070062000000f780000c02c00908f880083
:10d1fc00f0752200a08f88001e017800a18f80009e
:10d20c00908f8000ae100200010000000080eb0047
:10d21c00c2100200010000000080fa0000000600ad
:10d22c000200fa00004f780023c2bf006240600089
:10d23c000004e000fcff3a001e00fb0020118800f7
:10d24c000080fa00000006000000fa001003200025
:10d25c0018110200010000000080fa000000060016
:10d26c0000a0fe003400f800881f78002800200081
:10d27c00a80188004f0478000000fa0028d4bf00f1
:10d28c000004e000060032000040eb0028f4b70078
:10d29c00803e200070088800cd62a9000c00370089
:10d2ac0010c0b30028f4b70000a18000e30f5000b9
:10d2bc000700340000a180004300dd0070088800e6
:10d2cc0022d4bf000004e00001003200cd62a800af
:10d2dc008500a9000080fa003400f9000080fe00ef
:10d2ec00004006000000fa00c09c2900801f780056
:10d2fc00b2620200010000008f87e9000000eb0021
:10d30c0050088800803e20007008880000012a0028
:10d31c00900888008500a9009500a80013e1a800da
:10d32c000040eb0022f4b7000080fa000000060079
:00000001FF
